:020000040800F2
:10000000F84E032029AC0608016F0C08056F0C0898
:10001000116F0C08156F0C08216F0C080000000010
:1000200000000000000000000000000069700C08E3
:100030002D6F0C0800000000BD700C082F6F0C081D
:1000400047AC060847AC060847AC060847AC0608AC
:1000500047AC060847AC060847AC060847AC06089C
:1000600047AC060847AC060847AC060847AC06088C
:1000700047AC060847AC060847AC060847AC06087C
:1000800047AC060847AC060847AC060847AC06086C
:1000900047AC060847AC060847AC060847AC06085C
:1000A00047AC060847AC060847AC060847AC06084C
:1000B0003D6F0C0847AC060847AC060847AC06087D
:1000C00047AC060847AC060847AC060847AC06082C
:1000D00047AC060847AC060847AC060847AC06081C
:1000E000756F0C0847AC060847AC060847AC060815
:1000F00047AC060847AC060847AC060847AC0608FC
:1001000047AC0608B56F0C0847AC060847AC0608B4
:1001100047AC060847AC060847AC060847AC0608DB
:1001200047AC060847AC060847AC0608B96F0C0890
:1001300047AC0608BD6F0C0847AC060847AC06087C
:1001400047AC060847AC060847AC060847AC0608AB
:1001500047AC0608C16F0C0847AC0608C56F0C0811
:1001600047AC060847AC060847AC060847AC06088B
:1001700047AC0608D16F0C0847AC06080000000029
:1001800047AC060847AC060847AC060847AC06086B
:1001900047AC060847AC060847AC060847AC06085B
:1001A000ED6F0C0847AC06082D700C0847AC06082C
:1001B00047AC060847AC060847AC060847AC06083B
:1001C00047AC060847AC060810B500F0004420F024
:1001D0000040C20DC0F3160040F400007F2A02DA8E
:1001E0000020014610BD0021962A03DCC2F19602D0
:1001F000D04002E0963A6AF0CCFA002CF2D000230C
:10020000D0EB030063EB010110BD70B5C1F30A52DE
:1002100001F000450024C1F3130140F2FF3341F423
:1002200080119A4202DA0020014670BD40F2334349
:100230009A42A2F2334203DC52426AF09AFA01E097
:100240006AF0A7FA2C43F0D00023D0EB030063EB55
:10025000010170BDF0B400F0004221F0004120F037
:100260000040CE0DC30DC1F3160141F40001C0F3EF
:1002700016004C42154640F40000761E09E010EBD3
:10028000440002D582F0004240428842F7D8400044
:100290005B1EB342F9DA18B1F0BC002103F0F1BAE9
:1002A0002846F0BC704700000FF2060CDCF800C0D6
:1002B000604719DA060800000FF2060CDCF800C0EF
:1002C000604739DA060800000FF2060CDCF800C0BF
:1002D000604759DA060800000FF2060CDCF800C08F
:1002E00060479BDB0608F0B4CA17CB0F5040514063
:1002F000C61841F100054FEAC372314628004FF09D
:10030000960303D0B623F0BC03F0BBBA30460021FD
:10031000F9E73EB5CA17CB0F002450405140C01832
:100320006141DA0740F233430094CDE901232246CC
:1003300023466AF085F903B030BD000091F9004012
:100340004AF8204003F00ABFB1F900404AF82040C3
:1003500003F004BF0C884AF8204003F0FFBE000001
:100360000C684AF8204003F0F9BE0000D1E90045CE
:100370000AEB8000C0E9004503F0F0BE5AF8200007
:10038000087003F0EBBE00005AF82000088003F06C
:10039000E5BE00005AF82000086003F0DFBE000050
:1003A0000AEB8000D0E90045C1E9004503F0D6BE64
:1003B000C7F808803B6E074800689847002840F05F
:1003C000048000F0ADBA00F004B84BF8240003F04C
:1003D000C5BE00003804012002460A480068634692
:1003E0004DF8045DC7F808807D6EA84701B000286D
:1003F00040F0048000F094BA00F004B84BF82400F8
:1004000003F0ACBE38040120002940F0038003490A
:1004100000F068B9796100F083BA000060B10008AB
:10042000002B40F003800B4900F05CB95AF8221011
:100430000029C0F20C809C6803F10C03A14280F2F9
:10044000068053F821204AF8202003F087BE024995
:1004500000F048B960B10008C0B100085AF8222085
:10046000002B40F003800A4900F03CB95AF8210003
:100470000028C0F20A809C6803F10C03A04280F2BD
:10048000048043F8202003F069BE024900F02AB935
:1004900060B10008C0B1000807480068A2F0FEF98A
:1004A000B84200F00680002840F0028003F05ABEF7
:1004B000074603F04DBE0000400401205BF8200019
:1004C0000446384671F00AF94DF8040D71F00AF946
:1004D00005465DF8040B2946224671F01DF90028F7
:1004E00000F0098041464FF0030203463846B5F05C
:1004F00053F803F02DBE2C6003F030BE5BF82110E2
:10050000002940F00380104900F0ECB85BF820406F
:10051000C2F100020D464DF8042D3846224674F013
:100520006BFA002800F00A8001B041464FF0020249
:1005300003463846B5F030F803F00ABE5DF8042BE8
:10054000AC5003F00BBE000060B100085BF8225015
:10055000002840F003801A4900F0C4B85AF821C0BE
:10056000BCF1000FC0F2288083684DF8040D00EB49
:100570008C049C4580F21F80294671F0E9F8002820
:1005800040F0048001B00F4900F0ACB838465DF887
:10059000041B2A4674F030FA002800F00980414616
:1005A0004FF0010203463846B4F0F6FF03F0D0BD29
:1005B000E56003F0D3BD01B0034900F093B800003B
:1005C00060B1000820B20008C0B100084DF8041D59
:1005D00004463846694671F0D7F8002840F0038099
:1005E00001B003F0B5BD5DF8041B0D68384629461F
:1005F00074F021FA002800F0098041464FF0030210
:1006000003463846B4F0C8FF03F0A2BD4BF82450AF
:1006100003F0A4BD5BF82130002B40F003800D49AE
:1006200000F060B8C2F10004195904460D4638467E
:1006300074F001FA002800F0098041464FF00202F0
:1006400003463846B4F0A8FF03F082BD4BF82450AF
:1006500003F084BD60B10008002B40F00380144912
:1006600000F040B85AF822100029C0F21D809C68A2
:1006700003F10C03A14280F2178053F82140054694
:100680003846214674F0D7F9002800F00980414629
:100690004FF0010203463846B4F07EFF03F058BD28
:1006A0004BF8254003F05ABD024900F01BB800008A
:1006B00060B10008C0B1000888477869002840F0A0
:1006C0000B8096F90010012940F00280FFF7E4BE8C
:1006D00003F03EBD00F002B800F022B9C7F8088070
:1006E000FFF7DABEC7F808803846BAF0F3FF00F02B
:1006F00017B9000096F90010012940F0028000F0BF
:1007000073B851464DF804BD4DF804ADB1F9002061
:1007100012F4005340F00E809244B1F90220934449
:10072000D1F80480C7F800A0C7F804B0C7F8088063
:1007300000F00BB8ABEB0001384671F065F8D7F864
:1007400000A0D7F804B0D7F80880DAF8082092F9AA
:100750000630002B40F30480ABEB83042568FD607A
:100760000446DAF810503846294671F0B7F80028E8
:1007700040F0038002B000F0D3B8002D00F02080DC
:1007800000998D682946384671F0BEF8012840F07E
:100790001780284671F0BCF80199A1EB800211681E
:1007A000384674F048F9002800F00A8002B041464B
:1007B0004FF0040203463846B4F0EEFE03F0C8BC26
:1007C00002B0DAF80820204692F908200BEB8201EB
:1007D0004FF00002884280F2048040F8042BFFF7BB
:1007E000F9BF03F0BBBC000008F1FF38FFF776BF8C
:1007F0005BF82110002940F003800449FFF772BF25
:100800008B564AF8203003F0A9BC000060B1000804
:100810005BF82110002940F003800449FFF762BF14
:100820008B5E4AF8203003F099BC000060B10008EC
:100830005BF82110002940F003800449FFF752BF04
:100840008B5A4AF8203003F089BC000060B10008E0
:100850005BF82110002940F003800449FFF742BFF4
:100860008B584AF8203003F079BC000060B10008D2
:100870005BF82110002940F003800649FFF732BFE2
:100880001144D1E900450AEB8000C0E9004503F0BE
:1008900065BC000060B100085BF82110002940F041
:1008A00003800449FFF71EBF5AF820308B5403F031
:1008B00055BC000060B100085BF82110002940F031
:1008C00003800449FFF70EBF5AF820308B5203F023
:1008D00045BC000060B100085BF82110002940F021
:1008E00003800449FFF7FEBE5AF820308B5003F016
:1008F00035BC000060B100085BF82110002940F011
:1009000003800649FFF7EEBE0AEB8000D0E9004500
:100910000A44C2E9004503F021BC000060B10008B0
:10092000C7F808803846A4F01DFB03F011BC000096
:100930000FF2060CDCF800C0604701280708000031
:1009400018F8014B59F824F018F9011B4FEA21104F
:100950004FEA01714FEA21715AF821204AF820200C
:1009600003F0FCBB18F9010B18F9011B5AF8212000
:100970004AF8202003F0F2BB18F9010B18F9011B0B
:100980000AEB80000AEB8101D1E90023C0E90023D2
:1009900003F0E4BB18F9011B4FEA21104FEA017183
:1009A0004FEA21715BF821204BF8202003F0D6BBE1
:1009B00018F9010B18F9011B5BF821204BF82020D6
:1009C00003F0CCBB18F9010B18F9011B4AF82010F1
:1009D00003F0C4BB18F9010B38F9021B4AF82010C8
:1009E00003F0BCBB38F9021B18F9010B4AF82010C0
:1009F00003F0B4BB18F9010B38F8021B38F8022BCE
:100A000041EA02414AF8201003F0A8BB38F8021B63
:100A100038F8022B18F9010B41EA02414AF820107C
:100A200003F09CBB18F9010B18F9011B4FEAE172A6
:100A30000AEB80000160426003F090BB18F9010BE3
:100A40000AEB800038F8021B38F8022B41EA024119
:100A500040F8041B38F8021B38F8022B41EA024127
:100A6000016003F07BBB000098F908000AEB8000EE
:100A700038F8021B38F8022B41EA024140F8041B07
:100A800038F8021B38F8032B41EA0241016003F0F9
:100A900065BB000018F9010B38F8021B38F8022B6F
:100AA00041EA02414BF8201003F058BB38F8021B12
:100AB00038F8022B18F9010B41EA02414BF82010DB
:100AC00003F04CBB18F9010B4FF000014BF820105C
:100AD00003F044BB5BF8040CCBF8000003F03EBB12
:100AE0005BF8080CCBF8000003F038BB18F9010BD9
:100AF0004FF000014AF8201003F030BB18F9010B49
:100B00004FF001014AF8201003F028BB4FF000001D
:100B1000CAF8140003F022BB4FF000004AF8040C9E
:100B200003F01CBB18F9010B18F9011B5AF821201E
:100B30004FEA02624FEA22624AF8202003F00EBB1D
:100B400018F9010B18F9011B5AF821204FEA02424B
:100B50004FEA22424AF8202003F000BB18F9010BAB
:100B600018F9011B5AF821204FEA02424FEA1242BB
:100B70004AF8202003F0F2BA18F9010B18F9011B0A
:100B80005AF821204FEAE2730AEB800002604360CA
:100B900003F0E4BA18F9014B18F9013B0AEB83039F
:100BA00093ED000A73F018F80AEB8404206061608A
:100BB00003F0D4BA18F9014B18F9013B0AEB83038F
:100BC00093ED000B73F01DF80AEB84042060616064
:100BD00003F0C4BA18F9014B18F9013B5AF8230085
:100BE00073F028F810EE100A4AF8240003F0B6BAA1
:100BF00018F9014B18F9013B0AEB8303D3E9000113
:100C000073F01DF810EE100A4AF8240003F0A6BA9B
:100C100018F9014B18F9013B0AEB84045AF8230038
:100C200073F013F884ED000B03F098BA18F9014B38
:100C300018F9013B0AEB83030AEB8404D3E90001B2
:100C400073F009F884ED000B03F088BA18F9014B32
:100C500018F9013B0AEB84040AEB830393ED000AC5
:100C600073F000F884ED000B03F078BA18F9014B2B
:100C700018F9013B0AEB830393ED000B73F02EF898
:100C800010EE100A4AF8240003F068BA18F9014B74
:100C900018F9013B0AEB830393ED000A73F060F847
:100CA0004AF8240003F05ABA18F9014B18F9013B2D
:100CB0000AEB830393ED000B73F066F84AF8240007
:100CC00003F04CBA18F9082B4FEA98014FEA81015A
:100CD00031F8040C5AF8222073F06EF8804603F0C5
:100CE0003DBA000018F9040B4FEA98084FEA88084B
:100CF00058F8042B58F8043B38F8021B5AF8200027
:100D0000984200F30C809042C0F20980A0EB0200F0
:100D10004FEA400038F80000804403F01FBA8844CE
:100D200003F01CBA18F8010B804403F017BA000056
:100D300038F8020B804403F011BA000018F9010BD7
:100D400018F8011B5AF82020002A08BF884403F035
:100D500005BA000018F9010B18F8011B5AF82020F9
:100D6000002A18BF884403F0F9B9000018F9010BF4
:100D700018F8011B5AF82020002AB8BF884403F055
:100D8000EDB9000018F9010B18F8011B5AF82020E2
:100D9000002AD8BF884403F0E1B9000018F9010B1C
:100DA00018F8011B5AF82020002AA8BF884403F035
:100DB000D5B9000018F9010B18F8011B5AF82020CA
:100DC000002AC8BF884403F0C9B9000018F9010B14
:100DD00018F9011B18F8012B5AF820308B4208BF74
:100DE000904403F0BBB9000018F9010B18F9011B7E
:100DF00018F8012B5AF820308B4218BF904403F0AA
:100E0000ADB9000018F9010B18F9011B18F8012BF6
:100E10005AF820308B42A8BF904403F09FB90000DD
:100E200018F9010B18F9011B18F8012B5AF820309A
:100E30008B42D8BF904403F091B9000018F9010B20
:100E400018F9011B38F8022B5AF820305AF82140C3
:100E5000A34208BF904403F081B9000018F9011BB8
:100E60004FEA21104FEA01714FEA217118F8012B66
:100E70005AF820305AF82140A34208BF904403F0AA
:100E80006DB9000018F9010B18F9011B38F8022B95
:100E90005AF820305AF82140A34218BF904403F07A
:100EA0005DB9000018F9011B4FEA21104FEA0171EA
:100EB0004FEA217118F8012B5AF820305AF82140D6
:100EC000A34218BF904403F049B9000018F9010B80
:100ED00018F9011B38F8022B5AF820305AF8214033
:100EE000A342B8BF904403F039B9000018F9011BC0
:100EF0004FEA21104FEA01714FEA217118F8012BD6
:100F00005AF820305AF82140A342B8BF904403F069
:100F100025B9000018F9010B18F9011B38F8022B4C
:100F20005AF820305AF82140A342D8BF904403F029
:100F300015B9000018F9011B4FEA21104FEA0171A1
:100F40004FEA217118F8012B5AF820305AF8214045
:100F5000A342D8BF904403F001B9000018F9010B77
:100F600018F8011B5BF82020002A08BF884403F012
:100F7000F5B8000018F9010B18F8011B5BF82020E8
:100F8000002A18BF884403F0E9B8000018F8010BE4
:100F90005BF8041C002908BF804403F0DFB80000A0
:100FA00018F8010B5BF8041C002918BF804403F0FB
:100FB000D5B8000018F9010B18F9012B18F9014BED
:100FC0000AEB80010AEB8203D1E90001D3E9002397
:100FD00072F010FF4AF8240003F0C0B818F9014B72
:100FE00018F9012B4FEAE27318F9015B0AEB84044C
:100FF000D4E9000172F0FEFE4AF8250003F0AEB815
:1010000018F9012B18F9013B18F9014B5AF8220085
:101010005AF8231041EC100A72F0FCFE4AF8240042
:1010200003F09CB818F9012B18F9013B18F9014B92
:101030005AF822005AF8231041EC100A72F00DFF02
:101040004AF8240003F08AB818F901CB18F9015BBB
:1010500018F9014B0AEB8C0C0AEB85059CED000B93
:1010600095ED001B72F01BFF4AF8240003F076B8E0
:1010700018F901CB18F9015B18F9014B0AEB8C0C3C
:101080000AEB85059CED000B95ED001B72F034FF1B
:101090004AF8240003F062B818F9010B18F9011B93
:1010A0005AF8212002444AF8212003F057B80000E2
:1010B00018F9010B5AF8201001F101014AF820102B
:1010C00003F04CB818F9010B5AF8201001F1FF3168
:1010D0004AF8201003F042B818F9010B18F9011B67
:1010E00018F9012B5AF820005AF8211008444AF840
:1010F000220003F033B8000018F9010B18F9011BA6
:1011000018F9012B5AF8200008444AF8220003F08D
:1011100025B8000018F9010B18F9012B18F9014B3B
:101120000AEB80010AEB8203D1E90001D3E9002335
:10113000801841EB03010AEB8404C4E9000103F0C9
:101140000DB8000018F9010B18F9011B18F9014B33
:101150005AF820005AF8211041EC100A72F0F8FEFB
:1011600010EE100A4AF8240002F0F8BF18F9010B3B
:1011700018F9011B18F9014B0AEB800C0AEB8105E9
:101180000AEB84049CED000B95ED001B72F0FAFE57
:1011900084ED000B02F0E2BF18F9010B18F9011BF6
:1011A00018F9012B5AF820305AF82140A3EB040318
:1011B0004AF8223002F0D2BF18F9010B18F9012BBE
:1011C00018F9014B0AEB80010AEB8203D1E9000117
:1011D000D3E90023801A61EB03010AEB8404C4E91C
:1011E000000102F0BBBF000018F9010B18F9011B48
:1011F00018F9014B5AF820005AF8211041EC100A56
:1012000073F06CF910EE100A4AF8240002F0A6BF41
:1012100018F9010B18F9011B18F9014B0AEB800CA6
:101220000AEB81050AEB84049CED000B95ED001B95
:1012300073F06EF984ED000B02F090BF18F9010B0A
:1012400018F9011B18F9012B5AF820305AF82140DF
:1012500003FB04F04AF8220002F080BF18F9010BEA
:1012600018F9011B18F9012B5AF8203003FB01F083
:101270004AF8220002F072BF18F9010B18F9012B8D
:1012800018F901CB0AEB80010AEB8203D1E90001D6
:10129000D3E90023A0FB024500FB035501FB0255E7
:1012A0000AEB8C0CCCE9004502F058BF18F9010B91
:1012B00018F9011B18F9014B5AF820005AF82110AF
:1012C00041EC100A72F0C2FE10EE100A4AF8240037
:1012D00002F044BF18F9010B18F9011B18F9014B72
:1012E0000AEB800C0AEB81050AEB84049CED000BF1
:1012F00095ED001B72F0C4FE84ED000B02F02EBFD2
:1013000018F9010B18F9011B18F9014B5AF82000C4
:101310005AF82110002940F003800449FFF7E2B990
:1013200072F0FAFE4AF8240002F018BFA0B30008D9
:1013300018F9010B18F9011B18F9014B5AF8200094
:10134000002940F003800449FFF7CCB972F0E4FEB5
:101350004AF8240002F002BFA0B3000818F9010BFC
:1013600018F9012B18F9014B0AEB80010AEB8203F3
:10137000D1E90001D3E90023002A40F00680002BC8
:1013800040F003800549FFF7ADB972F0C8FE0AEBE3
:101390008404C4E9000102F0E1BE0000A0B300082B
:1013A00018F9010B18F9011B18F9014B5AF8200024
:1013B0005AF8211041EC100A72F0B6FE10EE100A35
:1013C0004AF8240002F0CABE18F9010B18F9011BF3
:1013D00018F9014B0AEB800C0AEB81050AEB840437
:1013E0009CED000B95ED001B72F0D2FE84ED000B1E
:1013F00002F0B4BE18F9010B18F9011B18F9014BE2
:101400005AF820005AF82110002940F003800449BE
:10141000FFF768B972F096FF4AF8240002F09EBE0A
:10142000A0B3000818F9010B18F9012B18F9014BAA
:101430000AEB80010AEB8203D1E90001D3E9002322
:10144000002A40F00680002B40F003800549FFF79A
:1014500049B972F07CFF0AEB8404C4E9000102F090
:101460007DBE0000A0B3000818F9010B18F9011B9C
:1014700018F9014B5AF820005AF8211041EC100AD3
:1014800072F06CFF10EE100A4AF8240002F066BEFB
:1014900018F9010B18F9011B18F9014B0AEB800C24
:1014A0000AEB81050AEB84049CED000B95ED001B13
:1014B00072F0A2FF84ED000B02F050BE18F9010B90
:1014C00018F9011B5AF82020C2F100004AF8210047
:1014D00002F044BE18F9010B18F9011B0AEB800059
:1014E000D0E90023544263EB43050AEB8101C1E9D3
:1014F000004502F033BE000018F9011B18F9014B3A
:101500004FF000400AEB810100EE100AD1ED000A15
:1015100072F0E4FF10EE100A4AF8240002F01EBE3A
:1015200018F9014B18F9015B0AEB84040AEB8505F5
:101530004FF000004FF0004141EC100B94ED001B08
:1015400072F0E6FF85ED000B02F008BE18F9010B02
:1015500018F9011B18F9012B5AF820305AF82140CC
:1015600004F01F0403FA04F04AF8220002F0F6BD6A
:1015700018F9010B18F9011B18F9012B5AF8203042
:1015800003FA01F04AF8220002F0E8BD18F9010B55
:1015900018F9011B18F9014B5AF821200AEB8005B4
:1015A000D5E9000173F032F80AEB8404C4E90001C4
:1015B00002F0D4BD18F9010B18F9011B18F9012B21
:1015C0005AF820305AF8214004F01F0443FA04F07E
:1015D0004AF8220002F0C2BD18F9010B18F9011BEC
:1015E00018F9012B5AF8203043FA01F04AF822008A
:1015F00002F0B4BD18F9010B18F9011B18F9014BE1
:101600005AF821200AEB8005D5E9000173F002F8B1
:101610000AEB8404C4E9000102F0A0BD18F9010B33
:1016200018F9011B18F9012B5AF820305AF82140FB
:1016300004F01F0423FA04F04AF8220002F08EBDE1
:1016400018F9010B18F9011B18F9014B5AF8212060
:101650000AEB8005D5E9000172F0E0FF0AEB840493
:10166000C4E9000102F07ABD18F9010B18F9011B59
:1016700018F9012B5AF820305AF8214003EA0400E7
:101680004AF8220002F06ABD18F9010B18F9011B93
:1016900018F9012B5AF8203003EA01004AF8220019
:1016A00002F05CBD18F9010B18F9012B18F9014B78
:1016B0000AEB80010AEB8203D1E90001D3E90023A0
:1016C00000EA020001EA03010AEB8404C4E9000114
:1016D00002F044BD18F9010B18F9011B18F9012B90
:1016E0005AF820305AF8214043EA04004AF8220010
:1016F00002F034BD18F9010B18F9012B18F9014B50
:101700000AEB80010AEB8203D1E90001D3E900234F
:1017100040EA020041EA03010AEB8404C4E9000143
:1017200002F01CBD18F9010B18F9011B18F9012B67
:101730005AF820305AF8214083EA04004AF822007F
:1017400002F00CBD18F9010B18F9011B18F9014B37
:101750000AEB80050AEB810CD5E90001DCE90023E6
:1017600080EA020081EA03010AEB8404C4E9000173
:1017700002F0F4BC18F9010B0AEB8000D0E9002359
:101780000360426002F0EABC18F9010B38F8021B52
:1017900038F8022B41EA0241FEF7D0BD18F9010BDF
:1017A00038F8021B38F8022B41EA0241FEF7CCBDA3
:1017B00018F9010B38F8021B38F8022B41EA0241F4
:1017C000FEF7C8BD18F9010B38F8021B38F8022BD8
:1017D00041EA0241FEF7C4BD18F9010B38F8021BBB
:1017E00038F8022B41EA0241FEF7C0BD73F022F93E
:1017F00018F9010B38F8021BFEF7A0BD73F01AF9B7
:1018000018F9010B38F8021BFEF79EBD73F012F9B0
:1018100018F9010B38F8021BFEF79CBD73F00AF9AA
:1018200018F9010B38F8021BFEF79ABD73F002F9A4
:1018300018F9010B38F8021BFEF798BD18F9010BD7
:1018400038F8021B38F8022B41EA0241FEF796BD38
:1018500018F9010B38F8021B38F8022B41EA024153
:10186000FEF792BD18F9010B38F8021B38F8022B6D
:1018700041EA0241FEF78EBD18F9010B38F8021B50
:1018800038F8022B41EA0241FEF78ABD73F0D2F824
:1018900018F9010B38F8021BFEF770BD73F0CAF897
:1018A00018F9010B38F8021BFEF76EBD73F0C2F891
:1018B00018F9010B38F8021BFEF76CBD73F0BAF88B
:1018C00018F9010B38F8021BFEF76ABD18F9014B35
:1018D00038F8020B38F8021B40EA0141FEF768BDF8
:1018E00038F8024B38F8025B44EA05414FF0FF3408
:1018F000FEF75EBDFFF7EABF18F9014B18F9015B6F
:101900005AF82550002D80F203800649FEF7EABE02
:10191000284638F8021B38F8022B41EA0241FEF74C
:101920005BBD0000F0B1000818F9014B18F9015B2C
:101930005AF82550002D80F203800649FEF7D2BEEA
:101940004FEA450038F8021B38F8022B41EA024101
:10195000FEF742BDF0B1000818F9014B18F9015B20
:101960005AF82550002D80F203800649FEF7BABED2
:101970004FEA850038F8021B38F8022B41EA024191
:10198000FEF72ABDF0B1000818F9014B18F9015B08
:101990005AF82550002D80F203800649FEF7A2BEBA
:1019A0004FEAC50038F8021B38F8022B41EA024121
:1019B000FEF712BDF0B1000818F9015B18F9013B00
:1019C00018F8012B38F8020B38F8021B40EA0141E5
:1019D000C7F808804DF8044D4DF8045D384672F0A4
:1019E00021FE02B0002840F00280FEF799BF02F00D
:1019F000B5BB000038F8022B38F8023B18F9010B90
:101A000018F9011B0AEB80000BEB810142EA034449
:101A1000A746000000F000B8384672F095FE012895
:101A200040F00D8096F90000012840F0048008F194
:101A3000FF38FEF753BE02F091BB00F002B802F08F
:101A400087BB000096F90010012940F00280FEF7E4
:101A5000CBBE18F9010B5BF82010FEF7D5BC0000D7
:101A600096F90010012940F00280FEF7BDBE5BF838
:101A7000041CFEF7C9BC000018F9012B38F8023B22
:101A800038F8024B43EA04405BF82210002900F0CA
:101A9000088072F0DDFE002840F003800249FEF766
:101AA00021BE02F05BBB000000B4000818F9015B26
:101AB00018F9013B38F8024B38F802CB44EA0C40E5
:101AC0005BF82310002940F004804FF0000000F084
:101AD00002B872F0BDFE4AF8250002F03FBB0000DC
:101AE00018F9010B18F9011B18F9012B5BF82130CB
:101AF000002B40F003800B49FEF7F4BD5AF822108A
:101B00000029C0F20B809C6803F10C03A14280F213
:101B100005805A564AF8202002F020BB0249FEF701
:101B2000E1BD000060B10008C0B1000818F9010B68
:101B300018F9011B18F9012B5BF82130002B40F03C
:101B400003800C49FEF7CEBD5AF822100029C0F2DE
:101B50000D809C6803F10C03A14280F207804FEADC
:101B600041015A5E4AF8202002F0F8BA0249FEF715
:101B7000B9BD000060B1000800B4000818F9010BFD
:101B800018F9011B18F9012B5BF82130002B40F0EC
:101B900003800C49FEF7A6BD5AF822100029C0F2B6
:101BA0000D809C6803F10C03A14280F207804FEA8C
:101BB00041015A5A4AF8202002F0D0BA0249FEF7F1
:101BC00091BD000060B10008C0B1000818F9010B18
:101BD00018F9011B18F9012B5BF82130FEF720BC26
:101BE00018F9011B4FEA21104FEA01714FEA2172E7
:101BF0005BF8043CFEF714BC18F9010B18F9011B43
:101C000018F9012B5BF82130002B40F003800D49BF
:101C1000FEF768BD5AF822100029C0F210809C68B7
:101C200003F10C03A14280F20A8003EBC103D3E964
:101C300000450AEB8000C0E9004502F08FBA024976
:101C4000FEF750BD60B10008C0B1000818F9010BE3
:101C500018F9011B18F9012B5AF822205BF82030E3
:101C6000002B40F003800A49FEF73CBD5AF82100E2
:101C70000028C0F209809C6803F10C03A04280F2A6
:101C800003801A5402F06ABA0249FEF72BBD000025
:101C900060B10008C0B1000818F9010B18F9011B68
:101CA00018F9012B5AF822205BF82030002B40F065
:101CB00003800B49FEF716BD5AF821000028C0F238
:101CC0000B809C6803F10C03A04280F205804FEA70
:101CD00040001A5202F042BA0249FEF703BD00006A
:101CE00060B10008C0B1000818F9010B18F9011B18
:101CF00018F9012B5BF82030FEF7B0BB18F9012B67
:101D00004FEA22114FEA02724FEA22725BF8043C5A
:101D1000FEF7A4BB18F9010B18F9011B18F9012BE8
:101D20000AEB8202D2E900455BF82030002B40F03C
:101D300003800C49FEF7D6BC5AF821000028C0F2F7
:101D40000D80D3F808C003F10C03604580F20680D3
:101D500003EBC003C3E9004502F000BA0249FEF7F5
:101D6000C1BC000060B10008C0B1000818F9010B47
:101D700018F9011B5BF82120002A40F00380044978
:101D8000FEF7B0BC91684AF8201002F0E7B90000F5
:101D900060B1000818F9010B18F9011B38F8022B83
:101DA0005BF820305BF82140A34208BF904402F06A
:101DB000D5B9000018F9011B4FEA21104FEA017153
:101DC0004FEA217118F8012B5BF820305BF82140B5
:101DD000A34208BF904402F0C1B9000018F9010BFA
:101DE00018F9011B38F8022B5BF820305BF8214012
:101DF000A34218BF904402F0B1B9000018F9011BCA
:101E00004FEA21104FEA01714FEA217118F8012BB6
:101E10005BF820305BF82140A34218BF904402F0E9
:101E20009DB9000018F9011B4FEA211001F00F01C4
:101E3000FD686A564AF8202002F090B918F9011B93
:101E40004FEA211001F00F014FEA4101FD686A5E7F
:101E50004AF8202002F082B918F9011B4FEA21103C
:101E600001F00F014FEA4101FD686A5A4AF820204B
:101E700002F074B918F9011B4FEA211001F00F01AB
:101E8000FD6855F821204AF8202002F067B90000CB
:101E900018F9011B4FEA211001F00F01FD6805EB55
:101EA0008105D5E900230AEB8000C0E9002302F098
:101EB00055B9000018F9010B18F9011B18F8012B8E
:101EC000FEF796BC18F9010B18F9011B18F8012B45
:101ED000FEF79EBC18F9010B18F9011B18F8012B2D
:101EE000FEF7A6BC18F9010B18F9011B18F8012B15
:101EF000FEF7AEBC18F9011B4FEA21104FEA017141
:101F00004FEA21714FF00802FEF7A2BC18F9010B4D
:101F100018F9011B18F8012BFEF7AABC18F9011BD0
:101F20004FEA211001F00F01FD685AF820206A5491
:101F300002F014B918F9011B4FEA211001F00F014A
:101F40004FEA4101FD685AF820206A5202F006B9B2
:101F500018F9011B4FEA211001F00F01FD685AF832
:101F6000202045F8212002F0F9B8000018F9011BE3
:101F70004FEA211001F00F010AEB8000D0E90023A5
:101F8000FD6805EB8105C5E9002302F0E7B8000014
:101F900018F9010B18F9011B18F8012BFEF77CBC8E
:101FA00018F9010B18F9011B18F8012BFEF784BC76
:101FB00018F9010B18F9011B18F8012BFEF78CBC5E
:101FC00018F9010B18F9011B18F8012BFEF794BC46
:101FD00018F9012B5BF82220002A40F00380094900
:101FE000FEF780BBC7F8088007480068394672F0E2
:101FF0004BFC96F90010012940F00280FEF74CBA24
:1020000002F0A6B860B100084C04012018F9012BB9
:102010005BF82220002A40F003800949FEF762BBEA
:10202000C7F808800748006839468CF015FF96F914
:102030000010012940F00280FEF72EBA02F088B8A5
:1020400060B100084C040120FA68C7F8088007480E
:102050000068394672F018FC96F90010012940F02A
:102060000280FEF719BA02F073B800004C04012098
:10207000FA68C7F808800748006839468CF0ECFE1B
:1020800096F90010012940F00280FEF705BA02F02F
:102090005FB800004C040120C7F8088072F03EFCD5
:1020A00096F90010012940F00280FEF7F5B902F020
:1020B0004FB8000018F9010B0AEB80013846C7F849
:1020C000088072F053FC96F90010012940F002805C
:1020D000FEF7E2B902F03CB818F9010B18F9011B40
:1020E0000AEB80005BF82110002940F003801149C1
:1020F000FEF7F8BAC7F8088072F070FC012840F0CB
:1021000003800D49FEF7EEBA032840F003800B4927
:10211000FEF7E8BA022840F003800949FEF7E2BA68
:1021200096F90010012940F00280FEF7B5B902F0DF
:102130000FB8000060B1000870B30008B0B200082A
:1021400010B3000818F9010B38F8021B38F8022BFD
:1021500041EA0241FEF7B2B972F06CFC18F9010BCA
:1021600038F8021BFEF7AAB918F9011B4FEA211033
:1021700001F00F01FD685BF82020C1F100044DF86B
:10218000042D3846294672F037FC002800F00A80FA
:1021900001B041464FF0020203463846B3F0FCF965
:1021A00001F0D6BF5DF8042B45F8242001F0D6BF1E
:1021B00018F9010B18F9011B18F8012BFEF79EB94D
:1021C00018F9010B18F9011B18F8012B18F8013B3D
:1021D00042EA0322FEF792B918F9012B4FEA2211C5
:1021E0004FEA02724FEA22725BF8080CFEF7AEB9B2
:1021F00018F9013B18F9011B18F9012B5BF82300B2
:10220000FEF7A4B9A8F1010218F9010B38F8021B76
:1022100038F8023B41EA0341FEF7D8B972F00AFCF4
:10222000A8F1010218F9010B38F8021BFEF7CEB92C
:1022300018F9010B18F9011B18F8012BFEF7EAB980
:1022400018F9010B18F9011B18F8012B18F8013BBC
:1022500042EA0322FEF7DEB918F9011B4FEA21100A
:1022600001F00F01FD68C1F1000455F82440054656
:102270003846214672F0DFFB002800F00980414615
:102280004FF0020203463846B3F086F901F060BF12
:102290004BF8254001F062BF18F9011B4FEA2110ED
:1022A0004FEA01714FEA21725BF8043CFEF7D4B9A2
:1022B00018F9010B18F9011B18F9012B5BF82130F3
:1022C000FEF7CAB996F90010012940F00280FEF726
:1022D0008BBA38F8020BA8EB000801F03FBF0000F2
:1022E00096F90010012940F00280FEF77DBA18F837
:1022F000010BA8EB000801F031BF000096F90000C7
:10230000012840F0048008F1FF38FEF7E7B901F03A
:1023100025BF000038F8021B38F8022B41EA0241C1
:102320003846C7F80880FEF7C7B900000149FEF734
:10233000D9B90000A0B50008C7F8088098F80600D1
:1023400000F00F002DE9000D6C46ADEBC00D98F9C3
:10235000040098F905100AEB800A0BEB810B98F842
:10236000075008F1080800F09FB818F8011BCA07C9
:102370004FEAD10200F019805BF8041B06B47B48D9
:10238000006872F05CFB002840F00880A84494E8E4
:10239000000DA54603B07649FEF7A4B906BC01F1CD
:1023A0000C014DF8221000F07FB88B074FEA417303
:1023B00040F12F807AE90201002BC0F206800DEB7C
:1023C0008202C2E9000100F06FB84FEAC2029744EE
:1023D00000BF41EC100B00F067B841EC110B00F0AE
:1023E00063B841EC120B00F05FB841EC130B00F046
:1023F0005BB841EC140B00F057B841EC150B00F042
:1024000053B841EC160B00F04FB841EC170B00F03D
:102410004BB85AF8040D002B80F244804FEAC202F8
:10242000974400BF00EE100A00F03EB800EE900A9C
:1024300000F03AB801EE100A00F036B801EE900A4A
:1024400000F032B802EE100A00F02EB802EE900A48
:1024500000F02AB803EE100A00F026B803EE900A46
:1024600000F022B804EE100A00F01EB804EE900A44
:1024700000F01AB805EE100A00F016B805EE900A42
:1024800000F012B806EE100A00F00EB806EE900A40
:1024900000F00AB807EE100A00F006B807EE900A3E
:1024A00000F002B84DF822006D1E7FF55EAF454684
:1024B00094E8000DB8F80000B8F8021040EA014CAA
:1024C0000FBCE047A54603B0D7F814C0BCF1000F1D
:1024D00000F00580A846FEF723BA00F046B898F849
:1024E00006C04FEA1C1CBCF1000F00F03480BCF1A8
:1024F000060F40F009800B46024698F90410384652
:1025000072F0A8FA00F027B8BCF1080F40F009807B
:1025100053EC102B98F90410384672F0A5FA00F02D
:102520001AB8BCF1090F40F00880024698F905106E
:10253000384672F0A2FA00F00EB8BCF1070F40F076
:10254000048010EE102A00F001B8024698F9041039
:10255000384672F096FAA84696F90000012840F035
:102560000280FEF7BBB801F0F9BD0000380401207D
:10257000B0B2000896F90010012940F00280FEF781
:1025800033B918F9014B18F9013B38F9022B0BEB61
:1025900083030AEB84041968002940F0038007498B
:1025A000FEF7A0B8C7F80880F96038464DF8044D2A
:1025B0009CF03AFC01B001F0CBBD000060B1000816
:1025C00096F90010012940F00280FEF70DB918F8C5
:1025D000012B5B4654461968002940F003800749E7
:1025E000FEF780B8C7F80880F96038464DF8044D0A
:1025F0009CF01AFC01B001F0ABBD000060B1000816
:1026000096F90010012940F00280FEF7EDB818F9A4
:10261000014B18F9013B38F9022B0BEB83030AEB52
:1026200084041968002940F003800749FEF75AB86E
:10263000C7F80880F96038464DF8044D72F028FA62
:1026400001B001F085BD000060B1000896F90010EE
:10265000012940F00280FEF7C7B818F9013B18F9CC
:10266000012B38F8020B38F8021B40EA01410BEB52
:1026700082020AEB8303D2F800C0BCF1000F40F0E5
:1026800003800649FEF72EB8C7F80880C7F80CC0CB
:10269000384672F065FA01F05BBD000060B10008D9
:1026A00096F90010012940F00280FEF79DB838F835
:1026B000020B38F8021B40EA01415A465346D2F851
:1026C00000C0BCF1000F40F003800649FEF70AB8D5
:1026D000C7F80880C7F80CC0384672F041FA01F01C
:1026E00037BD000060B1000896F90010012940F0E4
:1026F0000280FEF779B818F9013B18F9012B38F878
:10270000020B38F8021B40EA01414FF0000CC7F8F9
:102710000CC00BEB82020AEB8303C7F80880384633
:1027200072F01EFA01F014BD96F90010012940F074
:102730000280FEF759B838F8020B38F8021B40EA5D
:1027400001414FF0000CC7F80CC05A465346C7F879
:102750000880384672F004FA01F0FABC96F90010CD
:10276000012940F00280FEF73FB818F9012B18F953
:10277000011B38F8024B38F8025B0BEB81010AEBC6
:1027800082020B68002B40F003800849FDF7AABFC6
:10279000C7F80880FB6038464DF8045D4DF8044DDD
:1027A00072F0A6F902B001F0D3BC000060B10008DD
:1027B00096F90010012940F00280FEF715B818F8CC
:1027C000012B5B46F9685446CBF80010C7F8088027
:1027D00038464DF8044D9CF027FB01B001F0B8BC21
:1027E00096F90010012940F00280FDF7FDBF38F88E
:1027F000020B38F8021B40EA01415A46FD68534675
:102800001560C7F80880384672F0AAF901F0A0BC3C
:1028100098F900200BEB8200FDF76CBF5846FDF7DE
:1028200069BF0000ABF10400FDF764BFABF1080025
:10283000FDF760BF96F90010012940F00280FDF716
:10284000D3BF18F9010B18F8011B5AF82020002AF1
:1028500008BFA8EB010801F081BC000096F9001048
:10286000012940F00280FDF7BFBF18F9010B18F8ED
:10287000011B5AF82020002A18BFA8EB010801F01C
:102880006DBC000096F90010012940F00280FDF7B0
:10289000ABBF18F9010B18F8011B5AF82020002AC9
:1028A000B8BFA8EB010801F059BC000096F9001070
:1028B000012940F00280FDF797BF18F9010B18F8C5
:1028C000011B5AF82020002AD8BFA8EB010801F00C
:1028D00045BC000096F90010012940F00280FDF788
:1028E00083BF18F9010B18F8011B5AF82020002AA1
:1028F000A8BFA8EB010801F031BC000096F9001058
:10290000012940F00280FDF76FBF18F9010B18F89C
:10291000011B5AF82020002AC8BFA8EB010801F0CB
:102920001DBC000096F90010012940F00280FDF75F
:102930005BBF18F9010B18F9011B38F8022B5AF884
:1029400020305AF82140A34208BFA8EB020801F04A
:1029500005BC000096F90010012940F00280FDF747
:1029600043BF18F9010B18F9011B38F8022B5AF86C
:1029700020305AF82140A34218BFA8EB020801F00A
:10298000EDBB000096F90010012940F00280FDF730
:102990002BBF18F9010B18F9011B38F8022B5AF854
:1029A00020305AF82140A342B8BFA8EB020801F03A
:1029B000D5BB000096F90010012940F00280FDF718
:1029C00013BF18F9011B4FEA21104FEA01714FEABA
:1029D000217118F8012B5AF820305AF82140A342EF
:1029E000B8BFA8EB020801F0B9BB000096F90010CF
:1029F000012940F00280FDF7F7BE18F9010B18F924
:102A0000011B38F8022B5AF820305AF82140A34213
:102A1000D8BFA8EB020801F0A1BB000096F9001096
:102A2000012940F00280FDF7DFBE18F9011B4FEAD3
:102A300021104FEA01714FEA217118F8012B5AF861
:102A400020305AF82140A342D8BFA8EB020801F079
:102A500085BB000096F90010012940F00280FDF7C7
:102A6000C3BE18F9010B18F9011B38F8022B5BF8EB
:102A700020305BF82140A34208BFA8EB020801F018
:102A80006DBB000096F90010012940F00280FDF7AF
:102A9000ABBE18F9010B18F9011B38F8022B5BF8D3
:102AA00020305BF82140A34218BFA8EB020801F0D8
:102AB00055BB000096F90010012940F00280FDF797
:102AC00093BE18F9010B18F8011B5BF82020002AAF
:102AD00008BFA8EB010801F041BB000096F9001007
:102AE000012940F00280FDF77FBE18F9010B18F8AC
:102AF000011B5BF82020002A18BFA8EB010801F099
:102B00002DBB000018F9010B18F9011B18F8012B57
:102B100018F8013B42EA0322FDF76ABE18F9010BDF
:102B200018F9011B18F8012B18F8013B42EA03229F
:102B3000FDF76EBE18F9010B18F9011B18F8012BEF
:102B400018F8013B42EA0322FDF772BE18F9010BA7
:102B500018F9011B18F8012B18F8013B42EA03226F
:102B6000FDF776BE18F9010B18F9011B18F8012BB7
:102B700018F8013B42EA0322FDF77ABE18F9010B6F
:102B800018F9011B18F8012B18F8013B42EA03223F
:102B9000FDF782BE18F9010B18F9011B18F8012B7B
:102BA00018F8013B42EA0322FDF786BE18F9010B33
:102BB00018F9011B18F8012B18F8013B42EA03220F
:102BC000FDF78ABE18F9010B18F9011B18F8012B43
:102BD00018F8013B42EA0322FDF78EBE71F0D6FFE2
:102BE00008F1010818F8014B59F824F008F1010820
:102BF00018F8014B59F824F03846A8F1010171F09A
:102C0000C7FF7969002940F00B80002840F004805C
:102C100001F09EBA00F002B801F0A0BA00F002B8CC
:102C2000FDF77EBE01B400680FF2080C5CF820C00E
:102C300001BC6047395007083D50070801B40068DF
:102C40000FF2080C5CF820C001BC60474150070837
:102C50004550070801B400680FF2080C5CF820C06A
:102C600001BC6047495007084D50070801B400688F
:102C70000FF2080C5CF820C001BC604751500708F7
:102C8000575007080FF2060CDCF800C060475D5093
:102C9000070800000FF2060CDCF800C06047695618
:102CA0000708000001B400680FF2080C5CF820C0AF
:102CB00001BC6047296007084360070801B4006849
:102CC0000FF2080C5CF820C001BC60474F60070899
:102CD0007D60070801B400680FF2080C5CF820C0A2
:102CE00001BC604789600708CF6007080FF2060C37
:102CF000DCF800C06047B3610708000001B4006859
:102D00000FF2080C5CF820C001BC6047498107083D
:102D10006B8107080FF2060CDCF800C06047C98120
:102D20000708A0F16101192900D8203870470EB5B5
:102D300040F2334202920022CDE90022134667F0AE
:102D40007FFC03B000BD00007F2801D9002208E00D
:102D5000064A02EB5002C007127800D1120902F0B5
:102D60000F0201209040084070470000889D0C0829
:102D70000FF2060CDCF800C06047C9950708000098
:102D80000FF2060CDCF800C06047C596070800008B
:102D90000FF2060CDCF800C060478B97070803466B
:102DA00011F8012B00F8012B002AF9D118467047C1
:102DB000CAB2401E10F8011F8A4202D00029F9D180
:102DC000002070470FF2060CDCF800C060471DE5DC
:102DD000080800000FF2060CDCF800C06047C9B517
:102DE000070800000FF2060CDCF800C060473FB790
:102DF000070800000FF2060CDCF800C0604771B74E
:102E0000070800000FF2060CDCF800C060477DB731
:102E1000070800000FF2060CDCF800C06047ADB7F1
:102E20000708000001B400680FF2080C5CF820C02D
:102E300001BC6047D5B707080BB807080FF2060CAE
:102E4000DCF800C060471FB8070800000FF2060C4E
:102E5000DCF800C060470BCE070800000FF2060C3C
:102E6000DCF800C0604739CE0708000001B40068F4
:102E70000FF2080C5CF820C001BC604745CE070883
:102E80004DCE07080FF2060CDCF800C0604759CEA3
:102E9000070800000FF2060CDCF800C0604787CE80
:102EA0000708000001B400680FF2080C5CF820C0AD
:102EB00001BC604793CE07089DCE070801B40068A7
:102EC0000FF2080C5CF820C001BC6047A9CE0708CF
:102ED000CBCE07080FF2060CDCF800C0604721CF0C
:102EE000070800000FF2060CDCF800C060470DD0A8
:102EF000070800000FF2060CDCF800C060471DD088
:102F00000708A0F14101192900D8203070470000BE
:102F10000FF2060CDCF800C06047E940080800002A
:102F20000FF2060CDCF800C060479542080800006C
:102F300001B400680FF2080C5CF820C001BC6047C7
:102F4000A54208083D4308080FF2060CDCF800C053
:102F50006047AF43080800000FF2060CDCF800C021
:102F60006047B743080800000FF2060CDCF800C009
:102F70006047C943080800002DE9FF4F087881B079
:102F80009946FF2805D0491C2D2804D00024002391
:102F900008E000230BE00124F9E703EB830300EBD7
:102FA0004303491C0878FF28F7D104B15B42002095
:102FB0000090147801462D2C01D02B2C04D1521CEA
:102FC0002D2C12D00024009400251678FF2E0ED050
:102FD0000A24A0FB04C801FB0481002700FB0711A1
:102FE000521C16EB0C006941EFE70124EBE7994412
:102FF00050EA01020ED00024AA4D2646DFF8A8822E
:10300000FFF795FE82468B46B9F1000009DAC9F157
:1030100000071BE001980021C0E9001105B0BDE8E0
:10302000F08F074612E0F80707D022462B463046BD
:10303000414667F0BDFB0646884622462B461046B1
:10304000194667F0B5FB04460D467F10002FEAD104
:10305000B9F1000F324643465046594602DA67F04E
:1030600019FC01E067F0A4FB009A0AB181F000416D
:10307000019AC2E90001D1E72DE9FF4F1F468DB04B
:10308000D7E901464FF0FF382E2045464FF00009A2
:103090000B90B9696D1C0E988847396A824688473B
:1030A0000028F6D1BAF1FF3F0AD024F4D064002EF4
:1030B00011DDBAF12B0F08D0BAF12D0F0BD102E0C0
:1030C000404611B0ABE744F48064B9696D1C0E98BA
:1030D00088478246761E6946600501D52D2000E0AE
:1030E0002B208DF8000001F1010B0DF1200809E003
:1030F000B9696D1C0E98884782460F9844F4007495
:10310000761E0560002E02DDBAF1300FF0D00B996B
:103110008A453ED144F0800406E00F99681CA9F16D
:10312000010944F400740860B9696D1C761E0E989C
:10313000884782463028F0D02BE00B998A4505D18C
:10314000200603D444F08004761E18E0504681F037
:1031500044F908B30DF11301761E44F400748B4555
:1031600008D2AAF130000BF8010B200607D5A9F10F
:10317000010003E0200602D409F101008146A00508
:1031800002D50F99681C0860B9696D1C0E988847B4
:103190008246002ED1DC53E0002E51DDBAF1650FDE
:1031A00002D0BAF1450F4BD1A00549D5B9696D1CC4
:1031B00024F44074761E0E9888478246002E0CDD5B
:1031C0002B2804D0BAF12D0F07D144F48074B969CB
:1031D0006D1C0E9888478246761EE00501D52D218C
:1031E00000E02B2108F8011BCDF82C8021E00DF127
:1031F0002901761E44F4007488450CD2AAF13000EF
:1032000010F0FF0088F8000002D10B99884509D919
:1032100008F1010806E0E00501D5244801E042F28A
:103220000F708146B9696D1C0E98884782460F98C9
:103230000560002E04DD504681F0CFF80028D6D17D
:10324000F9690E988847FF208BF8000088F8000085
:103250000020069007904B466A4608A906A8FFF78B
:103260008BFEA00502D46FF001002AE714F0240FB2
:103270000AD0E00714D1DDE906123868031D3B606F
:103280000068C0E900120BE0DDE9060100F0A5FDD1
:103290000146E00704D13868021D3A600068016009
:1032A00028460EE7000024400000F03FF1D8FFFF61
:1032B000426842B1016811F8013B23B1521EC0E9D6
:1032C0000012184670470121C160881E704742688D
:1032D0005AB1C368016843B983688B4205D0491E5F
:1032E000521CC0E90012002070474FF0FF307047B9
:1032F000C0B24FF4F051FFF727BD00000FF2060CEB
:10330000DCF800C06047E943080800000FF2060C33
:10331000DCF800C06047E744080800000FF2060C24
:10332000DCF800C06047ED44080800000FF2060C0E
:10333000DCF800C06047C945080800000FF2060C21
:10334000DCF800C06047296B080800000FF2060C8B
:10335000DCF800C060479170080800000FF2060C0E
:10336000DCF800C060477D71080800000FF2060C11
:10337000DCF800C06047A171080800000FF2060CDD
:10338000DCF800C060477F77080800000FF2060CE9
:10339000DCF800C060473BA80808000000000000FF
:1033A000ADB40808000000000FF2060CDCF800C005
:1033B0006047C9B4080800000FF2060CDCF800C032
:1033C000604755B5080800000FF2060CDCF800C095
:1033D000604765B50808000001B400680FF2080CEA
:1033E0005CF820C001BC604701B7080809B70808AD
:1033F0000FB4002300B589B00CA900910B996FF0B0
:103400000042CB601E4B06931E4B07930423CDE96D
:1034100001321D4A089202466B460020FFF72CFE3F
:1034200009B05DF814FB70B586B006464FF0FF306A
:103430000091CDE90101002015460C46049032466A
:10344000694604A8FFF7D4FF02460498211825B165
:1034500008B1084600E020462860049800280DD0F6
:10346000002A02DD0098884208D0081B0094CDE9AC
:1034700001043246694604A8FFF7BAFF06B070BDE2
:10348000B1320008CF320008F1320008000000001D
:1034900000000000FDB7080887B80808E7B808086A
:1034A0005BB90808D5B9080859BA0808E5BA080888
:1034B0005DBB08080000000000000000C3BB080856
:1034C0003FBC0808B7BC080835BD0808B1BD0808EE
:1034D00027BE0808A3BE080831BF08080000000086
:1034E00000000000B5BF0808DFBF080849C0080891
:1034F0008FC00808ADC008080FC10808CDC1080872
:103500004FC208080000000000000000BFC2080809
:1035100045C30808C7C3080815C408085DC40808DF
:10352000A1C4080827C50808BFC508080000000096
:103530004DC60808ABC608080FF2060CDCF800C040
:10354000604707CB080800000FF2060CDCF800C04B
:10355000604715CB0808000001B400680FF2080CA2
:103560005CF820C001BC604731CB08086BCB080871
:103570000FF2060CDCF800C06047F9D408080EB55D
:1035800040F2334102910021CDE900110A460B4679
:1035900067F056F803B000BD0FF2060CDCF800C06F
:1035A00060479DE0080800000FF2060CDCF800C040
:1035B0006047B9E4080800000FF2060CDCF800C010
:1035C000604715E5080800000FF2060CDCF800C0A3
:1035D00060471DE5080800000FF2060CDCF800C08B
:1035E0006047F5E8080800000FF2060CDCF800C0A0
:1035F000604731EB080800000FF2060CDCF800C051
:103600006047FDEB080800000FF2060CDCF800C074
:10361000604749EC080800000FF2060CDCF800C017
:1036200060477DEC080800000FF2060CDCF800C0D3
:10363000604785EE080800000FF2060CDCF800C0B9
:103640006047ABEE080800000FF2060CDCF800C083
:103650006047BBEE080800000FF2060CDCF800C063
:103660006047E7EE0808000001B400680FF2080C9C
:103670005CF820C001BC604709EF080885EF080826
:1036800001B400680FF2080C5CF820C001BC604770
:1036900089EF080865F0080810B5044604E00B78C7
:1036A00000F8013B03B1491C521EF8D2204610BD60
:1036B00001B400680FF2080C5CF820C001BC604740
:1036C000BDF208080DF3080801B400680FF2080CF9
:1036D0005CF820C001BC60471DF3080821F308080E
:1036E00001B400680FF2080C5CF820C001BC604710
:1036F00025F3080829F308080FF2060CDCF800C0CF
:1037000060472DF3080800000FF2060CDCF800C03B
:10371000604733F3080800000000000000000000CC
:10372000C5110908D5110908EF1109081712090870
:1037300051120908000000007F1209080FF2060C60
:10374000DCF800C06047E5120908000001B4006819
:103750000FF2080C5CF820C001BC60471D1409087A
:10376000451409080FF2060CDCF800C06047491444
:10377000090800000FF2060CDCF800C060474D1489
:103780000908000001B400680FF2080C5CF820C0C2
:1037900001BC6047C5160908CB160908421C10F881
:1037A000011B0029FBD1801A7047000001B400689A
:1037B0000FF2080C5CF820C001BC6047F540090816
:1037C000F94009080FF2060CDCF800C060473541EB
:1037D0000908000001B400680FF2080C5CF820C072
:1037E00001BC60474F410908554109080FF2060C1A
:1037F000DCF800C060479941090800000FF2060C90
:10380000DCF800C06047BB41090800000FF2060C5D
:10381000DCF800C060471542090800000FF2060CF2
:10382000DCF800C060472542090800000FF2060CD2
:10383000DCF800C060472D42090800000FF2060CBA
:10384000DCF800C060473342090800F0004230F065
:1038500000400AD0C10D01F56071C0F3160042EAC4
:103860000151C208400711437047002001467047CC
:103870000029A8BF7047401C490008BF20F0010084
:10388000704710B4B0FA80FC00FA0CF050EA010462
:1038900004BF10BC704749B1CCF1200421FA04F4F4
:1038A00011FA0CF118BF012121430843A3EB0C01CD
:1038B000CB1D4FEA00614FEA102042BF002010BC30
:1038C000704700EBC35010440029A4BF10BC7047E0
:1038D000401C490008BF20F0010010BC70470000E8
:1038E0000FF2060CDCF800C06047A1610908000077
:1038F0000FF2060CDCF800C06047A961090800005F
:103900000FF2060CDCF800C06047BD61090800003A
:103910000FF2060CDCF800C060477D620908000069
:103920000FF2060CDCF800C06047C962090800000D
:103930000FF2060CDCF800C060472D6A0908000091
:103940000FF2060CDCF800C06047656A0908000049
:103950000FF2060CDCF800C06047816A09082DE907
:10396000F04D00231A461B1A8A4103DB0020014652
:10397000BDE8F08DC1F30A52C1F3130141F4801583
:103980004FF0000BD10702D100186D41521E0027E5
:10399000044640F2FF11384601EB620A3E4680467B
:1039A000024600204FF4801166F0E3FEC219714117
:1039B000BB1846EB0100B4EB030C75EB000C04D311
:1039C000E41A65EB000517460E46241908F10100BC
:1039D0006D4180463428E3DDF91946EB0600091BEA
:1039E000A84103D24FF0FF32134601E000221346F4
:1039F0001BEB070046EB0A51BDE8F04D66F011BE27
:103A000070B5C1F30A5201F000450024C1F313015F
:103A100040F2FF3341F480119A4201DA002070BD78
:103A200040F233439A42A2F2334203DC524266F040
:103A3000A0FE00E090402C43F1D0404270BD70B534
:103A400021F0004303430CD0C1F30A550024D5EB09
:103A5000040564EB0403D617AD1AB34102DB002062
:103A6000014670BD201841EB025170BD2DE9F041B7
:103A7000054621F000400C46284309D0C4F30A5003
:103A800040F23341884205DD28462146BDE8F081F9
:103A90002846FBE740F2FE31884210DC0CDB4FEA9F
:103AA000043040EA155050EA053105D0104804F0C2
:103AB000004101430020E9E700200146E6E7A0F2CB
:103AC00033404642C6F140022846214666F061FE78
:103AD0000746884628462146324666F04AFE434657
:103AE0003A4666F09EFD3246BDE8F04166F051BEB2
:103AF0000000F03F2DE9FE4FC3F30A5701F00045E7
:103B00000024C1F30A56C3F31303C1F3130143F4B2
:103B1000801312EB020AA64641F48011009543EB94
:103B2000030CA7F1010B16E0B0EB0A0061EB0C01EE
:103B3000071E71F1000707DA4FF00008D0EB08000C
:103B400085F0004568EB0101171A73EB0107EBD311
:103B5000761E001849415E45F6DA50EA010209D0A6
:103B6000CDE900E500221346029666F069FD03B038
:103B7000BDE8F08F20460099F9E70EB5C10F80EA45
:103B8000E0700844CA07002140F233438DE80E007C
:103B90000A460B4666F054FD03B000BD81F00041BB
:103BA000704700000FF2060CDCF800C06047E176B9
:103BB000090800000FF2060CDCF800C06047E97647
:103BC000090800000FF2060CDCF800C06047F5762B
:103BD000090800000FF2060CDCF800C06047597FAE
:103BE000090800000FF2060CDCF800C06047AB804B
:103BF000090800000FF2060CDCF800C060470D84D5
:103C0000090830B504460020034600E05B1C9342DF
:103C100003D2E05CCD5C401BF8D030BD30B505462A
:103C20000020034600E05B1C934205D2EC5CC85CBC
:103C3000201A01D1002CF6D130BD00000FF2060C85
:103C4000DCF800C060473985090800000FF2060C57
:103C5000DCF800C060476D85090800000FF2060C13
:103C6000DCF800C06047219A090800000FF2060C3A
:103C7000DCF800C06047A1A2090800000FF2060CA2
:103C8000DCF800C06047A9A2090800000FF2060C8A
:103C9000DCF800C060475DA4090800000FF2060CC4
:103CA000DCF800C0604789A4090800000FF2060C88
:103CB000DCF800C06047B1AC090800000FF2060C48
:103CC000DCF800C0604767BF090800000FF2060C6F
:103CD000DCF800C060476DBF090800000FF2060C59
:103CE000DCF800C06047E5C0090800000FF2060CD0
:103CF000DCF800C0604761CB09082DE9F0410024E1
:103D0000061B254671F1000605DA01240027D0EBD9
:103D1000070067EB0101161E73F1000605DA0027A4
:103D2000D2EB0702012567EB030366F002FF86462C
:103D30000E4617469C46AC4204D00025D0EB050E3B
:103D400065EB010624B10020D2EB000760EB030C09
:103D5000704631463A466346BDE8F0810FF2060CE4
:103D6000DCF800C06047B7DA090800000FF2060C63
:103D7000DCF800C0604715E2090800000FF2060CED
:103D8000DCF800C0604717E2090800000FF2060CDB
:103D9000DCF800C06047AFE2090800000FF2060C33
:103DA000DCF800C06047B5E2090800000FF2060C1D
:103DB000DCF800C06047B7E2090800000FF2060C0B
:103DC000DCF800C06047E9E2090800000FF2060CC9
:103DD000DCF800C060470DEF090801F0004330B483
:103DE00021F0004150EA010206D00A0DA2F56072EE
:103DF000C1F31301002A02DC30BC00207047440FDD
:103E000044EAC104C100E01830BC00EBC250FFF727
:103E10002FBD00000000000000000000ADF2090806
:103E2000E3F20908F1F2090813F309083BF3090862
:103E30006DF30908A7F30908CBF309080000000097
:103E400000000000E1F3090809F409082DF409084D
:103E500059F4090881F40908A3F40908CDF4090804
:103E600007F509080FF2060CDCF800C06047FDF901
:103E7000090800000FF2060CDCF800C060472905B5
:103E80000A0800000FF2060CDCF800C06047B526F7
:103E90000A0800000FF2060CDCF800C06047492D4C
:103EA0000A0800000FF2060CDCF800C06047792D0C
:103EB0000A0800000FF2060CDCF800C06047A72DCE
:103EC0000A0800000FF2060CDCF800C06047D32D92
:103ED0000A0800000FF2060CDCF800C06047F93059
:103EE0000A0800000FF2060CDCF800C06047193128
:103EF0000A0800000FF2060CDCF800C06047ED3144
:103F00000A0800000FF2060CDCF800C060473132EE
:103F10000A0800000FF2060CDCF800C06047753A92
:103F20000A0800000FF2060CDCF800C06047AD3A4A
:103F30000A0800000FF2060CDCF800C06047EB3BFB
:103F40000A0800000FF2060CDCF800C06047113CC4
:103F50000A0800000FF2060CDCF800C060473D3C88
:103F60000A0800000FF2060CDCF800C06047593C5C
:103F70000A0800000FF2060CDCF800C06047DF53AF
:103F80000A0800000FF2060CDCF800C060474D562E
:103F90000A0800000FF2060CDCF800C06047AD56BE
:103FA0000A0800000FF2060CDCF800C06047397206
:103FB0000A0800000FF2060CDCF800C06047317AF6
:103FC0000A0800000FF2060CDCF800C060478D7A8A
:103FD0000A0800000FF2060CDCF800C06047E17A26
:103FE0000A0800000FF2060CDCF800C0604789A741
:103FF0000A0800000FF2060CDCF800C06047D5ADDF
:104000000A0800000FF2060CDCF800C0604779B324
:104010000A0800000FF2060CDCF800C0604771D6F9
:104020000A0800000FF2060CDCF800C06047F5F645
:104030000A0800000FF2060CDCF800C06047F7F633
:104040000A0800000FF2060CDCF800C06047FBF61F
:104050000A0800000FF2060CDCF800C06047EBF71E
:104060000A0800000FF2060CDCF800C0604769F88F
:104070000A0800000FF2060CDCF800C06047E1F807
:104080000A0800000FF2060CDCF800C060479D0E25
:104090000B08000030B5041E71F1000404DB4FF082
:1040A0000044404264EB0101141E73F1000405DB7F
:1040B0001C464FF00043524263EB04038B4208BF9F
:1040C000824230BD10B5002200E0521C835C8C5C43
:1040D000A34201D1002BF8D1D8B2E1B2401A10BDF1
:1040E0000FF2060CDCF800C0604759AB0B0800006B
:1040F0000FF2060CDCF800C06047FD2F0B0810B56E
:10410000431A934209D28318881803E010F8011D5E
:1041100003F8011D521EF9D210BD40EA01039B07AE
:1041200003D009E008C9121F08C0042AFAD203E02C
:1041300011F8013B00F8013B521EF9D210BD0000FE
:104140002DE9F05F0746DFF82490D9F80090084E7B
:10415000D7F80880D7F800A0D7F804B018F8014BBA
:1041600059F824F0BDE8F05F7047000048030120D3
:104170004C0301200FF2060CDCF800C060477543C9
:104180000B0800000FF2060CDCF800C06047AD43DE
:104190000B08000001680029B4BF4A420A460260C9
:1041A000FFF7DCBF016850F8042C9142B4BF0B4606
:1041B00013460360FFF7D2BF016850F8042C914208
:1041C000ACBF0B4613460360FFF7C8BF0FF2060CE7
:1041D000DCF800C06047F5B80B0800000FF2060CD1
:1041E000DCF800C0604759B90B0800000FF2060C5C
:1041F000DCF800C060475DBC0B0800000FF2060C45
:10420000DCF800C0604771BC0B0800000FF2060C20
:10421000DCF800C060478DBC0B0800000000000007
:10422000000000000000000000000000000000008E
:104230004C6E008100000000748C01082001910187
:10424000C4CD0008BCCD0008C8CD000814000C0087
:10425000000000000000000000000000000000005E
:10426000456E028100000000F48C01082002A801C4
:104270007CD2000874D2000884D200081400080020
:10428000000000000000000000000000000000002E
:10429000446E028100000000048D01082002A70185
:1042A000A4D200089CD20008ACD200081400080078
:1042B00000000000000000000000000000000000FE
:1042C000436E028100000000148D01082002A60147
:1042D000CCD20008C4D20008D4D2000818000800CC
:1042E00000000000000000000000000000000000CE
:1042F000426E028100000000248D01082002A50109
:10430000F4D20008ECD20008FCD200081400080027
:10431000000000000000000000000000000000009D
:10432000416E028100000000348D01082002A401CA
:104330001CD3000814D3000824D30008140008007C
:10434000000000000000000000000000000000006D
:10435000406E028100000000448D01082002A3018C
:1043600044D300083CD300084CD3000814000800D4
:10437000000000000000000000000000000000003D
:104380004F6E018100000000548D01082002A2013F
:104390006CD3000864D3000874D30008140008002C
:1043A000000000000000000000000000000000000D
:1043B0004D6E018100000000648D01080100A00124
:1043C000CCC2000800000000000000000000000057
:1043D0004C6E018100000000748D010820019F01D6
:1043E00094D300088CD3000898D3000814000C0064
:1043F00000000000000000000000000000000000BD
:10440000426E018100000000848D010801009701C7
:10441000B4CB000800000000000000000000000015
:10442000416E018100000000948D01082001960179
:10443000B4D30008ACD30008B8D3000814000C00B3
:10444000000000000000000000000000000000006C
:104450004E6E008100000000A48D0108200293012F
:10446000D4D30008CCD30008DCD3000818000C001B
:10447000000000000000000000000000000000003C
:104480004D6E008100000000B48D010820029201F1
:10449000FCD30008F4D3000804D400081C00140066
:1044A000000000000000000000000000000000000C
:1044B000466E018100000000D48D010820029A019F
:1044C00054D400084CD400088CDC00081400080008
:1044D00000000000000000000000000000000000DC
:1044E000486E008100000000E48D010820028E016A
:1044F00084D400087CD400088CD400081000040088
:1045000000000000000000000000000000000000AB
:10451000496E018100000000F48D010820039D0117
:10452000A8D40008A0D40008B4D400081C000C00D3
:10453000000000000000000000000000000000007B
:10454000466E008100000000248E010820029D00BC
:10455000C4D50008B4D50008CCD500080C00040070
:10456000000000000000000000000000000000004B
:10457000486E008100000000348E010820012F01E8
:10458000F8D50008F0D50008FCD5000814000C0090
:10459000000000000000000000000000000000001B
:1045A000486E028100000000448E01080100AA014B
:1045B000E04D0008000000000000000000000000C6
:1045C000416E028100000000548E010801001D00B0
:1045D0003CCB0008000000000000000000000000CC
:1045E0004D6E008100000000648E0108200442002E
:1045F00044D7000838D6000854D700081400040037
:1046000000000000000000000000000000000000AA
:10461000496E008100000000748E010820044000F3
:10462000A0D8000898D70008B0D8000814000400EB
:10463000000000000000000000000000000000007A
:10464000476E008100000000948E010820012E01B9
:104650001CD9000814D9000820D900081000040053
:10466000000000000000000000000000000000004A
:104670004A6E008100000000A48E010828010E008F
:104680003CD900080000000000E700080800000016
:10469000C027020800000000000000000000000029
:1046A000456E028100000000B48E01082001220046
:1046B00088D9000800000000ACDD000814000C00E0
:1046C00000000000000000000000000000000000EA
:1046D0004B6E018100000000D48E010801003A01F8
:1046E000FCCB0008000000000000000000000000FB
:1046F000426E018100000000E48E01082001CA0121
:1047000054DC00084CDC0008605601080C00040072
:104710000000000000000000000000000000000099
:10472000476E018100000000F48E010830019B01FA
:1047300088DC0008000000008CDC00080800000095
:104740000840020800000000000000000000000017
:104750004F6E038100000000048F01080100400239
:10476000D07F0008000000000000000000000000F2
:10477000466E028100000000348F010820012300F2
:104780006CDD000864DD000870DD0008280008000A
:104790000000000000000000000000000000000019
:1047A000446E028100000000448F010830012100A6
:1047B000A8DD0008A0DD0008ACDD00080C0000004A
:1047C00090660208000000000000000000000000E9
:1047D0004C6E008100000000548F01083005D600A7
:1047E000F0590108E0840108F88401081C00100059
:1047F0006447020800000000000000000000000004
:104800004B6E028100000000648F01082001280027
:1048100004DE0008FCDD000808DE000814000C00BF
:104820000000000000000000000000000000000088
:104830004B6E018100000000748F010820029E0170
:104840002CDE00081CDE000834DE00080C0004002A
:104850000000000000000000000000000000000058
:10486000446E038100000000A48F01082001610054
:1048700088DE000880DE0008202901081C000000F6
:104880000000000000000000000000000000000028
:104890004E6E018100000000C48F01082001A101BB
:1048A00064DF00085CDF000868DF00081000080013
:1048B00000000000000000000000000000000000F8
:1048C0004E6E018100000000D48F010801003C0100
:1048D00070B00008000000000000000000000000B0
:1048E000486E018100000000E48F010830012902B8
:1048F000B4DF0008ACDF0008B8DF000808000000E3
:10490000F872020800000000000000000000000033
:10491000466E018100000000F48F0108300127027B
:10492000D8DF0008D0DF0008DCDF00080800000046
:104930000C730208000000000000000000000000EE
:10494000456E01810000000004900108300126023C
:10495000FCDF0008F4DF000800E0000808000000A9
:1049600020730208000000000000000000000000AA
:10497000436E018100000000149001083001240200
:1049800020E0000818E0000824E00008080000000B
:104990003473020800000000000000000000000066
:1049A000426E0181000000002490010830012302C2
:1049B00044E000083CE0000848E00008080000006F
:1049C0004873020800000000000000000000000022
:1049D000416E018100000000349001083001220284
:1049E00068E0000860E000086CE0000808000000D3
:1049F0005C730208000000000000000000000000DE
:104A0000406E018100000000449001083001210245
:104A10008CE0000884E0000890E000080800000036
:104A20007073020800000000000000000000000099
:104A30004E6E0081000000005490010830011F02FA
:104A4000B0E00008A8E00008B4E00008080000009A
:104A50008473020800000000000000000000000055
:104A60004D6E0081000000006490010830011E02BC
:104A7000D4E00008CCE00008D8E0000808000000FE
:104A80009873020800000000000000000000000011
:104A90004C6E0081000000007490010830011D027E
:104AA000F8E00008F0E00008FCE000080800000062
:104AB000AC730208000000000000000000000000CD
:104AC000436E00810000000084900108300117024D
:104AD0001CE1000814E1000820E1000808000000C3
:104AE000C073020800000000000000000000000089
:104AF000426E00810000000094900108300116020F
:104B000040E1000838E1000844E100080800000026
:104B1000D473020800000000000000000000000044
:104B20004F6E038100000000A490010830011502BF
:104B300064E100085CE1000868E10008080000008A
:104B4000E873020800000000000000000000000000
:104B5000406E018100000000B490010820034E0265
:104B60006865010800000000A0E1000810000800CE
:104B70000000000000000000000000000000000035
:104B80004D6E008100000000C490010830014B020E
:104B900024E20008BCE1000828E200080C00040040
:104BA0005474020800000000000000000000000033
:104BB0004D6E018100000000D490010830013B01DE
:104BC0006CE200080000000018EB0008100008006C
:104BD000A4530208000000000000000000000000D4
:104BE000476E008100000000E490010820039F0050
:104BF0008872010818E3000850E30008380020001C
:104C000000000000000000000000000000000000A4
:104C1000486E028100000000F49001082002D901D2
:104C20007052010824E400082CE4000828000C005D
:104C30000000000000000000000000000000000074
:104C40004E6E008100000000049101080100C601C1
:104C5000E0A50008000000000000000000000000C7
:104C6000476E018100000000149101082004FD013D
:104C70005C7F0108E0840108F88401081C00100032
:104C80003480020800000000000000000000000066
:104C9000496E0181000000002491010820020E01EC
:104CA0007481010860E4000868E40008280014002A
:104CB00000000000000000000000000000000000F4
:104CC000436E038100000000349101082001E201DD
:104CD000A0E4000898E40008A4E400080C00040024
:104CE00000000000000000000000000000000000C4
:104CF000486E0181000000004491010820029C01DF
:104D0000C0E40008B8E40008C8E400081400080083
:104D10000000000000000000000000000000000093
:104D2000486E008100000000549101080100F2016A
:104D3000B053000800000000000000000000000068
:104D4000476E0281000000006491010801004201E9
:104D500030B6000800000000000000000000000065
:104D6000496E008100000000749101080100A1005B
:104D70004054000800000000000000000000000097
:104D8000456E008100000000849101082001C001EF
:104D900068E5000860E50008041101080C00040043
:104DA0000000000000000000000000000000000003
:104DB0004A6E028100000000949101082001AC01BC
:104DC0008CE5000884E5000890E500081000040068
:104DD00000000000000000000000000000000000D3
:104DE000496E028100000000A49101082003AB017C
:104DF000A4E50008000000000C8401082000140055
:104E000000000000000000000000000000000000A2
:104E10004B6E008100000000B491010830010F00CA
:104E200000E600080000000000E70008080000009D
:104E3000B85B020800000000000000000000000055
:104E4000436E018100000000C49101082001980117
:104E50000CE6000804E6000810E600081000080050
:104E60000000000000000000000000000000000042
:104E70004F6E008100000000D49101082001C7019D
:104E800054E600084CE6000858E600081000080048
:104E90000000000000000000000000000000000012
:104EA000416E008100000000F491010810023800FA
:104EB000103D0108CCE60008D4E600081400040008
:104EC0002481020800000000000000000000000033
:104ED000496E0081000000000492010820020D00CC
:104EE000F8E60008E8E6000800E700080C00040007
:104EF00000000000000000000000000000000000B2
:104F0000476E008100000000149201082002080092
:104F100034E7000824E700083CE700080C00040020
:104F20000000000000000000000000000000000081
:104F3000486E0081000000002492010830040C003B
:104F40001C5C0108E0840108F88401081C001000C2
:104F50005C5F02080000000000000000000000008C
:104F6000436E0281000000006492010820032000CB
:104F70006053010850530108C0E700081000080002
:104F80000000000000000000000000000000000021
:104F9000426E0281000000007492010820011E0090
:104FA000FCE70008F4E7000800E80008100008002B
:104FB00000000000000000000000000000000000F1
:104FC0004A6E02810000000084920108200227003E
:104FD0001CE8000814E8000824E800081000080095
:104FE00000000000000000000000000000000000C1
:104FF000466E028100000000C49201082002A9014F
:1050000034E900082CE900083CE900081400080015
:105010000000000000000000000000000000000090
:10502000436E038100000000E49201082001490161
:1050300038EA00088CE900083CEA00081000080083
:105040000000000000000000000000000000000060
:10505000466E038100000000F492010800043A0249
:105060002801010870EA0008BCEA000814000C00DE
:105070000000000000000000000000000000000030
:105080004A6E0181000000000493010820014B00DA
:10509000ECEA0008E4EA0008F0EA00080C0000006E
:1050A0000000000000000000000000000000000000
:1050B0004F6E0181000000001493010801004F00B1
:1050C0002077000800000000000000000000000041
:1050D000426E01810000000024930108200172004B
:1050E0000CEB000804EB0008604F010828000C00DE
:1050F00000000000000000000000000000000000B0
:105100004E6E0081000000003493010801006E0023
:1051100050770008000000000000000000000000C0
:10512000496E01810000000044930108200238010B
:105130004CEC000810EB000818EB000814000C0001
:10514000000000000000000000000000000000005F
:10515000496E0081000000005493010820013001D5
:1051600034EB00082CEB000838EB0008200010009E
:10517000000000000000000000000000000000002F
:10518000426E018100000000649301082001920238
:1051900074EB00086CEB000878EB000810000400CA
:1051A000DCBA02080000000000000000000000005F
:1051B000466E038100000000749301083001120262
:1051C0009CEB000894EB0008606C010808000000EC
:1051D000ECBF02080000000000000000000000001A
:1051E0004F6E028100000000A493010820012A00F4
:1051F00024EC00081CEC000828EC0008180004004F
:10520000000000000000000000000000000000009E
:105210004F6E018100000000C49301082001370196
:105220004CEC000844EC000854EC000810000800A6
:10523000000000000000000000000000000000006E
:105240004D6E0181000000000494010820014E0011
:10525000CCEC0008C0EC0008A43D01080C000000E4
:10526000000000000000000000000000000000003E
:10527000436E0281000000001494010800025300F4
:10528000D84A0108D0EC000800ED0008180008001A
:10529000000000000000000000000000000000000E
:1052A000416E008100000000B494010820029A00C1
:1052B00028ED000818ED0008B84301080C000400B0
:1052C00000000000000000000000000000000000DE
:1052D0004E6E008100000000149501082001F701C6
:1052E00040ED000838ED000844ED00080C00040013
:1052F00000000000000000000000000000000000AE
:10530000476E028100000000249501080002080297
:10531000BC7B01080000000058ED000850000C00A4
:10532000000000000000000000000000000000007D
:10533000446E00810000000034950108300118021D
:105340008CED000884ED00086C46010808000000A0
:10535000B48202080000000000000000000000000D
:105360004D6E0381000000004495010801003F02DA
:105370006CBC0008000000000000000000000000FD
:105380004B6E0181000000005495010820020102CB
:105390002859010800000000305901082C001400B1
:1053A00000000000000000000000000000000000FD
:1053B000496E008100000000649501083002F4018C
:1053C000FC44010800000000A0ED00080C000400EF
:1053D00078DD02080000000000000000000000006E
:1053E000466E028100000000749501083002410100
:1053F0002C3D01080CEE000814EE00080C0004001F
:1054000094DE020800000000000000000000000020
:10541000406E018100000000849501082002A80070
:1054200040EE000838EE00080440010814000C00AB
:10543000000000000000000000000000000000006C
:105440004A6E008100000000949501082002A3002C
:10545000BC3F01080000000048EE000814000C00EA
:10546000000000000000000000000000000000003C
:105470004A6E038100000000A49501082001B901D3
:1054800068EE000860EE0008FC47010820000800F4
:10549000000000000000000000000000000000000C
:1054A000436E038100000000C495010820018F00B5
:1054B0006CEE000800000000403E01080C000000F7
:1054C00000000000000000000000000000000000DC
:1054D000496E038100000000D49501082002F2000B
:1054E00078EE000870EE000880EE000824000C0042
:1054F00000000000000000000000000000000000AC
:10550000496E038100000000E49501081004500179
:10551000B8EE00080000000098EE0008200010001F
:1055200098E20208000000000000000000000000F7
:105530004A6E038100000000F495010800034F014A
:10554000B8EE000800000000C8EE000820001000BF
:10555000000000000000000000000000000000004B
:10556000486E0381000000000496010800034E010C
:10557000AC010108E8EE000834EF000814000C004C
:10558000000000000000000000000000000000001B
:105590004A6E008100000000149601083001D3001B
:1055A0005CEF000800000000742C010808000000F7
:1055B000148E02080000000000000000000000003F
:1055C000406E01810000000064960108000395010F
:1055D0008C64010894EF0008505701082000140063
:1055E00000000000000000000000000000000000BB
:1055F000496E008100000000749601082002FC0042
:1056000008F3000800000000BCEF000818000000CC
:10561000000000000000000000000000000000008A
:105620004D6E008100000000849601082001F60103
:10563000D4EF000800000000F4F700081C000C0084
:10564000000000000000000000000000000000005A
:10565000486E018100000000949601082002FF01BD
:1056600054260108F0EF0008F05A01081400080061
:10567000000000000000000000000000000000002A
:10568000476E018100000000A496010820020C0171
:10569000F8EF0008000000003C5C01081400000066
:1056A00000000000000000000000000000000000FA
:1056B0004D6E008100000000B496010820036D00CB
:1056C00000F00008E0840108F88401081C001000C4
:1056D00000000000000000000000000000000000CA
:1056E000486E038100000000C496010820011302E7
:1056F00014F000080CF00008185E01080C0004000B
:105700000000000000000000000000000000000099
:105710004A6E008100000000D496010820018F012C
:1057200034F0000818F00008005D01080C000400C7
:105730000000000000000000000000000000000069
:10574000496E028100000000E49601082003560023
:10575000185D0108E0840108F884010820001400A5
:105760000000000000000000000000000000000039
:105770004C6E038100000000F49601083003BB0169
:1057800038F00008E0840108F88401081C001000CB
:1057900024A5020800000000000000000000000036
:1057A000476E0281000000000497010800032500F5
:1057B000A0FD0008FCF0000804F10008280020000B
:1057C00000000000000000000000000000000000D9
:1057D000406E018100000000349701082002430060
:1057E000A0F2000868F10008A8F200081C000800F8
:1057F00000000000000000000000000000000000A9
:10580000406E0381000000004497010830015D00F4
:10581000F0F20008000000002029010850000000FC
:10582000F406030800000000000000000000000073
:105830004B6E0281000000005497010820045800BC
:10584000F4F2000800000000202901081000040004
:105850000000000000000000000000000000000048
:105860004F6E0081000000008497010830010301A1
:1058700004F30008000000001C00010808000000FC
:105880001CAE020800000000000000000000000044
:105890004C6E008100000000A49701082002000166
:1058A00010F300080000000018F3000810000800C2
:1058B00000000000000000000000000000000000E8
:1058C0004A6E018100000000B497010830012B02EC
:1058D00034F300082CF30008DC690108080000001C
:1058E000D0AE020800000000000000000000000030
:1058F0004E6E038100000000C4970108000485017A
:10590000FC8301080000000038F3000824001400A4
:105910000000000000000000000000000000000087
:10592000436E038100000000D4970108300210028A
:10593000FC6D010800000000606C01081400080004
:10594000D0BF0208000000000000000000000000BE
:10595000446E018100000000E49701082001FA0173
:1059600020F4000818F40008BC6D010814000C00B5
:105970000000000000000000000000000000000027
:10598000426E038100000000F49701083001830299
:105990002CF4000824F40008945A010808000000C0
:1059A000D410030800000000000000000000000008
:1059B000416E01810000000004980108010071009F
:1059C000D0500008000000000000000000000000AF
:1059D000496E03810000000014980108200365004F
:1059E00068F500080000000074F5000810000400CD
:1059F00000000000000000000000000000000000A7
:105A0000486E008100000000349801082003A000C7
:105A1000D07C010800000000E8F500080C0004003C
:105A20000000000000000000000000000000000076
:105A30004A6E0081000000004498010820013101F5
:105A40001CF6000814F60008707D0108100008001C
:105A50000000000000000000000000000000000046
:105A60004D6E008100000000549801082001C5011E
:105A700090F6000888F6000894F600080C00040070
:105A80000000000000000000000000000000000016
:105A9000496E008100000000649801082001C301E4
:105AA000B0F60008A8F60008C0F6000810000800CC
:105AB00000000000000000000000000000000000E6
:105AC000486E008100000000749801083001C20196
:105AD000BCF60008B4F60008C0F600080800000094
:105AE000E03D03080000000000000000000000008E
:105AF000426E0281000000008498010830027A02A0
:105B0000E4F60008D4F60008204801080800000068
:105B1000883E0308000000000000000000000000B4
:105B2000466E038100000000949801082801E601F8
:105B3000ECF6000800000000D85B01080800000037
:105B400050C2020800000000000000000000000039
:105B5000476E008100000000A498010820013E006B
:105B600058F7000850F700085CF700080C00040024
:105B70000000000000000000000000000000000025
:105B8000466E008100000000B498010820013D002D
:105B900084F700087CF7000888F700080C00040070
:105BA00000000000000000000000000000000000F5
:105BB000456E008100000000C498010820013C00EF
:105BC000A4F700089CF70008A8F700080C000400E0
:105BD00000000000000000000000000000000000C5
:105BE000456E028100000000F498010820010502C2
:105BF000BC450108BCF70008C4F700081400040005
:105C00000000000000000000000000000000000094
:105C1000426E008100000000049901082002430246
:105C2000B8010108000000002071010820001800E0
:105C30000000000000000000000000000000000064
:105C40004C6E01810000000014990108200203023B
:105C5000E03C010800000000C4F700081400080040
:105C60000000000000000000000000000000000034
:105C70004A6E008100000000249901083002F501FD
:105C8000ECF70008E4F70008F4F70008100008003B
:105C90005CDD0208000000000000000000000000C1
:105CA000436E008100000000349901083001F001CA
:105CB0000CF8000800000000940001080800000033
:105CC00098DD020800000000000000000000000055
:105CD000486E02810000000044990108300243012F
:105CE00018F8000810F80008F879010810000800FA
:105CF00078DE020800000000000000000000000044
:105D0000426E018100000000549901083001A90091
:105D100020F800080000000004400108080000000E
:105D2000B4DE0208000000000000000000000000D7
:105D30004D6E038100000000649901082001640297
:105D40002444010800000000285801081000080041
:105D50000000000000000000000000000000000043
:105D6000416E038100000000749901082002EA00DE
:105D70006CF9000864F9000874F9000820000800B4
:105D80000000000000000000000000000000000013
:105D90004F6E028100000000849901083002DD018D
:105DA0001C520108000000002852010818000C00D5
:105DB00080EB02080000000000000000000000006E
:105DC000466E0081000000009499010820052D0115
:105DD000F85B0108E0840108F88401082000140041
:105DE00000000000000000000000000000000000B3
:105DF0004C6E038100000000A499010820033600C6
:105E00002C5C01080000000084FA0008180008005B
:105E1000D075030800000000000000000000000032
:105E20004C6E038100000000B49901083001270185
:105E3000ACFB0008000000009C7501080800000091
:105E4000B0EF0208000000000000000000000000A9
:105E5000446E008100000000C49901082002730212
:105E6000E8350108B0FB0008C4FB0008240010005E
:105E70000000000000000000000000000000000022
:105E80004A6E008100000000D49901080001FD0065
:105E9000ECFB000800000000F0FB00081400040008
:105EA00000000000000000000000000000000000F2
:105EB0004B6E008100000000E499010870016B0046
:105EC00008FC000800FC00080CFC00080C000400A2
:105ED00038830308000000000000000000000000FC
:105EE0004A6E008100000000F499010830016A0048
:105EF00024FC000800000000CC0601080800000097
:105F0000ECF20208000000000000000000000000A9
:105F1000496E018100000000049A01083001D2019D
:105F200040FC000800000000A43001080800000048
:105F300030F3020800000000000000000000000034
:105F4000496E038100000000149A0108200431000A
:105F5000045F010800000000981E010868001C0092
:105F60000000000000000000000000000000000031
:105F70004D6E008100000000249A01082002D70025
:105F80000C5301084CFD00085CFD000818000C00D3
:105F90000000000000000000000000000000000001
:105FA0004C6E028100000000449A01082001240088
:105FB000A0FD000898FD0008ACFD000810000800D6
:105FC00000000000000000000000000000000000D1
:105FD000426E018100000000549A01082002050170
:105FE000F8FD0008000000008443010820000400C0
:105FF00000000000000000000000000000000000A1
:10600000416E028100000000649A0108200206022D
:10601000BC45010800FE0008A4FE0008280010008E
:106020000000000000000000000000000000000070
:10603000416E018100000000749A010830014400A3
:10604000F0FE0008E8FE0008F4FE0008080000006A
:10605000149403080000000000000000000000008D
:10606000436E018100000000849A01083001450060
:1060700010FF000808FF000814FF000808000000D7
:106080004C94030800000000000000000000000025
:10609000466E018100000000949A010830024D0212
:1060A000686501080000000038FF00080C000400CB
:1060B0007C06030800000000000000000000000053
:1060C0004E6E028100000000A49A010801005B00EE
:1060D000E060000800000000000000000000000078
:1060E0004F6E028100000000B49A010830015C008C
:1060F000C4FF000800000000202901083000000053
:106100007C9903080000000000000000000000006F
:106110004D6E028100000000C49A010820035A005D
:10612000D0FF0008C8FF0008202901081C00080053
:10613000000000000000000000000000000000005F
:106140004C6E028100000000D49A01080100590041
:10615000C4BB0008000000000000000000000000B8
:10616000406E018100000000E49A01082002040151
:10617000F4FF000800000000FCFF00081800040005
:10618000000000000000000000000000000000000F
:106190004E6E008100000000F49A01082002020106
:1061A00014000108000000001C0001081C0004008D
:1061B00000000000000000000000000000000000DF
:1061C0004D6E008100000000049B010820020101C7
:1061D00034000108000000003C0001081800040021
:1061E00000000000000000000000000000000000AF
:1061F000486E038100000000149B010828018602FC
:106200006C00010800000000945A0108080000001A
:10621000F40A030800000000000000000000000075
:10622000446E028100000000249B0108200132021C
:106230007000010800000000DC6901082800180057
:10624000000000000000000000000000000000004E
:106250004A6E038100000000449B01083001E901FF
:106260008400010800000000D85B0108080000005D
:10627000440F0308000000000000000000000000C0
:106280004F6E038100000000549B01082001EE01C5
:10629000900001088800010894000108200008000F
:1062A00000000000000000000000000000000000EE
:1062B0004B6E008100000000649B01082002D400A6
:1062C000A47B0108A8000108B800010818000C0010
:1062D00000000000000000000000000000000000BE
:1062E000476E038100000000849B0108000339020F
:1062F00028010108DC0001083801010814000C0025
:10630000000000000000000000000000000000008D
:10631000456E008100000000A49B0108200142029C
:10632000B801010800000000207101081C001400E1
:10633000000000000000000000000000000000005D
:10634000426E008100000000D49B0108200267001B
:106350000802010800000000CC0601081800040033
:10636000000000000000000000000000000000002D
:106370004D6E038100000000E49B01082801F50038
:10638000100201080000000010420108080000008F
:106390004C11030800000000000000000000000095
:1063A000496E008100000000F49B010801007402A6
:1063B0009CBC00080000000000000000000000007D
:1063C000456E018100000000049C01083001FB01C2
:1063D0004C02010800000000BC6D0108080000002C
:1063E000A4130308000000000000000000000000EB
:1063F0004F6E028100000000149C010830010C0265
:106400000C460108000000005002010808000000CE
:10641000C8A7030800000000000000000000000002
:106420004A6E038100000000249C01082002F30052
:10643000840201087C0201088C0201082000080087
:10644000000000000000000000000000000000004C
:10645000436E018100000000349C01082801060100
:10646000A4020108000000008443010808000000A5
:10647000D01403080000000000000000000000002D
:106480004C6E008100000000449C01082004A6001E
:10649000A8020108000000000C8401082800180070
:1064A00000000000000000000000000000000000EC
:1064B000496E038100000000649C010830018702DE
:1064C0006006010800000000945A0108080000005E
:1064D000A4340308000000000000000000000000D9
:1064E000446E028100000000749C010830018300AA
:1064F0006406010800000000287A01080800000076
:10650000B834030800000000000000000000000094
:106510004E6E038100000000949C01082003660079
:10652000B006010800000000CC06010814000800B5
:10653000000000000000000000000000000000005B
:10654000466E008100000000A49C01082002690042
:10655000C4060108BC060108CC0601082400080096
:10656000000000000000000000000000000000002B
:106570004C6E018100000000C49C01082001150040
:10658000B07C0108A87C0108B87C01080C0004005C
:1065900000000000000000000000000000000000FB
:1065A000416E038100000000E49C01082801820282
:1065B00060080108000000002048010808000000F1
:1065C0007436030800000000000000000000000016
:1065D000456E008100000000049D01082004FE00BB
:1065E0004043010838430108300A01082800180018
:1065F000000000000000000000000000000000009B
:106600004E6E038100000000149D01082801ED0179
:106610005C0A010800000000D85B010808000000C7
:1066200080390308000000000000000000000000A6
:10663000426E008100000000249D0108200101003D
:106640000C570108600A01089C8001080C00040036
:1066500068DE0308000000000000000000000000E9
:106660004B6E028100000000549D010830010A02B7
:10667000F00B0108000000003826010808000000A7
:1066800018410308000000000000000000000000A6
:10669000446E028100000000649D010820023F0159
:1066A0004C0C010800000000640C010814000400F8
:1066B00000000000000000000000000000000000DA
:1066C000426E028100000000749D010820023E011C
:1066D0005C0C0108540C0108640C01080C00040057
:1066E00000000000000000000000000000000000AA
:1066F000486E018100000000849D010820013601E0
:10670000800C0108780C0108840C010808000000C6
:10671000CCBD0308000000000000000000000000E5
:10672000446E018100000000949D01082002460093
:10673000DC0C0108980C01085C3D01081400040001
:106740000000000000000000000000000000000049
:106750004F6E038100000000A49D01080100F600B7
:10676000907A000800000000000000000000000017
:106770004C6E038100000000B49D01083001EB0164
:106780005C0F010800000000D85B01080800000051
:10679000B84C0308000000000000000000000000EA
:1067A0004C6E018100000000D49D010828011101F8
:1067B0006C0F0108000000003C5C010808000000AC
:1067C000CC4C0308000000000000000000000000A6
:1067D000436E028100000000E49D01083001D601F3
:1067E000880F010800000000AC2B01080800000021
:1067F000C04D030800000000000000000000000081
:10680000486E038100000000049E010830016A0206
:10681000DC0F0108000000002C4401080800000003
:10682000184F0308000000000000000000000000F6
:106830004C6E018100000000149E010830015702D7
:106840005444010800000000F00F01080800000097
:10685000E0C303080000000000000000000000008A
:10686000466E008100000000349E01087001C101E5
:1068700000110108000000000411010818001000B8
:106880002483030800000000000000000000000056
:10689000466E038100000000449E0108200463004E
:1068A000201101081811010830110108100004001E
:1068B00000000000000000000000000000000000D8
:1068C000456E028100000000549E01082001D7019E
:1068D0007011010800000000AC2B01081400040036
:1068E00018C80308000000000000000000000000BD
:1068F000486E008100000000649E01082002D10063
:10690000F414010800000000FC1401080800000055
:10691000BCD60308000000000000000000000000DA
:10692000416E028100000000749E01082003B60041
:106930003878010820150108307D010814000C008A
:106940000000000000000000000000000000000047
:10695000486E028100000000849E0108200361024D
:10696000F0830108000000000C84010820001400DE
:106970000000000000000000000000000000000017
:10698000446E018100000000949E010800039901FB
:10699000E4660108A4160108B41601080C000400FE
:1069A00000000000000000000000000000000000E7
:1069B000456E038100000000A49E01082001ED0047
:1069C00000170108F8160108041701080C0004005C
:1069D00000000000000000000000000000000000B7
:1069E000416E038100000000C49E010820014601A1
:1069F000CC180108C4180108D018010810000400C0
:106A00000000000000000000000000000000000086
:106A1000476E008100000000D49E010800026E0253
:106A20001C350108201901082C1901081000040068
:106A30000000000000000000000000000000000056
:106A4000426E008100000000E49E010820023A002E
:106A5000A81D010800000000305901083000100096
:106A60000000000000000000000000000000000026
:106A70004E6E038100000000F49E010830023700D2
:106A8000C81D0108B01D0108D01D01081000040038
:106A900020E10308000000000000000000000000EA
:106AA0004B6E038100000000049F01083003350095
:106AB000F068010800000000F81D01081800080037
:106AC00018E20308000000000000000000000000C1
:106AD0004A6E038100000000149F01083003330058
:106AE00060490108000000003C1E01082800180051
:106AF000E475030800000000000000000000000032
:106B0000486E038100000000249F01082005320028
:106B1000045F010800000000981E010868001C00C6
:106B20000000000000000000000000000000000065
:106B3000456E038100000000349F010820034C01D2
:106B4000743B0108441F0108F01F010820000C00DD
:106B50000000000000000000000000000000000035
:106B6000406E018100000000449F01082002C8011E
:106B70003020010824200108382001080C000400FE
:106B80000000000000000000000000000000000005
:106B9000466E018100000000549F010800020B01B5
:106BA0004069010800000000486901081400040061
:106BB00000000000000000000000000000000000D5
:106BC000456E018100000000649F01080002090178
:106BD0007421010800000000C47B0108540010006B
:106BE00000000000000000000000000000000000A5
:106BF000476E018100000000749F01080001CF0171
:106C00005422010800000000582201081C000C005A
:106C10000000000000000000000000000000000074
:106C2000456E008100000000849F01083001CE0005
:106C30009822010800000000B47301080800000059
:106C400008EC030800000000000000000000000045
:106C5000406E038100000000A49F010820018E0007
:106C6000442301083C2301084823010814000400C0
:106C70000000000000000000000000000000000014
:106C8000416E028100000000C49F010830038000B3
:106C90005824010848240108287A0108100004003B
:106CA00008F10308000000000000000000000000E0
:106CB000496E018100000000D49F010830011300DB
:106CC0006C240108642401087024010808000000F5
:106CD00080F1030800000000000000000000000038
:106CE000486E018100000000E49F0108300112009D
:106CF0009024010888240108942401080800000059
:106D000094F10308000000000000000000000000F3
:106D1000476E018100000000F49F010830017600F9
:106D2000DC240108AC240108A876010818000C0036
:106D3000F8F7030800000000000000000000000059
:106D4000496E02810000000004A0010830038800A1
:106D50009073010828250108287A01081000040012
:106D600088F8030800000000000000000000000098
:106D7000496E02810000000014A0010830010902E0
:106D800034260108282601083826010808000000DA
:106D90005CFC030800000000000000000000000090
:106DA000496E01810000000024A001083001FE01AD
:106DB000542601084C2601085C2601080C0000003E
:106DC00070FC03080000000000000000000000004C
:106DD0004B6E03810000000044A001082002F40073
:106DE000FC260108F42601081042010820000800D2
:106DF0000000000000000000000000000000000093
:106E0000456E03810000000054A0010820014A01E2
:106E1000C03A010804270108803B0108180004005B
:106E20000000000000000000000000000000000062
:106E3000426E03810000000064A001082001EB0005
:106E400004280108FC270108082801080C00040098
:106E50000000000000000000000000000000000032
:106E6000456E03810000000074A00108300162003B
:106E700004290108FC280108202901080C0004004D
:106E8000500904080000000000000000000000009D
:106E9000426E03810000000084A00108200260000F
:106EA000103E010808290108202901081C000C00D7
:106EB00000000000000000000000000000000000D2
:106EC0004A6E02810000000094A0010820035700D0
:106ED0003C2901083429010848290108140004004C
:106EE00000000000000000000000000000000000A2
:106EF000486E038100000000A4A001082003640084
:106F000060290108000000006C2901081C000C0029
:106F10000000000000000000000000000000000071
:106F2000416E038100000000C4A0010830045F002E
:106F30008C290108802901089C29010824001400DB
:106F4000589C030800000000000000000000000042
:106F50004B6E028100000000D4A0010828016202EB
:106F60009C2B0108000000002858010818000000B0
:106F7000449D030800000000000000000000000025
:106F80004F6E018100000000E4A001082001D5013E
:106F9000A82B0108A02B0108AC2B01081800080041
:106FA00000000000000000000000000000000000E1
:106FB000496E008100000000F4A001082002D20008
:106FC000444C010800000000742C01080800000077
:106FD0009014040800000000000000000000000001
:106FE000406E03810000000004A101082001E900B7
:106FF0009C2C0108942C0108A02C0108100008000A
:107000000000000000000000000000000000000080
:10701000446E02810000000014A101082003B900A1
:10702000B42C010800000000306501080C000400C9
:107030000000000000000000000000000000000050
:10704000456E01810000000024A101080100CD016E
:10705000E0620008000000000000000000000000E6
:10706000436E03810000000034A101082001EC0000
:10707000202D0108182D0108242D010810000400FE
:107080000000000000000000000000000000000000
:10709000456E02810000000044A101080100840047
:1070A000B4BC000800000000000000000000000068
:1070B000426E01810000000034BE01080100DA00C8
:1070C00030B40008000000000000000000000000D4
:1070D000436E02810000000054A1010820018200DB
:1070E000B82D0108B02D0108287A010818001000F9
:1070F0000000000000000000000000000000000090
:10710000466E03810000000064A101080100EE004A
:1071100020A00008000000000000000000000000A7
:10712000416E02810000000074A1010830015C0280
:10713000943001088C30010828580108080000002C
:107140003C1F0408000000000000000000000000D8
:10715000436E01810000000084A101082001CB01E1
:10716000A030010898300108A43001081000040084
:10717000000000000000000000000000000000000F
:107180004D6E03810000000094A10108200152010E
:10719000C4300108BC300108C83001080C000400EC
:1071A00000000000000000000000000000000000DF
:1071B0004A6E018100000000F4C0010801001400C3
:1071C0006CCB000800000000000000000000000080
:1071D000496E028100000000A4A101080001E40042
:1071E0008431010800000000883101081400080003
:1071F000000000000000000000000000000000008F
:10720000426E038100000000B4A10108000448019F
:1072100040530108C0330108E83301081800040096
:10722000000000000000000000000000000000005E
:10723000446E038100000000C4A10108000347015F
:107240004053010860340108843401081800040028
:10725000000000000000000000000000000000002E
:10726000416E008100000000D4A1010800036F02FC
:107270001C3501080C3501082835010814000800E8
:1072800000000000000000000000000000000000FE
:10729000476E008100000000E4A1010800044802DC
:1072A000685B01081C5B01086C35010824000C00B8
:1072B00000000000000000000000000000000000CE
:1072C000426E028100000000F4A101082001B70015
:1072D000DC350108D0350108307D01080C000400C0
:1072E000000000000000000000000000000000009E
:1072F000456E00810000000004A201082001720216
:10730000E8350108E0350108F035010818000800EB
:10731000000000000000000000000000000000006D
:10732000436E01810000000024A2010820017300C7
:107330002839010820390108604F01081C000C00A1
:10734000000000000000000000000000000000003D
:10735000436E00810000000034A2010801005601C4
:107360001CCD00080000000000000000000000002C
:10737000456E00810000000044A20108300368004F
:10738000243A0108E0840108303A01082000100086
:1073900054B60308000000000000000000000000D8
:1073A000416E03810000000054A20108200268021F
:1073B000C03A0108B83A01082C4401081C00080032
:1073C00000000000000000000000000000000000BD
:1073D000466E03810000000064A2010820024B01F8
:1073E000743B0108C83A0108803B01081C000800F2
:1073F000000000000000000000000000000000008D
:10740000446E00810000000074A2010830010500F4
:10741000F43B010800000000B079010808000000FA
:1074200038BD03080000000000000000000000005C
:10743000496E00810000000084A2010828018E022C
:10744000043C0108F83B0108244C01080800000036
:107450004CBD030800000000000000000000000018
:107460004C6E018100000000A4A2010820027702F6
:10747000083C010800000000103C01080C0004005A
:1074800000000000000000000000000000000000FC
:10749000476E008100000000B4A2010801008C02C8
:1074A000B0B4000800000000000000000000000070
:1074B000466E028100000000C4A2010800026002C2
:1074C000383C01082C3C0108287E0108100004000B
:1074D00000000000000000000000000000000000AC
:1074E000456E028100000000D4A2010801005F0285
:1074F000B074000800000000000000000000000060
:10750000406E028100000000E4A2010820011C007E
:10751000403C0108000000005C6F0108080000000A
:10752000000000000000000000000000000000005B
:10753000406E038100000000F4A2010830022B001D
:1075400050780108443C01089C3C010814000400E8
:1075500088D60308000000000000000000000000C2
:107560004E6E01810000000004A301082001020208
:10757000E03C010800000000E83C010810000400A5
:1075800000000000000000000000000000000000FB
:10759000456E03810000000024A301082001E501DD
:1075A000203D0108183D0108D85B010808000000D3
:1075B000304404080000000000000000000000004B
:1075C000496E02810000000034A30108300140012F
:1075D0002C3D0108243D0108343D01080C00040045
:1075E000004504080000000000000000000000004A
:1075F000476E01810000000044A3010830014800EB
:10760000583D0108000000005C3D01081000080022
:1076100064460408000000000000000000000000B4
:107620004C6E01810000000054A3010800024D00CF
:10763000903D0108843D0108287E010810000400E7
:10764000000000000000000000000000000000003A
:107650004B6E01810000000064A3010801004C0092
:10766000207600080000000000000000000000007C
:10767000406E02810000000084A301083001500028
:10768000A03D010800000000A43D01080800000022
:1076900074BF0308000000000000000000000000AC
:1076A000426E00810000000094A3010820039B00AB
:1076B000B83D010800000000B84301081C000800A4
:1076C00000000000000000000000000000000000BA
:1076D000426E028100000000A4A3010800025200D3
:1076E000D03D0108C43D0108287E010810000400B7
:1076F000000000000000000000000000000000008A
:10770000416E028100000000B4A301080100510095
:10771000D07600080000000000000000000000001B
:10772000446E028100000000C4A30108000154005F
:10773000E43D0108D83D0108E83D010814000800B7
:107740000000000000000000000000000000000039
:10775000406E018100000000E4A3010820017000D8
:10776000203E0108183E0108604F010820000C006F
:107770000000000000000000000000000000000009
:107780004F6E008100000000F4A3010820016F008B
:107790002C3E0108243E0108604F01080C00000047
:1077A00000000000000000000000000000000000D9
:1077B0004E6E02810000000004A4010830018C001C
:1077C000303E010800000000403E010808000000B3
:1077D0007CC0030800000000000000000000000062
:1077E0004D6E02810000000014A4010828018B00E6
:1077F0003C3E0108343E0108403E010808000000FC
:1078000090C003080000000000000000000000001D
:10781000456E03810000000024A4010820039000AD
:10782000B03F0108543E0108145101082C0010001B
:107830000000000000000000000000000000000048
:10784000416E01810000000044A401082001A20053
:10785000BC3F010800000000C43F01081000080000
:107860000000000000000000000000000000000018
:107870004D6E00810000000054A401083001A700F3
:10788000E43F0108DC3F01080C8401080800000007
:10789000A4480408000000000000000000000000F0
:1078A0004E6E03810000000064A4010800029800ED
:1078B000F43F0108E83F0108287E01081000040099
:1078C00000000000000000000000000000000000B8
:1078D0004D6E03810000000074A4010801009700B0
:1078E000A078000800000000000000000000000078
:1078F0004E6E01810000000084A401083001B30035
:10790000FC3F01080000000064400108080000007E
:10791000A4C00308000000000000000000000000F8
:10792000436E01810000000094A401083001AA0008
:1079300000400108000000000440010808000000A9
:10794000B8C00308000000000000000000000000B4
:10795000466E018100000000A4A401083001AC00C3
:107960002C400108204001083040010808000000B8
:10797000E4480408000000000000000000000000CF
:10798000496E018100000000B4A401080002AE00AD
:10799000B862010844400108287E01081000040074
:1079A00000000000000000000000000000000000D7
:1079B000486E018100000000C4A401080100AD0070
:1079C00080790008000000000000000000000000B6
:1079D0004C6E018100000000D4A401083001B10008
:1079E0005040010800000000644001080800000049
:1079F000CCC00308000000000000000000000000F0
:107A00004B6E018100000000E4A401082001B000D9
:107A10005C4001085440010864400108080000006F
:107A200010490408000000000000000000000000F1
:107A30004F6E018100000000F4A401083001B40081
:107A400060400108000000006440010808000000D8
:107A5000F4C0030800000000000000000000000067
:107A6000496E01810000000004A501083003DC001C
:107A7000D441010878400108E04101085C00280079
:107A800018C1030800000000000000000000000012
:107A9000416E00810000000014A501082001F700DC
:107AA0000C420108000000001042010814000C0004
:107AB00000000000000000000000000000000000C6
:107AC000486E00810000000024A501082001FB0091
:107AD00028420108000000002C42010808000000B4
:107AE0000000000000000000000000000000000096
:107AF0004B6E00810000000034A501082005FF0046
:107B00004043010838430108544301082C001C007D
:107B10000000000000000000000000000000000065
:107B2000446E01810000000044A5010830010701F6
:107B300080430108000000008443010808000000A1
:107B400068C1030800000000000000000000000001
:107B50004B6E01810000000054A5010830011001A6
:107B600098430108000000003C5C01080800000088
:107B70007CC10308000000000000000000000000BD
:107B80004A6E01810000000064A5010801000F0198
:107B90008CBD000800000000000000000000000094
:107BA000446E03810000000074A50108000220015A
:107BB000A84301089C430108287E01081400040022
:107BC00000000000000000000000000000000000B5
:107BD000436E03810000000084A5010801001F011D
:107BE000A07B000800000000000000000000000072
:107BF000486E03810000000094A5010820017F0168
:107C0000B043010800000000E87C01080800000003
:107C10000000000000000000000000000000000064
:107C2000456E008100000000A4A5010830019C0001
:107C3000B443010800000000B84301080800000038
:107C400090C10308000000000000000000000000D8
:107C50004C6E028100000000B4A501083003DE0173
:107C60001C520108EC430108285201083400180096
:107C700048C30308000000000000000000000000EE
:107C8000496E038100000000C4A5010801006B02D9
:107C9000A4BD00080000000000000000000000007B
:107CA0004E6E028100000000D4A50108300166027A
:107CB000FC430108F44301080044010808000000E7
:107CC000A84B0408000000000000000000000000B5
:107CD0004F6E018100000000E4A5010801005A0276
:107CE000C08000080000000000000000000000004C
:107CF0004B6E038100000000F4A5010820026C0215
:107D0000244401081C4401082C4401081000080008
:107D10000000000000000000000000000000000063
:107D20004D6E01810000000004A6010830015902D7
:107D300050440108484401085C4401080800000060
:107D40005C4C04080000000000000000000000007F
:107D50004B6E01810000000014A601083002580299
:107D600054440108000000005C44010808000000C1
:107D7000704C04080000000000000000000000003B
:107D8000486E01810000000024A601083001540261
:107D90007C44010874440108804401080800000084
:107DA000B84C0408000000000000000000000000C3
:107DB000476E01810000000044A601080100530243
:107DC000DCBE000800000000000000000000000011
:107DD000456E01810000000054A601080100520216
:107DE000BCBD000800000000000000000000000012
:107DF000446E01810000000064A6010820015102C8
:107E0000988001089C440108A4440108080000006F
:107E1000CC4C04080000000000000000000000003E
:107E20004E6E02810000000074A601083003DF01DD
:107E3000C4440108BC440108D04401081C001000DF
:107E4000F4C3030800000000000000000000000070
:107E50004B6E00810000000084A601083001F30190
:107E6000FC44010800000000044501080C00040067
:107E7000F04D0408000000000000000000000000B9
:107E8000406E02810000000094A601082003070252
:107E9000BC45010818450108C84501083000140018
:107EA00000000000000000000000000000000000D2
:107EB0004E6E028100000000A4A6010830020D02EF
:107EC0000C460108000000001446010808000000EC
:107ED00038C403080000000000000000000000009B
:107EE0004D6E028100000000B4A6010820010B02C3
:107EF00048460108404601084C46010808000000B9
:107F0000044E040800000000000000000000000013
:107F1000476E008100000000D4A6010830011B025A
:107F200068460108604601086C4601080800000028
:107F3000B84E04080000000000000000000000002F
:107F4000456E008100000000E4A601082802190225
:107F50000479010884460108D04601080C00040099
:107F6000CC4E0408000000000000000000000000EB
:107F7000466E008100000000F4A6010810021A02FB
:107F80008C7A0108044701085447010834001000A6
:107F9000501F040800000000000000000000000066
:107FA000416E02810000000004A701082001310297
:107FB000D847010800000000DC6901082800100013
:107FC00000000000000000000000000000000000B1
:107FD000416E00810000000014A701082001410249
:107FE000DC47010800000000E04701081000040021
:107FF0000000000000000000000000000000000081
:10800000436E00810000000024A701082001440203
:10801000F04701080000000020710108100008006E
:108020004CC4030800000000000000000000000035
:10803000466E00810000000034A7010810034602CC
:108040008484010838840108908401081000080025
:1080500030100408000000000000000000000000D4
:108060004A6E00810000000044A701083001490267
:10807000F447010800000000207101081400080006
:10808000A4C403080000000000000000000000007D
:10809000436E00810000000064A701083001BF01A9
:1080A000F847010800000000FC4701080800000034
:1080B00050C603080000000000000000000000009F
:1080C0004D6E02810000000074A7010820026502C5
:1080D0001448010800000000285801083000200062
:1080E0000000000000000000000000000000000090
:1080F0004C6E02810000000094A701086801800214
:108100001C48010800000000204801080800000089
:1081100060DA050800000000000000000000000018
:10812000496E018100000000A4A7010840012A0255
:108130005048010844480108544801080C00000058
:10814000000000000000000000000000000000002F
:10815000476E018100000000B4A70108400235010C
:108160009848010868480108A04801081000080064
:1081700000000000000000000000000000000000FF
:108180004A6E038100000000B4C00108300394006F
:10819000C448010800000000D04801081000000099
:1081A00020A2040800000000000000000000000001
:1081B000426E018100000000D4A7010840025F0167
:1081C000F8480108EC480108287E01081000040066
:1081D000000000000000000000000000000000009F
:1081E000476E028100000000E4A701087002E3006E
:1081F000BC580108AC5801086C770108280014002D
:1082000008C9040800000000000000000000000091
:10821000416E038100000000F4A7010840020F0234
:1082200030490108004901083849010810000800D8
:10823000000000000000000000000000000000003E
:108240004C6E028100000000A4C0010830027F00D3
:108250009073010854490108287A010810000400AD
:10826000A01605080000000000000000000000004B
:10827000456E02810000000004A8010870022F0072
:1082800060490108000000006C490108280018003E
:10829000A0740408000000000000000000000000BE
:1082A000486E01810000000014A801084002D101BD
:1082B0007C66010874660108C849010814000C00B6
:1082C00034D204080000000000000000000000009C
:1082D0004E6E02810000000024A801086005BF0066
:1082E000B06A0108E0840108F88401081C0010004D
:1082F000000000000000000000000000000000007E
:10830000416E01810000000034A801087005D90009
:10831000E04A0108E0840108F88401082000100008
:10832000ACFA04080000000000000000000000009B
:108330004A6E01810000000044A801084002D301F8
:10834000184A010874660108204A01081000080054
:108350004475050800000000000000000000000057
:108360004F6E00810000000054A801084002200266
:10837000E45A0108704A01087C4A01080C00000018
:1083800000000000000000000000000000000000ED
:108390004C6E03810000000064A8010870036B01AB
:1083A000087D0108E0840108F88401081C00100021
:1083B0008CED040800000000000000000000000038
:1083C000496E02810000000094A801087004D800E2
:1083D000E04A0108E0840108F88401082000100048
:1083E00008B40508000000000000000000000000C4
:1083F000496E018100000000C4C0010830024A003B
:10840000FC4A010800000000044B01080C000400B5
:10841000A8C70408000000000000000000000000E1
:10842000436E008100000000C4A801087002F9003A
:10843000284B0108204B0108304B010828001C0084
:10844000084F0508000000000000000000000000C8
:108450004E6E038100000000D4A801087001530192
:10846000E04B010800000000E44B01081400080084
:1084700094B60508000000000000000000000000A5
:10848000406E018100000000E4A80108680191022B
:10849000204C010800000000244C010808000000E6
:1084A000B0C8050800000000000000000000000047
:1084B0004C6E008100000000E4BC01083001100097
:1084C000404C0108384C01084C51010814000C00C4
:1084D00028790508000000000000000000000000EE
:1084E0004A6E01810000000014A901084100390111
:1084F00094C7000800000000000000000000000019
:10850000426E00810000000034A901087001890159
:108510004C4C010800000000047401080C00040029
:10852000EC670508000000000000000000000000EB
:10853000436E01810000000044A90108700361013D
:10854000AC7B0108E0840108F88401081C001000DD
:10855000F4EF04080000000000000000000000002C
:108560004B6E03810000000054A901085003510123
:1085700088580108504C01089C4C01082800100044
:1085800098710408000000000000000000000000D6
:108590004E6E03810000000064A901087001EF0025
:1085A000C46C0108BC6C0108F84C010828001000DC
:1085B000005F040800000000000000000000000050
:1085C000456E01810000000084A9010870019E0031
:1085D0008872010878720108044E0108140008002E
:1085E000146104080000000000000000000000000A
:1085F000446E008100000000D4A90108400145023A
:10860000C84E0108BC4E0108CC4E01080C00000009
:10861000000000000000000000000000000000005A
:108620004F6E02810000000004BD010870010300CC
:10863000A8790108E04E0108E84E01080C0004008A
:10864000BCDC040800000000000000000000000086
:10865000486E01810000000064BF0108300149003C
:108660000C4F0108044F0108104F010808000000DA
:108670002CA505080000000000000000000000001C
:108680004D6E02810000000004AA01084003BD00F5
:10869000F85F0108244F0108005901080C0004008C
:1086A00000000000000000000000000000000000CA
:1086B000466E018100000000C4BE01083001750053
:1086C0005C4F0108544F0108604F01081400080076
:1086D0001C740508000000000000000000000000FD
:1086E000416E00810000000044BE010841002B01E2
:1086F0000900000000000000000000000000000071
:108700004B6E02810000000014AA010870027F0273
:10871000F4750108744F0108904F0108100004001F
:10872000F80905080000000000000000000000003B
:10873000406E02810000000024AA01086003790253
:10874000345001081450010840500108140008007A
:108750000000000000000000000000000000000019
:108760004A6E02810000000034AA01087004DA0198
:10877000D4500108E0840108F88401081C001000AE
:10878000746F0408000000000000000000000000FA
:10879000476E03810000000044AA010841004D011A
:1087A00010A600080000000000000000000000000B
:1087B000466E01810000000054AA010870046501A2
:1087C0004C560108E4500108F88401081C00100010
:1087D00034690508000000000000000000000000EF
:1087E0004B6E03810000000084AA01087002C700DC
:1087F000445601083C560108B47301081C000000EF
:1088000024590508000000000000000000000000DE
:10881000466E008100000000D4BD01083002070050
:108820000051010800000000A07A010808000000C3
:10883000EC680508000000000000000000000000D7
:10884000476E038100000000B4BC010830019100B4
:1088500010510108085101081451010808000000D6
:10886000542E050800000000000000000000000079
:10887000416E038100000000B4AA01087001E1010B
:108880003C51010800000000AC5C01080800000039
:10889000EC78050800000000000000000000000067
:1088A000476E01810000000014BF01083001110073
:1088B00048510108405101084C51010808000000CE
:1088C000E4A6050800000000000000000000000011
:1088D000486E03810000000054BD0108300392007F
:1088E000F0520108000000006C5101081000000067
:1088F000B0A4050800000000000000000000000017
:108900004C6E03810000000004BF01083003960094
:108910008851010800000000945101081000000077
:10892000C0A50408000000000000000000000000D6
:108930004A6E038100000000F4AA01084002880288
:10894000BC510108B0510108C45101080C000000DD
:108950000000000000000000000000000000000017
:108960004B6E02810000000004AB01086801440165
:10897000F051010800000000F8790108080000002B
:1089800084D705080000000000000000000000007F
:10899000476E00810000000024AB0108600158010F
:1089A000FC510108F4510108005201080C000400B8
:1089B00000000000000000000000000000000000B7
:1089C000446E03810000000054AB01087003840270
:1089D0006C7F0108E0840108F88401081C00100085
:1089E000F8AB0408000000000000000000000000D8
:1089F000426E03810000000074AB01086001DC01DD
:108A00001C520108000000002852010818000C0048
:108A1000043605080000000000000000000000000F
:108A2000466E00810000000094AB01087001CF0089
:108A30005052010800000000545201080C000400CC
:108A40001CDC040800000000000000000000000022
:108A50004D6E028100000000B4AB010870023402C8
:108A600084520108785201088C5201080C0004005D
:108A700014DB0408000000000000000000000000FB
:108A8000436E00810000000044BD010830033B003C
:108A9000B06C010800000000B0520108240018006A
:108AA00090850508000000000000000000000000A4
:108AB000496E03810000000004AC0108400225015A
:108AC000E8520108DC520108287E01081400040065
:108AD0000000000000000000000000000000000096
:108AE000456E02810000000044AC0108700463017F
:108AF000DC590108E0840108F88401081C0010001A
:108B000084160508000000000000000000000000BE
:108B10004E6E02810000000064AC010860021F007C
:108B200060530108505301086C5301080C00040005
:108B30000000000000000000000000000000000035
:108B40004D6E02810000000074AC010860037701E3
:108B50003C540108A0530108485401080C000400CB
:108B60000000000000000000000000000000000005
:108B7000416E01810000000084AC010870044F02C6
:108B8000B4540108E0840108F88401081C001000B6
:108B90000072040800000000000000000000000057
:108BA000486E018100000000B4AC01084003760269
:108BB0005855010828550108005901080C00040007
:108BC00000000000000000000000000000000000A5
:108BD000426E038100000000C4AC010860027A010B
:108BE00074550108645501087C55010818000400FB
:108BF0000000000000000000000000000000000075
:108C0000416E028100000000F4AC010870046E01A6
:108C1000C8550108E0840108F88401081C00100010
:108C200024B4040800000000000000000000000060
:108C3000436E03810000000004C0010830012C00D5
:108C4000F4550108D8550108F8550108140008002A
:108C5000D4820408000000000000000000000000B2
:108C6000436E028100000000F4BE010841001501BE
:108C700004000000000000000000000000000000F0
:108C80004C6E01810000000014AD010840022D026D
:108C90002056010814560108287E0108100004001F
:108CA00000000000000000000000000000000000C4
:108CB0004F6E03810000000034AD010870012A01ED
:108CC00034560108000000009C75010808000000EF
:108CD000E0BB0508000000000000000000000000EC
:108CE000456E00810000000044AD010868018C0160
:108CF0003856010800000000047401080800000054
:108D000068220508000000000000000000000000CC
:108D1000426E00810000000054AD01087001C600E1
:108D2000445601083C560108B47301081C000000B9
:108D300088B10508000000000000000000000000ED
:108D4000416E01810000000074AD01087001C9018D
:108D50005C56010800000000605601080800000091
:108D6000E016050800000000000000000000000000
:108D7000416E008100000000E4C1010830020200E1
:108D80000C57010878560108145701081C001400FC
:108D9000C8A7040800000000000000000000000058
:108DA0004B6E028100000000A4AD01085002940146
:108DB0008C64010800000000505701081C001000DE
:108DC000AC000508000000000000000000000000EA
:108DD0004E6E038100000000D4AD01084002BD01C9
:108DE000A85701089C570108287E010810000400BC
:108DF0000000000000000000000000000000000073
:108E00004E6E018100000000E4AD010860027802AE
:108E1000D0570108B0570108D857010814000C00BA
:108E20000000000000000000000000000000000042
:108E30004C6E02810000000024C00108280163027A
:108E40002458010800000000285801081C000C00EC
:108E500038D60408000000000000000000000000F8
:108E60004C6E02810000000014AE01087001E200A7
:108E7000BC580108AC5801086C77010820000C00B0
:108E800074860508000000000000000000000000DB
:108E9000406E02810000000024AE01084003E000A3
:108EA000F4580108C4580108005901080C000400D6
:108EB00000000000000000000000000000000000B2
:108EC000446E01810000000034AE010870043401DA
:108ED00018590108E0840108F88401081C001000FA
:108EE000ACBF04080000000000000000000000000B
:108EF000466E02810000000044AE01084100BB0044
:108F0000DCC40008000000000000000000000000B9
:108F1000426E03810000000054AE01087001390068
:108F200028590108000000003059010828001000ED
:108F3000D02B050800000000000000000000000029
:108F4000456E01810000000074AE010870056401E7
:108F5000DC590108E0840108F88401081C001000B5
:108F6000D4590408000000000000000000000000C8
:108F70004C6E01810000000084AE01087004D50031
:108F8000F0590108E0840108F88401081C00100071
:108F9000D8420508000000000000000000000000AA
:108FA0004B6E008100000000A4AE010840025A018F
:108FB000BC6B0108145A01085C5A01081000080033
:108FC00000000000000000000000000000000000A1
:108FD000426E028100000000F4BC010830018100F3
:108FE0008C5A0108845A0108287A010808000000F8
:108FF000A8060508000000000000000000000000B6
:109000004D6E018100000000E4AE01084100040241
:10901000F4C4000800000000000000000000000090
:10902000466E03810000000004AF0108680185025C
:10903000905A010800000000945A0108080000003E
:10904000CC16050800000000000000000000000031
:109050004E6E03810000000014AF01087004C900C7
:10906000A85A0108E0840108F88401081C001000D7
:10907000A8640408000000000000000000000000D8
:109080004F6E02810000000024AF010840021C0165
:10909000C45A0108B85A0108287E010814000400C7
:1090A00000000000000000000000000000000000C0
:1090B000436E00810000000034AF010870047102AB
:1090C000CC5A0108E0840108F88401081C00100053
:1090D000FC6E04080000000000000000000000001A
:1090E0004D6E03810000000054AF01084100BC0137
:1090F000D08D00080000000000000000000000000B
:109100004A6E01810000000074AF0108680100028E
:10911000EC5A010800000000F05A010808000000A5
:10912000504D050800000000000000000000000095
:10913000476E02810000000084AF01084001D801A1
:10914000085B0108000000000C5B01081C00140013
:10915000000000000000000000000000000000000F
:109160004E6E03810000000094AF010850034702D7
:10917000685B01081C5B0108785B010824000C0097
:1091800064CF05080000000000000000000000009F
:109190004B6E038100000000A4AF01087001EA01DA
:1091A000D45B010800000000D85B01080800000043
:1091B000C865040800000000000000000000000076
:1091C0004F6E01810000000044BF010830011B0008
:1091D000F45B0108EC5B01085C6F010818000C00EF
:1091E0003CAB05080000000000000000000000008B
:1091F000466E028100000000B4AF010870042C012B
:10920000F85B0108E0840108F88401081C001000E4
:1092100094D60408000000000000000000000000D8
:10922000476E028100000000E4AF01087004720183
:109230000C5C0108E0840108F88401081C0010009F
:1092400054A7050800000000000000000000000016
:10925000426E028100000000F4AF010870030B00B1
:109260001C5C0108E0840108F88401081C0010005F
:109270002468050800000000000000000000000055
:10928000426E00810000000004B001087004CB00B1
:10929000B45F0108E0840108F88401081C00100094
:1092A000908F050800000000000000000000000092
:1092B000456E03810000000024B0010870026001C7
:1092C0006C7F0108E0840108F88401081C0010008C
:1092D00040CA040800000000000000000000000078
:1092E000446E02810000000094BE01084100160196
:1092F0000B00000000000000000000000000000063
:109300004D6E00810000000034B0010841005C0196
:1093100000980008000000000000000000000000AD
:109320004E6E02810000000064B0010841001B0184
:109330008090000800000000000000000000000015
:109340004D6E01810000000074B001086801120137
:10935000385C0108000000003C5C010808000000C7
:109360008CE0040800000000000000000000000085
:10937000446E00810000000084B0010870018B0180
:10938000505C01080000000004740108080000009F
:109390002CAF0508000000000000000000000000E5
:1093A0004E6E01810000000094B0010860021301BC
:1093B000545C0108000000005C5C01082000100003
:1093C000000000000000000000000000000000009D
:1093D000406E038100000000A4B001087001E001AC
:1093E000A85C010800000000AC5C01080C00000053
:1093F000A8E80408000000000000000000000000D1
:10940000426E028100000000B4B0010870057001D6
:10941000C45C0108E0840108F88401081C00100005
:10942000A8D70408000000000000000000000000B1
:109430004D6E018100000000D4BF010830017A00A8
:10944000F85C0108F05C0108A8760108080000003B
:10945000C0570408000000000000000000000000E9
:109460004B6E008100000000D4B001087001900133
:10947000FC5C010800000000005D0108080000001D
:1094800044DC0508000000000000000000000000AF
:109490004E6E038100000000E4B0010870020A0073
:1094A000185D0108E0840108F88401081C00100020
:1094B000F0B00508000000000000000000000000FF
:1094C000446E008100000000F4B001084100FA0081
:1094D00064C400080000000000000000000000005C
:1094E000446E03810000000014B1010860017C019A
:1094F0002C5D0108245D0108305D01080C000400AA
:10950000000000000000000000000000000000005B
:109510004D6E018100000000F4BD01083003180009
:10952000A46501088C650108B065010818001000E9
:1095300000D9040800000000000000000000000046
:109540004F6E01810000000034BD010830017C0035
:10955000585D0108505D0108A87601080800000068
:109560002CB3040800000000000000000000000010
:10957000416E03810000000044B101086001C00099
:10958000705D01080000000030650108100008004F
:1095900000000000000000000000000000000000CB
:1095A0004B6E028100000000F4C101087001DB0174
:1095B0007C5D0108745D0108805D010814000800ED
:1095C00078260508000000000000000000000000F0
:1095D000406E01810000000054B101084002F80112
:1095E000F05D0108C05D0108F85D01081000080089
:1095F000000000000000000000000000000000006B
:109600004D6E03810000000064B10108680114027E
:10961000145E010800000000185E01080800000048
:10962000EC830408000000000000000000000000BF
:109630004F6E03810000000084B101085005550100
:1096400014700108BC6F010828700108180004009C
:1096500060CD0508000000000000000000000000D0
:10966000466E03810000000094B101086001C10052
:109670002C5E0108000000003065010810000800A1
:1096800000000000000000000000000000000000DA
:10969000496E02810000000054BE0108300226001D
:1096A000C85E0108305E0108D05E01082000180085
:1096B000B0380508000000000000000000000000B5
:1096C000426E028100000000A4B101086003300076
:1096D000045F010800000000185F010868001C001A
:1096E000000000000000000000000000000000007A
:1096F000416E008100000000C4B101087005CC007B
:10970000B45F0108E0840108F88401081C0010001F
:1097100094060508000000000000000000000000A2
:109720004F6E038100000000E4B101084100BE015A
:109730001CC1000800000000000000000000000044
:10974000476E038100000000A4BD010841002E0007
:109750000600000000000000000000000000000003
:10976000456E008100000000F4B1010841008B0249
:10977000E0AF000800000000000000000000000052
:10978000426E01810000000004B2010870046F0104
:10979000EC730108E0840108F88401081C00100043
:1097A000D4B6040800000000000000000000000023
:1097B000406E03810000000014B2010841000E0257
:1097C000108F0008000000000000000000000000F2
:1097D0004A6E02810000000034B2010870013302B9
:1097E0001060010804600108146001080C00040006
:1097F000ACA9050800000000000000000000000007
:109800004E6E00810000000064B2010840025D015C
:10981000486001083C600108287E0108100004002F
:109820000000000000000000000000000000000038
:109830004C6E03810000000084B201087004C8006F
:1098400058600108E0840108F88401081C00100039
:109850008006050800000000000000000000000075
:10986000416E03810000000094B20108700279018A
:109870007860010868600108806001081000040039
:10988000BC7404080000000000000000000000009C
:109890004B6E008100000000B4B2010850011C02B0
:1098A0000C610108BC600108106101081000000093
:1098B0008CC9050800000000000000000000000046
:1098C000416E028100000000E4B2010860013D0128
:1098D00038610108000000003C61010818000C001C
:1098E0000000000000000000000000000000000078
:1098F000496E028100000000F4B2010870057D028B
:10990000D4810108E0840108F88401081C001000DB
:10991000A062040800000000000000000000000039
:10992000416E03810000000004B3010868013702A2
:1099300050610108000000002071010808000000CB
:10994000D0A1050800000000000000000000000099
:109950004D6E03810000000024B3010868018301FB
:109960005461010800000000D47A010808000000DA
:10997000F065040800000000000000000000000086
:109980004F6E03810000000054B3010870046D02A3
:10999000C8620108C0620108F88401081C001000B8
:1099A000EC8404080000000000000000000000003B
:1099B000416E02810000000074B30108600275016D
:1099C000B8670108D8620108E86201080C000400C9
:1099D0000000000000000000000000000000000087
:1099E000476E02810000000084B301087001180175
:1099F000C06301080C630108C4630108080000008B
:109A0000BC5304080000000000000000000000003B
:109A10004E6E038100000000A4B30108400229013A
:109A20003064010824640108287E01081000040045
:109A30000000000000000000000000000000000026
:109A4000476E018100000000C4B3010841006601B7
:109A500020AF00080000000000000000000000002F
:109A6000406E028100000000D4B3010840023002C1
:109A700044640108386401084C64010810000000C7
:109A800000000000000000000000000000000000D6
:109A9000406E038100000000E4B30108700236024A
:109AA0008464010878640108207101080C00040036
:109AB00070720508000000000000000000000000B7
:109AC000406E03810000000004B4010860027801C8
:109AD000BC6E010898640108F464010820001000BD
:109AE0000000000000000000000000000000000076
:109AF000496E02810000000014B401086001BC003E
:109B00002C65010800000000306501081000080005
:109B10000000000000000000000000000000000045
:109B2000416E01810000000034B4010870014C0254
:109B30006865010800000000746501080800000065
:109B4000006905080000000000000000000000009F
:109B5000466E03810000000044B401087002170043
:109B6000A46501088C650108B065010818001000A3
:109B70001CA5040800000000000000000000000018
:109B8000466E02810000000054B40108680117010C
:109B9000E465010800000000E86501080800000015
:109BA0003433050800000000000000000000000041
:109BB000466E00810000000064B4010868018D0158
:109BC000706601080000000004740108080000002D
:109BD00010B40408000000000000000000000000B5
:109BE000466E02810000000074B401084001D001FB
:109BF0007C6601087466010884660108100008008C
:109C0000885604080000000000000000000000006A
:109C10004F6E038100000000C4BC010830039900AE
:109C2000F066010800000000FC660108100000005A
:109C3000786A050800000000000000000000000035
:109C40004B6E028100000000B4B40108600376018D
:109C5000B867010818670108C4670108100004000C
:109C600000000000000000000000000000000000F4
:109C7000436E018100000000C4B401084002DB0013
:109C800040680108106801084868010828001800A9
:109C900000000000000000000000000000000000C4
:109CA000426E008100000000D4B401085002EF01B0
:109CB0009068010860680108986801080C000400B9
:109CC00070520408000000000000000000000000C6
:109CD000406E028100000000E4B4010870046D01D0
:109CE000B0680108E0840108F88401081C00100035
:109CF0002CDF04080000000000000000000000004D
:109D0000466E038100000000E4C0010841002D0000
:109D1000070000000000000000000000000000003C
:109D2000496E03810000000084BD010830039300E8
:109D3000C868010800000000D46801081000000095
:109D4000B4AC0408000000000000000000000000A7
:109D5000416E02810000000014B501087002340059
:109D6000F068010800000000FC6801081800080005
:109D7000449A0508000000000000000000000000F8
:109D80004C6E00810000000024B5010848010A0162
:109D90004069010800000000486901081000000047
:109DA0008CDF05080000000000000000000000003B
:109DB000446E01810000000034B501084002250214
:109DC0007C690108706901088469010810000000BD
:109DD0000000000000000000000000000000000083
:109DE0004F6E02810000000044B5010870011900A7
:109DF000546F0108486F01085C6F010810000800EB
:109E0000F84D050800000000000000000000000000
:109E10004D6E01810000000054B5010840016A0147
:109E2000C0690108B8690108C46901080C00040090
:109E300034A605080000000000000000000000003B
:109E40004D6E01810000000064B5010868012E021A
:109E5000D869010800000000DC6901080800000062
:109E60008CA70508000000000000000000000000B2
:109E70004F6E03810000000074B501085003870194
:109E8000406A0108F46901084C6A010810000800E2
:109E9000F07704080000000000000000000000004F
:109EA0004C6E01810000000054BF010830017900B0
:109EB000AC6A0108A46A0108A8760108080000003D
:109EC000608605080000000000000000000000009F
:109ED0004F6E028100000000A4B501086004BE00BE
:109EE000B06A0108E0840108F88401081C00100031
:109EF0000000000000000000000000000000000062
:109F0000486E028100000000B4B5010870047301BE
:109F1000C46A0108E0840108F88401081C001000EC
:109F2000B85005080000000000000000000000001C
:109F3000466E038100000000C4B5010850022201F2
:109F4000046B0108D46A01080C6B01080C000400C2
:109F5000A47E0408000000000000000000000000D3
:109F60004B6E038100000000D4B5010840022601B9
:109F7000546B0108246B01085C6B01081000080099
:109F800000000000000000000000000000000000D1
:109F90004A6E008100000000E4B5010840035B0147
:109FA000BC6B0108746B0108C86B01081000080045
:109FB00000000000000000000000000000000000A1
:109FC000446E008100000000F4B501084001F10179
:109FD000F06B010800000000F46B01082000040091
:109FE00004740508000000000000000000000000EC
:109FF000456E03810000000004B6010870011102E3
:10A000005C6C010800000000606C010808000000A2
:10A0100090DD0508000000000000000000000000C6
:10A02000476E03810000000024B601087002F000B2
:10A03000C46C0108BC6C0108CC6C0108280010003D
:10A04000DC23050800000000000000000000000004
:10A05000466E01810000000034B601087001FC0169
:10A06000B86D010800000000BC6D01080800000088
:10A07000C0590408000000000000000000000000BB
:10A08000436E02810000000094C101083002B80054
:10A09000DC6D010800000000E46D01081000040000
:10A0A00090E704080000000000000000000000002D
:10A0B0004A6E01810000000064B6010840035602A8
:10A0C000346E0108046E0108406E0108100004009F
:10A0D0000000000000000000000000000000000080
:10A0E000436E01810000000094B601084002330174
:10A0F000F46E0108C46E0108FC6E01080C00040037
:10A10000000000000000000000000000000000004F
:10A11000466E028100000000A4B6010870047101BF
:10A12000146F0108E0840108F88401081C00100085
:10A1300094940508000000000000000000000000EA
:10A140004B6E01810000000084C1010830017800DD
:10A150002C6F0108246F0108A87601080800000090
:10A16000980F05080000000000000000000000003B
:10A17000436E008100000000B4B6010870048A013B
:10A18000386F0108306F0108F88401081C001000C6
:10A1900094640408000000000000000000000000BB
:10A1A0004E6E01810000000034C0010830021A0028
:10A1B000546F0108486F01085C6F01081000080027
:10A1C000D46B040800000000000000000000000044
:10A1D000476E02810000000094BF01083001860034
:10A1E000886F0108806F0108287A010808000000C4
:10A1F00084DE0508000000000000000000000000F0
:10A200004B6E038100000000D4B601086004810198
:10A210008C6F0108E0840108F88401081C0010001C
:10A22000000000000000000000000000000000002E
:10A230004E6E018100000000E4B601087005DE00EA
:10A240009C6F0108E0840108F88401081C001000DC
:10A2500080AF0508000000000000000000000000C2
:10A26000416E00810000000004B701085004540151
:10A2700014700108BC6F0108287001081800040060
:10A28000908B0508000000000000000000000000A6
:10A290004E6E02810000000034C101083001290027
:10A2A000F8700108F0700108FC7001080800000057
:10A2B000B07305080000000000000000000000006E
:10A2C000436E03810000000024B7010868013802D2
:10A2D0001C71010800000000207101080800000046
:10A2E000D8D80408000000000000000000000000B2
:10A2F0004D6E02810000000034B7010870021A019F
:10A3000044710108000000004C71010824000000A5
:10A3100040EE040800000000000000000000000003
:10A32000456E018100000000B4BF01083002AB009F
:10A33000B071010800000000B87101080C000400B1
:10A34000909C0508000000000000000000000000D4
:10A350004E6E02810000000044B701087005E7005E
:10A36000E8710108E0840108F88401081C0010006D
:10A3700050840408000000000000000000000000FD
:10A38000426E00810000000064B701087004700292
:10A39000FC710108E0840108F88401081C00100029
:10A3A000B0AD040800000000000000000000000044
:10A3B0004C6E01810000000074B70108680169015A
:10A3C0000C72010800000000107201080800000073
:10A3D000F89E0408000000000000000000000000DB
:10A3E000436E00810000000094B701087004CD00A6
:10A3F00038720108E0840108F88401081C0010008C
:10A400008881040800000000000000000000000037
:10A410004E6E028100000000A4B7010870013502F1
:10A420005472010848720108587201080C000400B7
:10A43000DC560408000000000000000000000000DE
:10A440004B6E038100000000C4B701087003BA011D
:10A4500094720108E0840108F88401081C001000CF
:10A4600088670408000000000000000000000000F1
:10A470004F6E038100000000D4B7010870028A0209
:10A48000BC720108A0720108C47201081000040027
:10A49000A4DD05080000000000000000000000002E
:10A4A000476E018100000000E4B701084002280265
:10A4B00054730108487301085C7301080C00000024
:10A4C000000000000000000000000000000000008C
:10A4D0004B6E018100000000F4B7010841002C021E
:10A4E000808C000800000000000000000000000058
:10A4F000416E03810000000024BD010830017E0090
:10A5000090730108887301089C730108100004000F
:10A5100074DE0408000000000000000000000000DD
:10A520004F6E03810000000004B801086001CA00FA
:10A53000B073010800000000B473010814000800A3
:10A54000000000000000000000000000000000000B
:10A55000476E03810000000014B8010870057E01F9
:10A56000EC730108E0840108F88401081C00100065
:10A5700040CB0408000000000000000000000000C4
:10A58000416E00810000000034B8010870018801AC
:10A5900000740108000000000474010814000C009D
:10A5A000105F05080000000000000000000000002F
:10A5B000406E02810000000044B8010860021401EE
:10A5C00020740108000000002C7401083000100005
:10A5D000000000000000000000000000000000007B
:10A5E000406E03810000000054B801085004670267
:10A5F000EC74010894740108FC740108180004004C
:10A6000038B4040800000000000000000000000052
:10A610004A6E01810000000064B801084001680131
:10A62000847501087C750108887501081000000018
:10A630000C7C040800000000000000000000000086
:10A64000456E03810000000074B80108700121010B
:10A6500098750108000000009C75010818000800AA
:10A66000B0890508000000000000000000000000A4
:10A67000436E03810000000094B8010870057B015F
:10A68000FC750108E0840108F88401081C00100032
:10A690002C2E050800000000000000000000000053
:10A6A0004C6E028100000000A4B80108700219017C
:10A6B0001076010800000000187601082000000054
:10A6C00010C30508000000000000000000000000AA
:10A6D000416E028100000000B4B801084001E100B1
:10A6E0007C76010800000000807601081400080054
:10A6F000000000000000000000000000000000005A
:10A70000496E018100000000C4BD010830017700DE
:10A71000A47601089C760108A876010808000000CC
:10A72000603C050800000000000000000000000080
:10A73000466E018100000000D4B801087003CE010C
:10A74000BC760108E0840108F88401081C001000B0
:10A750004036050800000000000000000000000076
:10A760004F6E018100000000E4B801087005DF00B1
:10A77000C8760108E0840108F88401081C00100074
:10A7800028AB0508000000000000000000000000E9
:10A79000456E02810000000004B901084100BA00C2
:10A7A00064C100080000000000000000000000007C
:10A7B000486E03810000000014B9010870043B02D8
:10A7C000E4760108E0840108F88401081C00100008
:10A7D000806E04080000000000000000000000007F
:10A7E000406E03810000000034B9010870021D01B1
:10A7F000F476010800000000FC7601081C0004004B
:10A8000010A7040800000000000000000000000085
:10A81000476E00810000000044B901084001D000EB
:10A820005477010800000000587701081400040064
:10A830000000000000000000000000000000000018
:10A840004D6E02810000000054B901086001E6006D
:10A8500068770108000000006C77010820000800FC
:10A8600000000000000000000000000000000000E8
:10A870004D6E03810000000064B901084100280109
:10A88000109A000800000000000000000000000016
:10A89000496E03810000000094B901084100800165
:10A8A0009CBF000800000000000000000000000045
:10A8B000456E02810000000054C1010830035500BC
:10A8C0006C780108647801087878010808000000B5
:10A8D000009B0508000000000000000000000000D0
:10A8E0004C6E008100000000F4BF010830016C00D4
:10A8F00098780108907801089C78010828001800D1
:10A90000749A04080000000000000000000000002D
:10A91000436E00810000000004BE01083002040004
:10A92000A87901080C790108B07901081C0014000D
:10A9300004D2040800000000000000000000000035
:10A94000446E018100000000F4B901087004CC01DC
:10A95000D0790108E0840108F88401081C00100087
:10A96000187A050800000000000000000000000048
:10A970004C6E02810000000004BA01087005AD01B0
:10A98000E0790108E0840108F88401081C00100047
:10A9900040710408000000000000000000000000FA
:10A9A0004E6E01810000000014BA01084100D4017C
:10A9B000E09B000800000000000000000000000014
:10A9C0004E6E02810000000024BA010868014501B2
:10A9D000F479010800000000F8790108080000007F
:10A9E000D8B50508000000000000000000000000CD
:10A9F0004A6E02810000000064C001083001890035
:10AA0000247A01081C7A0108287A0108080000004D
:10AA10003C69040800000000000000000000000085
:10AA2000456E00810000000064BD01083001060091
:10AA30009C7A0108947A0108A07A010808000000B5
:10AA4000C4B5050800000000000000000000000080
:10AA5000446E00810000000044BA01087003C20087
:10AA6000947C0108E0840108F88401081C001000AF
:10AA700018B1050800000000000000000000000000
:10AA80004C6E03810000000054BA0108600282018C
:10AA9000CC7A0108C07A0108D47A010814000C00AD
:10AAA00000000000000000000000000000000000A6
:10AAB0004D6E03810000000064BA01084100EC0102
:10AAC000C09F00080000000000000000000000001F
:10AAD0004A6E00810000000014C001083003C40168
:10AAE000F87A010800000000047B01081800080043
:10AAF000EC5E040800000000000000000000000000
:10AB0000456E00810000000074BA01087001570111
:10AB10004C7B010800000000507B01081400040079
:10AB20009C67040800000000000000000000000016
:10AB3000476E03810000000084BA010870042301FD
:10AB4000847B0108E0840108F88401081C001000DF
:10AB500000C905080000000000000000000000001F
:10AB6000496E03810000000094BA01087005C50019
:10AB7000947C0108E0840108F88401081C0010009E
:10AB800048D304080000000000000000000000009E
:10AB9000446E018100000000B4BA01087004620133
:10ABA000AC7B0108E0840108F88401081C00100057
:10ABB0002C7A0508000000000000000000000000E2
:10ABC000486E028100000000C4BA0108400108017B
:10ABD000BC7B010800000000C47B010850000C0091
:10ABE000E0A70508000000000000000000000000D1
:10ABF000426E008100000000D4BA01086001F80034
:10AC0000F87B0108F07B0108FC7B01080C000400C4
:10AC10000000000000000000000000000000000034
:10AC2000496E03810000000094C001083004E8016F
:10AC3000107C0108E0840108F88401081C00100061
:10AC4000583405080000000000000000000000006B
:10AC50004F6E028100000000E4BA01087005E800B0
:10AC6000207C0108E0840108F88401081C00100021
:10AC700088BD040800000000000000000000000083
:10AC80004C6E00810000000004BB01084002750208
:10AC9000407C0108347C0108487C01080C0000005D
:10ACA00000000000000000000000000000000000A4
:10ACB000496E00810000000024BB010870045901A6
:10ACC000847C0108E0840108F88401081C0010005D
:10ACD000D83505080000000000000000000000005A
:10ACE0004A6E03810000000034BB01087004C400F8
:10ACF000947C0108E0840108F88401081C0010001D
:10AD00008C26050800000000000000000000000084
:10AD10004B6E01810000000074BF01083002160074
:10AD2000B07C0108A87C0108B87C01080C00040074
:10AD3000C8F6040800000000000000000000000049
:10AD4000486E03810000000054BB0108410024014B
:10AD5000B08A0008000000000000000000000000B1
:10AD6000456E03810000000094BB010870017D0165
:10AD7000E47C0108DC7C0108E87C01080800000094
:10AD80001033050800000000000000000000000073
:10AD90004F6E018100000000A4BB010870046C012B
:10ADA000087D0108E0840108F88401081C001000F7
:10ADB000C4C80408000000000000000000000000FB
:10ADC000486E038100000000B4BB01084100F1009F
:10ADD0009085000800000000000000000000000056
:10ADE000476E038100000000C4BB01087004C3006B
:10ADF000187D0108E0840108F88401081C00100097
:10AE00005C290508000000000000000000000000B0
:10AE1000406E028100000000E4BD01083002B50070
:10AE2000287D010800000000307D010808000000B6
:10AE3000B42C050800000000000000000000000025
:10AE4000416E018100000000E4BB010841005E0189
:10AE5000B0810008000000000000000000000000B9
:10AE60004B6E03810000000054C0010830039500C0
:10AE7000447D010800000000507D01081000000022
:10AE8000041305080000000000000000000000009E
:10AE9000426E018100000000F4BB0108680132012C
:10AEA0006C7D010800000000707D010808000000B2
:10AEB00048450508000000000000000000000000F8
:10AEC0004A6E02810000000004BC01084002E50057
:10AED0008C7D0108847D0108947D01080C0004002C
:10AEE0000000000000000000000000000000000062
:10AEF0004D6E01810000000014BC01087001DD00EE
:10AF0000B47D0108A47D0108B87D01081400080083
:10AF1000AC71040800000000000000000000000008
:10AF2000486E01810000000024BC01084002670156
:10AF3000207E0108147E0108287E0108100004000C
:10AF40000000000000000000000000000000000001
:10AF5000416E03810000000034BC010870021E0134
:10AF60003C7E010800000000447E0108180000003B
:10AF7000CC490508000000000000000000000000AF
:10AF80004D6E02810000000074BC01087004AE0127
:10AF9000187F0108E0840108287F01081C001000C8
:10AFA00098210508000000000000000000000000DB
:10AFB0004D6E03810000000084BC010870035E0038
:10AFC0005C7F0108E0840108F88401081C0010007F
:10AFD000746305080000000000000000000000008D
:10AFE000466E00810000000094BC01087001090059
:10AFF0006C7F0108E0840108F88401081C0010003F
:10B000009092040800000000000000000000000012
:10B010004B6E008100000000A4BC010830034A020E
:10B02000D87F010800000000E47F0108180010002C
:10B03000E8420408000000000000000000000000DA
:10B04000456E01810000000014C20108700000007C
:10B0500098800108000000009C80010808000000A2
:10B06000CCE1050800000000000000000000000026
:10B070004D6E02810000000024C2010868018102B7
:10B08000E4800108C4800108E8800108080000008D
:10B09000D4E10508000000000000000000000000EE
:10B0A0004C6E00810000000034C201085001900283
:10B0B00008810108F88001080C81010818000400CB
:10B0C000E8E10508000000000000000000000000AA
:10B0D0004F6E02810000000044C201082002AF014F
:10B0E000348101082C8101083C81010820000C00FA
:10B0F00004E205080000000000000000000000005D
:10B10000436E00810000000054C2010870010D016F
:10B11000748101086C8101087C81010820000C0009
:10B1200018E2050800000000000000000000000018
:10B13000406E02810000000064C2010870045B02DE
:10B14000B4810108AC810108F88401081C001000DA
:10B150003CE20508000000000000000000000000C4
:10B16000496E01810000000074C20108700455029C
:10B17000C4810108E0840108F88401081C00100063
:10B1800050E2050800000000000000000000000080
:10B19000476E03810000000084C2010870047C0235
:10B1A000D4810108E0840108F88401081C00100023
:10B1B00064E205080000000000000000000000003C
:10B1C0004A6E02810000000094C2010870057E02F0
:10B1D000E8810108E0840108F88401081C001000DF
:10B1E00078E20508000000000000000000000000F8
:10B1F0004C6E038100000000A4C2010870048902A3
:10B20000FC810108E0840108F88401081C0010009A
:10B210008CE20508000000000000000000000000B3
:10B22000476E038100000000B4C201087004B6013B
:10B230000C820108E0840108F88401081C00100059
:10B24000A0E205080000000000000000000000006F
:10B250004B6E038100000000C4C2010870043E026E
:10B260001C820108E0840108F88401081C00100019
:10B27000B4E205080000000000000000000000002B
:10B28000416E018100000000D4C201087005F9017F
:10B290002C820108E0840108F88401081C001000D9
:10B2A000C8E20508000000000000000000000000E7
:10B2B000476E018100000000E4C201087004E30150
:10B2C00060820108E0840108F88401081C00100075
:10B2D000DCE20508000000000000000000000000A3
:10B2E0004A6E038100000000F4C2010870043D02B0
:10B2F00040820108E0840108F88401081C00100065
:10B30000F0E205080000000000000000000000005E
:10B31000466E03810000000004C301087004B501FB
:10B3200050820108E0840108F88401081C00100024
:10B3300004E3050800000000000000000000000019
:10B34000446E03810000000014C301087005E4018D
:10B3500060820108E0840108F88401081C001000E4
:10B3600018E30508000000000000000000000000D5
:10B37000486E03810000000024C301087003E70148
:10B3800074820108E0840108F88401081C001000A0
:10B390002CE3050800000000000000000000000091
:10B3A000456E03810000000034C301087004B4013D
:10B3B00080820108E0840108F88401081C00100064
:10B3C00040E305080000000000000000000000004D
:10B3D0004F6E01810000000044C3010870052F0278
:10B3E00090820108E0840108F88401081C00100024
:10B3F00054E3050800000000000000000000000009
:10B40000436E01810000000054C301087004500223
:10B41000A4820108E0840108F88401081C001000DF
:10B4200068E30508000000000000000000000000C4
:10B43000446E02810000000064C3010841005E0206
:10B4400008000000000000000000000000000000F4
:10B45000436E02810000000074C3010841005D02D8
:10B460000A000000000000000000000000000000D2
:10B470004B6E00810000000084C3010841008F0270
:10B4800005000000000000000000000000000000B7
:10B49000496E03810000000094C301084100B80117
:10B4A00070B4000800000000000000000000000070
:10B4B000486E008100000000A4C3010841008D0215
:10B4C000A0B0000800000000000000000000000024
:10B4D000486E038100000000B4C301084100B701B9
:10B4E00000B10008000000000000000000000000A3
:10B4F000426E038100000000C4C3010841006902DC
:10B5000040B0000800000000000000000000000043
:10B51000426E038100000000D4C301083002B10173
:10B52000C4820108B4820108CC820108080000002E
:10B5300090E405080000000000000000000000008A
:10B54000416E038100000000E4C301082002B00145
:10B5500000830108F0820108088301081800000038
:10B5600000000000000000000000000000000000DB
:10B57000496E038100000000F4C3010870043C021E
:10B580003C830108E08401084C8301081C00100082
:10B59000A4E4050800000000000000000000000016
:10B5A000476E02810000000004C4010820047B02F1
:10B5B0008883010880830108F88401081C001000BA
:10B5C000000000000000000000000000000000007B
:10B5D000446E03810000000014C401087004B3012C
:10B5E00098830108E0840108F88401081C00100019
:10B5F000B8E40508000000000000000000000000A2
:10B60000436E03810000000024C401087004B201ED
:10B61000B0830108A8830108C08301081C00100042
:10B62000CCE405080000000000000000000000005D
:10B63000496E02810000000034C401086002A500C8
:10B64000F0830108000000000C8401081C001000B9
:10B6500000000000000000000000000000000000EA
:10B66000406E03810000000044C4010860038401AF
:10B67000FC830108000000000C8401081C0010007D
:10B6800000000000000000000000000000000000BA
:10B69000486E00810000000054C401085002860179
:10B6A0008484010838840108908401080C00040097
:10B6B0002007060800000000000000000000000055
:10B6C0004A6E02810000000064C401087004740125
:10B6D000E8840108E0840108F88401081C001000D7
:10B6E0003C0706084A6E018100000000848C0108B6
:10B6F00024020000A8D4000818CE00084F6E008174
:10B7000000000000948C010824010000FCD3000814
:10B7100000D00008496E008100000000A48C0108E0
:10B720003401000084D4000828D000084F6E008146
:10B7300000000000B48C01082402000044D7000877
:10B7400040D000084E6E008100000000C48C01084B
:10B750002403000044D7000850D000084B6E00813D
:10B7600000000000D48C010824020000A0D80008CA
:10B770005CD100084A6E008100000000E48C0108E2
:10B7800024030000A0D800086CD100084D6E018190
:10B7900000000000C48D0108060000000000000049
:10B7A00000000000436E008100000000048E0108CC
:10B7B0000600000000000000000000004E6E008146
:10B7C00000000000148E010806010000ACD500083E
:10B7D000000000004E6E018100000000848E010810
:10B7E000060001000000000000000000406E028121
:10B7F00000000000C48E01080600000000000000E8
:10B8000000000000446E008100000000148F010859
:10B8100046002B000000000000000000426E008186
:10B8200000000000248F010846002C0000000000EA
:10B8300000000000426E018100000000848F0108BA
:10B8400024010000A0F2000868DE0008426E0181B9
:10B8500000000000948F01080600000000000000B6
:10B8600000000000476E028100000000B48F010854
:10B870003401000034E900089CDE0008476E0181B5
:10B8800000000000E4910108060000000000000034
:10B8900000000000446E03810000000034920108A3
:10B8A0000602020070E7000800000000486E0181F7
:10B8B0000000000044920108060100007CE7000837
:10B8C000000000004E6E008100000000549201084C
:10B8D0000602020084E70008000000004A6E0281B0
:10B8E0000000000094920108060001000000000022
:10B8F00000000000486E028100000000A4920108D0
:10B9000004020000A0FD000898FD0008436E0381BA
:10B9100000000000B49201080600040000000000CE
:10B92000000000004E6E008100000000D49201086B
:10B9300024030000A802010800000000426E0381F9
:10B9400000000000849301080602000000EC0008DB
:10B9500000000000416E0381000000009493010884
:10B96000060301000CEC0008000000004A6E028192
:10B9700000000000B4930108060000000000000071
:10B9800000000000456E028100000000D493010811
:10B99000340100004C0C010800000000436E0281DD
:10B9A00000000000E4930108240100005C0C010881
:10B9B00068EC0008456E018100000000F493010866
:10B9C00034010000DC0C010898EC0008476E00818F
:10B9D00000000000249401080600000000000000A0
:10B9E000000000004D6E0381000000003494010847
:10B9F0000600010000000000000000004C6E038102
:10BA0000000000004494010806000200000000004D
:10BA1000000000004B6E03810000000054940108F8
:10BA2000060003000000000000000000446E0181D9
:10BA300000000000649401080600000000000000FF
:10BA4000000000004F6E00810000000074940108A7
:10BA5000060000000000000000000000436E0381AB
:10BA600000000000849401080600000000000000AF
:10BA700000000000476E018100000000949401085E
:10BA8000060001000000000000000000476E008179
:10BA900000000000A494010806000000000000005F
:10BAA000000000004D6E028100000000C4940108F7
:10BAB0000600000000000000000000004C6E038142
:10BAC00000000000D49401080600000000000000FF
:10BAD000000000004E6E018100000000E4940108A7
:10BAE000060000000000000000000000466E028119
:10BAF00000000000F49401080600000000000000AF
:10BB000000000000446E028100000000049501085E
:10BB10000601010030ED000800000000476E0381BF
:10BB200000000000B495010824030000F4F20008AE
:10BB300000000000476E0381000000002496010809
:10BB4000060000000000000000000000446E0381B9
:10BB500000000000349601080601010070EF0008A3
:10BB6000000000004F6E03810000000044960108B1
:10BB700034010000C81D010878EF00084D6E0381F4
:10BB800000000000549601083401000090EF000806
:10BB9000000000004C6E03810000000014970108B3
:10BBA000240100008402010840F10008486E018170
:10BBB00000000000249701083401000010F3000881
:10BBC000000000004F6E0381000000006497010830
:10BBD0002402000068F5000800000000486E0081A3
:10BBE00000000000749701083401000008020108F9
:10BBF00000000000416E01810000000094970108E0
:10BC00003401000008F3000800000000416E0081CC
:10BC1000000000002498010824020000D0FF000862
:10BC200088F50008446E008100000000D4980108E7
:10BC300024010000B83D010800000000436E0081AF
:10BC400000000000E498010824020000B83D01084B
:10BC5000000000004D6E028100000000349A0108CF
:10BC600034010000C85E010890FD00084E6E03819B
:10BC700000000000349B010834010000005101085D
:10BC800000000000466E018100000000749B010866
:10BC90000600000000000000000000004A6E008165
:10BCA00000000000949B010804020000AC010108A0
:10BCB000600101084B6E018100000000B49B010887
:10BCC000060000000000000000000000446E00813B
:10BCD00000000000C49B010834020000B06C0108A1
:10BCE00000000000466E028100000000549C010824
:10BCF000340200006C780108500601084B6E008188
:10BD000000000000849C010844010000BC6B010895
:10BD1000680601084F6E008100000000B49C010815
:10BD200034010000E0060108000000004A6E0181B5
:10BD300000000000D49C010834020000D441010836
:10BD4000E4060108466E038100000000F49C01082F
:10BD500034020000B03F0108D4080108466E00819B
:10BD600000000000349D0108240300004043010846
:10BD7000900A01084C6E008100000000449D0108FB
:10BD800034020000D87F010800000000426E0281EA
:10BD900000000000C49D010806020200600F0108B7
:10BDA000000000004A6E038100000000F49D0108BD
:10BDB000060000000000000000000000466E018147
:10BDC00000000000249E01080600000000000000A2
:10BDD00000000000456E028100000000B49E0108D2
:10BDE00034010000B03F010868170108496E008166
:10BDF00000000000949F0108060000000000000001
:10BE0000000000004B6E028100000000B49F01089A
:10BE1000060000000000000000000000456E0381E5
:10BE20000000000034A0010806000000000000002F
:10BE300000000000446E008100000000B4A0010872
:10BE40000600000000000000000000004B6E0181B1
:10BE50000000000014A2010834010000D4410108D0
:10BE6000A43601084D6E01810000000094A2010873
:10BE700024010000083C010800000000476E038117
:10BE80000000000014A3010814010000103D010887
:10BE9000083D0108476E02810000000074A30108FC
:10BEA000340100006C780108983D01084A6E038156
:10BEB00000000000D4A3010824010000103E010886
:10BEC000FC3D0108446E01810000000034A401081B
:10BED00034020000F0520108000000004F6E0281A1
:10BEE0000000000034A60108060000000000000069
:10BEF00000000000486E008100000000C4A6010898
:10BF0000060000000000000000000000446E0181F7
:10BF10000000000054A7010834010000D87F010888
:10BF2000000000004A6E00810000000084A70108A4
:10BF3000460004000000000000000000426E018185
:10BF400000000000C4A7010846011000BC48010819
:10BF5000000000004A6E018100000000C4C1010819
:10BF6000060000000000000000000000486E018193
:10BF700000000000B4BE0108060000000000000040
:10BF800000000000456E02810000000024BE010890
:10BF900046001E000000000000000000496E028103
:10BFA0000000000074A8010846001B00000000000B
:10BFB000000000004A6E01810000000084A8010812
:10BFC00044010000D84A0108A84A01084E6E0181C8
:10BFD00000000000A4A8010846013300F44A01084B
:10BFE000000000004D6E028100000000B4A80108AE
:10BFF00046003E0000000000000000004E6E02817E
:10C0000000000000F4A8010846002E000000000017
:10C01000000000004D6E03810000000004A901082B
:10C0200074010000B071010800000000406E018141
:10C030000000000024A9010864010000444C01082C
:10C0400000000000436E028100000000D4BE010821
:10C050000600000000000000000000004F6E01819B
:10C060000000000074A9010864010000D057010815
:10C07000E44D0108456E02810000000094A901080A
:10C0800046000B000000000000000000446E01812B
:10C0900000000000A4A9010844010000885801081C
:10C0A000B44E01084E6E028100000000B4A90108E0
:10C0B0004600090000000000000000004E6E0381F1
:10C0C00000000000C4A90108460022000000000092
:10C0D000000000004B6E028100000000E4A901088E
:10C0E00046004F0000000000000000004A6E03817F
:10C0F00000000000F4A9010846004E000000000006
:10C10000000000004F6E02810000000064AA0108D8
:10C1100046002F000000000000000000416E00817A
:10C120000000000074AA010846002D000000000075
:10C1300000000000436E00810000000094AA010886
:10C1400046034C00EC500108000000004D6E0081D9
:10C1500000000000A4AA010846000300000000003F
:10C1600000000000426E038100000000C4AA010824
:10C17000460057000000000000000000446E0381EC
:10C1800000000000D4AA01084600170000000000CB
:10C1900000000000456E008100000000E4AA0108D4
:10C1A00046004A000000000000000000456E0181CA
:10C1B0000000000014AB010846004200000000002F
:10C1C00000000000446E03810000000034AB010851
:10C1D0004600540000000000000000004C6E00818A
:10C1E0000000000044AB0108460148001452010859
:10C1F00000000000496E03810000000074C10108C6
:10C200004600260000000000000000004B6E018187
:10C210000000000064AB010846000D0000000000B3
:10C2200000000000456E01810000000084AB0108A1
:10C2300046000E000000000000000000496E028170
:10C2400000000000A4AB0108640100007052010866
:10C25000685201084F6E008100000000C4AB010865
:10C26000460001000000000000000000426E038153
:10C270000000000014C101080600000000000000DA
:10C2800000000000496E008100000000E4AB0108DE
:10C29000740100008484010800000000486E0281DF
:10C2A00000000000F4AB010846005200000000004E
:10C2B00000000000406E03810000000014AC010883
:10C2C00074010000F0520108000000004C6E028171
:10C2D0000000000024AC0108740100000C530108A8
:10C2E000FC520108406E01810000000034AC0108DE
:10C2F000460137001453010800000000406E02811F
:10C3000000000000A4BF01080600000000000000BB
:10C31000000000004E6E01810000000074BE0108A4
:10C32000460020000000000000000000466E03816F
:10C330000000000054AC0108440200004053010812
:10C340001C530108436E03810000000094AC0108F7
:10C350005403000014700108C45401084C6E03819A
:10C3600000000000A4AC010864010000245501088D
:10C370001C550108496E028100000000D4AC010880
:10C380004600510000000000000000004A6E0381DA
:10C3900000000000E4AC010874010000A46501087D
:10C3A000B0550108416E01810000000004AD010894
:10C3B000460143000C56010800000000426E008157
:10C3C0000000000024AD010846014D002856010878
:10C3D00000000000416E01810000000074C00108EF
:10C3E000060000000000000000000000486E02810E
:10C3F0000000000064AD0108740300004C56010801
:10C40000E08401084B6E01810000000084AD01084A
:10C41000460134004057010800000000446E0281CC
:10C420000000000094AD010846010C0048570108C7
:10C4300000000000446E01810000000004C20108F9
:10C440000600000000000000000000004E6E0081A9
:10C4500000000000B4AD0108460014000000000018
:10C4600000000000466E008100000000C4AD01081D
:10C47000740100000C5A0108945701084D6E0081A8
:10C4800000000000F4AD01085402000088580108C3
:10C490003C580108436E02810000000004AE010810
:10C4A000460132009458010800000000476E0281E6
:10C4B00000000000D4C1010846021D009C5801087C
:10C4C00000000000456E00810000000094AE0108ED
:10C4D000740200000C5A0108045A01084A6E0281D5
:10C4E00000000000B4AE0108460058000000000043
:10C4F000000000004F6E018100000000C4AE010882
:10C5000074010000545C010800000000416E0081CD
:10C5100000000000D4AE0108460028000000000022
:10C5200000000000406E038100000000F4AE01082E
:10C530004600070000000000000000004B6E038171
:10C540000000000044AF010874010000E45A010833
:10C55000DC5A0108406E01810000000064AF010850
:10C56000460012000000000000000000486E00813C
:10C5700000000000D4AF010846003A0000000000AF
:10C5800000000000456E03810000000014B00108A7
:10C59000460019000000000000000000436E018109
:10C5A0000000000044B0010846000F000000000039
:10C5B000000000004B6E00810000000054B0010834
:10C5C000740200002C5C010800000000466E01812E
:10C5D0000000000084BE010806000000000000000A
:10C5E00000000000446E028100000000A4BE0108AB
:10C5F0000600000000000000000000004C6E0381F7
:10C600000000000004C1010846022300D85C0108B4
:10C6100000000000436E018100000000C4B001086A
:10C6200046013600E85C0108000000004D6E008104
:10C6300000000000E4BF0108060000000000000048
:10C6400000000000446E03810000000004B10108F6
:10C650004600560000000000000000004E6E008101
:10C660000000000034B10108460346005C5D01088B
:10C67000000000004F6E02810000000074B101084C
:10C68000460008000000000000000000476E008126
:10C690000000000044C00108060000000000000087
:10C6A000000000004C6E008100000000B4B10108E1
:10C6B00046013900AC5F010800000000496E0181AD
:10C6C00000000000D4B1010844020000F85F010836
:10C6D000C85F0108406E018100000000D4C001085D
:10C6E000060000000000000000000000446E008111
:10C6F0000000000024B20108460005000000000010
:10C7000000000000436E02810000000044B20108F6
:10C71000460027000000000000000000476E028174
:10C720000000000054B201084601590034600108BD
:10C7300000000000486E02810000000074B2010891
:10C7400046011C0050600108000000004B6E008193
:10C7500000000000A4B2010846014900B4600108CD
:10C7600000000000486E028100000000C4B2010811
:10C7700074010000DC6D010800000000466E0081BD
:10C7800000000000D4B201084600150000000000BF
:10C79000000000004C6E02810000000014B301088C
:10C7A00046003F000000000000000000436E0381CF
:10C7B0000000000034B3010864020000387801086A
:10C7C00058610108476E02810000000044B301086F
:10C7D00044010000B8620108AC620108446E0281A5
:10C7E0000000000014BE0108060000000000000068
:10C7F00000000000426E03810000000064B30108E5
:10C800007401000010760108000000004F6E0081E6
:10C810000000000094BD01080600000000000000B8
:10C8200000000000436E018100000000A4C1010867
:10C83000460000000000000000000000436E02817E
:10C840000000000094B3010846001F000000000033
:10C85000000000004F6E018100000000B4B3010829
:10C860006403000020740108000000004A6E028189
:10C8700000000000F4B30108640100008C640108AA
:10C8800000000000476E03810000000024B401088E
:10C89000460216005C65010800000000446E02813B
:10C8A0000000000084B401084600310000000000D0
:10C8B00000000000456E01810000000094B40108F2
:10C8C00044020000E4660108D4660108426E00815B
:10C8D00000000000A4B401084600060000000000AB
:10C8E00000000000486E02810000000034BF010813
:10C8F000060000000000000000000000496E0181F9
:10C9000000000000F4B4010846013500C0680108C9
:10C91000000000004E6E00810000000004B5010818
:10C92000460002000000000000000000446E038189
:10C9300000000000B4BD010846011A00B0690108FA
:10C94000000000004F6E00810000000084B5010867
:10C95000460138009C6A0108000000004C6E00810E
:10C960000000000024BF010846002900000000006C
:10C97000000000004F6E00810000000024C101088B
:10C98000460018000000000000000000476E008113
:10C990000000000094B501084600530000000000AC
:10C9A00000000000446E01810000000084C0010806
:10C9B00006010100A86C0108000000004E6E008115
:10C9C00000000000E4BE01080600000000000000B6
:10C9D00000000000456E01810000000084BF0108D6
:10C9E0000600000000000000000000004C6E028104
:10C9F0000000000014B601086C010000B06C0108D2
:10CA000000000000416E01810000000044B60108F2
:10CA100046021100D06D010800000000426E028144
:10CA20000000000064BE01080600000000000000D5
:10CA300000000000446E03810000000054B60108AD
:10CA400064010000FC6D010800000000416E0281DD
:10CA50000000000044C101080600000000000000C2
:10CA600000000000406E01810000000074B6010863
:10CA700046014400586E010800000000426E028129
:10CA80000000000084B6010864010000BC6E0108CB
:10CA9000606E0108466E028100000000C4B6010805
:10CAA000460055000000000000000000426E0381B7
:10CAB00000000000F4B6010874010000CC7A0108FF
:10CAC000B06F01084A6E02810000000014B701082F
:10CAD0004600500000000000000000004B6E028184
:10CAE0000000000054B7010874020000D07C010867
:10CAF00000000000426E02810000000074BD0108C9
:10CB00000600000000000000000000004C6E0281E2
:10CB100000000000B4B70108640200008872010838
:10CB200078720108476E008100000000B4C101085E
:10CB300046002A000000000000000000406E038153
:10CB40000000000024B8010846003D00000000007D
:10CB500000000000436E01810000000014BD0108C8
:10CB60000600000000000000000000004A6E038183
:10CB700000000000C4BF01084600250000000000BE
:10CB800000000000416E00810000000084B8010830
:10CB900074010000F4750108D8750108426E018126
:10CBA00000000000D4BC01080600000000000000E6
:10CBB00000000000416E008100000000C4B80108C0
:10CBC000460021000000000000000000466E0081C9
:10CBD00000000000F4B8010846013B00DC760108C3
:10CBE00000000000446E00810000000024B901082C
:10CBF00046004B0000000000000000004C6E018168
:10CC00000000000074B90108460040000000000068
:10CC1000000000004B6E02810000000084B9010892
:10CC2000740100008C7D010828780108486E03819A
:10CC300000000000A4B90108640100003878010870
:10CC400030780108486E008100000000B4B9010886
:10CC50006401000050780108447801084D6E00819D
:10CC600000000000C4B901084601470058780108D7
:10CC7000000000004C6E028100000000D4B90108E1
:10CC8000460030000000000000000000496E0081F6
:10CC900000000000E4B901087401000004790108F3
:10CCA000B87801084B6E03810000000064C10108E0
:10CCB0004600240000000000000000004A6E0081D1
:10CCC0000000000034BA0108440100008C7A010819
:10CCD0003C7A0108436E028100000000A4BA0108FA
:10CCE00074010000A47B0108947B01084F6E008151
:10CCF00000000000F4BA0108460013000000000024
:10CD0000000000004F6E00810000000014BB01080D
:10CD100046024500747C010800000000446E00815A
:10CD20000000000044BB010846003C000000000079
:10CD3000000000004F6E00810000000064BB01088D
:10CD400064010000D07C010800000000466E0281F2
:10CD50000000000074BB010846000A00000000004B
:10CD600000000000456E03810000000084BB010844
:10CD700074010000287D010800000000466E01815A
:10CD800000000000D4BB0108460041000000000084
:10CD900000000000BCC0000800000000E40702081A
:10CDA000C40702088C0702085407020800000000AC
:10CDB000000000000000000000000000220022002F
:10CDC00094CD000840B0000820DD04086C6E040813
:10CDD000346B04084C850508540702088C070208C8
:10CDE000C4070208E4070208ECC6000800000000BF
:10CDF0001C4B020800000000ECC600080000000008
:10CE0000B00C020800000000ECC6000800000000A2
:10CE1000F49503080000000005000500E8CD0008B7
:10CE20004CCD000800000000FC11020800000000CA
:10CE300074C00008000000008C64040800000000BA
:10CE40001CC4000800000000FC11020800000000E3
:10CE50004CCD000800000000FC110208000000009A
:10CE600074C00008000000008C640408000000008A
:10CE70001CC4000800000000FC11020800000000B3
:10CE8000E4CB000800000000F4950308F4950308C3
:10CE9000A813020804080208481302082C08020814
:10CEA000B81202087C080208000000000000000020
:10CEB0000000000000000000000000000000000072
:10CEC00000000000000000004CCD00080000000041
:10CED00094140208000000001CC4000800000000B8
:10CEE00094140208000000004CCD0008000000006F
:10CEF00094140208000000001CC400080000000098
:10CF0000941402080000000094C100080000000012
:10CF1000F4950308F495030898170208EC08020832
:10CF2000BC16020854090208D4150208C4090208F4
:10CF300000000000000000000000000000000000F1
:10CF400000000000000000000000000000000000E1
:10CF5000ECC60008000000001C4B020800000000A6
:10CF6000ECC60008000000001C4B02080000000096
:10CF7000ECC60008000000001C4B02080000000086
:10CF8000ECC60008000000001C4B02080000000076
:10CF9000ECC60008000000001C4B02080000000066
:10CFA000ECC60008000000001C4B02080000000056
:10CFB000ECC60008000000001C4B02080000000046
:10CFC000ECC6000800000000380C02080000000059
:10CFD000ECC6000800000000600C02080000000021
:10CFE000ECC6000800000000B00C020800000000C1
:10CFF000ECC6000800000000B00C020800000000B1
:10D0000005000500F8CD0008ECC60008000000008F
:10D010001C4B020800000000ECC6000800000000E5
:10D020003C0E0208000000000500050008CE0008C4
:10D03000ECC60008000000001C4B020800000000C5
:10D040000A000C0020CE000830CE000840CE0008B8
:10D050000A004B0050CE000860CE000870CE0008D9
:10D0600000000000000000000000000000000000C0
:10D0700000000000000000000000000000000000B0
:10D0800000000000000000000000000000000000A0
:10D090000000000000000000000000000000000090
:10D0A0000000000000000000000000000000000080
:10D0B0000000000000000000000000000000000070
:10D0C0000000000000000000000000000000000060
:10D0D0000000000000000000000000000000000050
:10D0E0000000000000000000000000000000000040
:10D0F0000000000000000000000000000000000030
:10D10000000000000000000000000000000000001F
:10D11000000000000000000000000000000000000F
:10D1200000000000000000000000000000000000FF
:10D1300000000000000000000000000000000000EF
:10D1400000000000000000000000000000000000DF
:10D15000000000000000000080CE00080A000C0063
:10D16000C8CE000800000000D8CE00080A004A001F
:10D17000E8CE000800000000F8CE00080000000023
:10D18000000000000000000000000000000000009F
:10D19000000000000000000000000000000000008F
:10D1A000000000000000000000000000000000007F
:10D1B000000000000000000000000000000000006F
:10D1C000000000000000000000000000000000005F
:10D1D000000000000000000000000000000000004F
:10D1E000000000000000000000000000000000003F
:10D1F000000000000000000000000000000000002F
:10D20000000000000000000000000000000000001E
:10D21000000000000000000000000000000000000E
:10D2200000000000000000000000000000000000FE
:10D2300000000000000000000000000000000000EE
:10D2400000000000000000000000000000000000DE
:10D2500000000000000000000000000000000000CE
:10D2600000000000000000000000000000000000BE
:10D2700008CF00080500050050CF000840B00008A6
:10D2800064B8000820DD04086C6E0408346B0408E0
:10D290004C850508AC0B02081C4B02080500050074
:10D2A00060CF000840B0000864B8000820DD040822
:10D2B0006C6E0408346B04084C850508C00B02082A
:10D2C0001C4B02080500050070CF000840B00008A4
:10D2D00064B8000820DD04086C6E0408346B040890
:10D2E0004C850508D40B02081C4B020805000500FC
:10D2F00080CF000840B0000864B8000820DD0408B2
:10D300006C6E0408346B04084C850508E80B0208B1
:10D310001C4B02080500050090CF000840B0000833
:10D3200064B8000820DD04086C6E0408346B04083F
:10D330004C850508FC0B02081C4B02080500050083
:10D34000A0CF000840B0000864B8000820DD040841
:10D350006C6E0408346B04084C850508100C020838
:10D360001C4B020805000500B0CF000840B00008C3
:10D3700064B8000820DD04086C6E0408346B0408EF
:10D380004C850508240C02081C4B0208050005000A
:10D39000C0CF000840B0000820DD04086C6E04080F
:10D3A000346B04084C850508380C0208050005009C
:10D3B000D0CF000840B0000820DD04086C6E0408DF
:10D3C000346B04084C850508600C02080500050054
:10D3D000E0CF000840B00008FCB6000820DD0408DB
:10D3E0006C6E0408346B04084C850508880C020830
:10D3F000B00C020805000500F0CF000840B000089E
:10D40000FCB6000820DD04086C6E0408346B0408C8
:10D410004C8505089C0C0208B00C02084CCD000895
:10D4200000000000981002080000000074C000080E
:10D43000000000008C640408000000001CC4000808
:10D440000000000098100208000000000500050020
:10D4500008D0000840B0000864B8000854C50008AF
:10D4600000000000E8100208B8100208CC10020802
:10D4700000000000000000000000000005000500A2
:10D4800018D0000840B0000814B7000820DD0408D8
:10D490006C6E0408346B04084C8505083C0E0208C9
:10D4A0000500050030D0000840B0000864B800084E
:10D4B000E4B6000820DD04086C6E0408346B040830
:10D4C0004C850508600E02081C4B02084CCD000874
:10D4D00000000000FC1102080000000074C00008F9
:10D4E0000000000098110208000000001CC40008A1
:10D4F00000000000FC11020800000000E4CB00085E
:10D5000000000000F0130208CC130208A813020860
:10D510007013020848130208E0120208B812020849
:10D52000541202080000000000000000000000008B
:10D5300000000000000000000000000000000000EB
:10D54000000000004CCD0008000000009414020808
:10D55000000000001CC40008000000009414020831
:10D560000000000094C1000800000000F817020845
:10D57000C017020898170208E4160208BC16020831
:10D58000FC150208D415020814150208000000005A
:10D59000000000000000000000000000000000008B
:10D5A000000000000000000000000000010000007A
:10D5B00074C900080A000C001CD400082CD4000810
:10D5C0003CD4000840B00008D4CC000820DD04089A
:10D5D0006C6E0408346B04084C85050800100208C2
:10D5E0003410020884AD05088C6404089810020801
:10D5F000120012005CD4000840B0000820DD0408CE
:10D600006C6E0408346B04084C850508B8100208D9
:10D61000CC100208E810020854C500080000000001
:10D620000C1B0208D41A0208941A02080000000019
:10D6300000000000000000000A004B00CCD40008ED
:10D64000DCD40008ECD4000800000000000000005A
:10D6500000000000000000000000000000000000CA
:10D6600000000000000000000000000000000000BA
:10D6700000000000000000000000000000000000AA
:10D68000000000000000000000000000000000009A
:10D69000000000000000000000000000000000008A
:10D6A000000000000000000000000000000000007A
:10D6B000000000000000000000000000000000006A
:10D6C000000000000000000000000000000000005A
:10D6D000000000000000000000000000000000004A
:10D6E000000000000000000000000000000000003A
:10D6F000000000000000000000000000000000002A
:10D700000000000000000000000000000000000019
:10D710000000000000000000000000000000000009
:10D7200000000000000000000000000000000000F9
:10D7300000000000000000000000000000000000E9
:10D74000FCD4000840B00008D4CC00082CB7000876
:10D7500044B7000820DD04086C6E0408346B04082C
:10D760004C850508581102087011020884AD05089F
:10D7700098110208FC11020854120208B81202089B
:10D78000E01202084813020870130208A8130208E6
:10D79000CC130208F01302080A004A0044D500081E
:10D7A0000000000054D50008000000000000000048
:10D7B0000000000000000000000000000000000069
:10D7C0000000000000000000000000000000000059
:10D7D0000000000000000000000000000000000049
:10D7E0000000000000000000000000000000000039
:10D7F0000000000000000000000000000000000029
:10D800000000000000000000000000000000000018
:10D810000000000000000000000000000000000008
:10D8200000000000000000000000000000000000F8
:10D8300000000000000000000000000000000000E8
:10D8400000000000000000000000000000000000D8
:10D8500000000000000000000000000000000000C8
:10D8600000000000000000000000000000000000B8
:10D8700000000000000000000000000000000000A8
:10D880000000000000000000000000000000000098
:10D8900000000000000000000000000064D5000847
:10D8A00040B00008CCC200085CB7000874B700089C
:10D8B00020DD04086C6E0408346B04084C850508F0
:10D8C000B40205087C2D05082014020828C10508AB
:10D8D00048140208949604087C8D050894140208E4
:10D8E000DC14020814150208D4150208FC150208FD
:10D8F000BC160208E416020898170208C0170208AE
:10D90000F81702088CB7000800000000601A02082F
:10D91000000000001200120018D6000840B00008F5
:10D9200020DD04086C6E0408346B04084C8505087F
:10D93000941A0208D41A02080C1B020840B000080E
:10D94000B4CB000800000000E8280208AC28020858
:10D95000682802083429020820280208142902082D
:10D9600048280208382802080000000000000000D3
:10D9700000000000000000000000000000000000A7
:10D98000000000000000000040B00008B4CB000818
:10D9900000000000842902087C290208742902087A
:10D9A0006C290208642902085C290208542902082B
:10D9B0004C290208000000000000000000000000E8
:10D9C0000000000000000000000000000000000057
:10D9D00000000000ECC6000800000000C02902089A
:10D9E000000000004CCD000800000000642B02087D
:10D9F000000000001CC4000800000000642B0208A6
:10DA0000000000007CCD000800000000606C0208EF
:10DA100000000000A4C30008000000005C6D0208C4
:10DA2000A06C0208000000000000000064CA0008AA
:10DA300000000000D46C02087C6C020800000000AA
:10DA40000000000004CD000800000000A4B700089A
:10DA5000000000009C1D0208C41D0208EC1D020805
:10DA6000081E0208241E020800000000000000003A
:10DA7000000000000000000000000000ECC60008EC
:10DA8000000000001C4B020800000000ECC600086B
:10DA900000000000982E020800000000BCBD000835
:10DAA000000000001C3002083C30020800000000AA
:10DAB00000000000BCBD0008000000004830020863
:10DAC000683002080000000000000000BCBD000833
:10DAD00000000000743002089430020800000000CA
:10DAE00000000000BCBD000800000000A0300208DB
:10DAF000C03002080000000000000000BCBD0008AB
:10DB000000000000CC300208EC30020800000000E9
:10DB100000000000BCBD000800000000F830020852
:10DB2000183102080000000000000000BCBD000821
:10DB30000000000024310208443102080000000007
:10DB400000000000BCBD00080000000050310208C9
:10DB5000703102080000000000000000BCBD000899
:10DB6000000000007C3102089C3102080000000027
:10DB700000000000BCBD000800000000A831020841
:10DB8000C83102080000000000000000BCBD000811
:10DB900000000000D4310208F43102080000000047
:10DBA00000000000BCBD00080000000008320208B0
:10DBB000283202080000000000000000BCBD000880
:10DBC0000000000034320208543202080000000055
:10DBD00000000000BCB7000800000000C8220208D6
:10DBE000E8220208000000000000000074C90008DC
:10DBF0000000000008330208F0320208B0320208C8
:10DC00000000000000000000000000008CBA0008C6
:10DC100000000000603E0208000000004CCD00083B
:10DC20000000000064390208000000001CC4000865
:10DC3000000000006439020800000000ECC6000883
:10DC400000000000CC3E02080000000000000000C0
:10DC500004D9000840B00008ECC60008000000002D
:10DC6000843F020800000000ECC60008000000002D
:10DC7000943F020800000000ECC60008000000000D
:10DC80001C4B02080000000040B0000820DD040822
:10DC90006C6E0408346B04084C850508EC250208FA
:10DCA0001C4B0208ECC60008000000005CDF020804
:10DCB00000000000ECC6000800000000144102084B
:10DCC0000000000054C50008000000008C4102085C
:10DCD000644102084C4102080000000000000000FE
:10DCE0000000000054C5000800000000E4410208E4
:10DCF000BC410208A441020800000000000000002E
:10DD0000000000004CCD00080000000030C20208F6
:10DD1000000000004CCD0008000000009043020805
:10DD20000000000074C00008000000008C640408BB
:10DD3000000000001CC4000800000000904302081E
:10DD4000000000004CCD0008000000001C44020848
:10DD5000000000001CC40008000000001C44020871
:10DD6000000000002100210040D9000840B0000858
:10DD700020DD04086C6E0408346B04084C8505082B
:10DD800020280208382802084828020868280208C3
:10DD9000AC280208E82802081429020834290208DD
:10DDA000210021008CD9000840B0000820DD0408C3
:10DDB0006C6E0408346B04084C8505084C29020875
:10DDC000542902085C290208642902086C29020807
:10DDD000742902087C29020884290208ECC600087C
:10DDE00000000000F846020800000000ECC6000831
:10DDF000000000001C4B02080000000005000500A8
:10DE0000D4D9000840B0000820DD04086C6E040876
:10DE1000346B04084C850508C02902080A000C0070
:10DE2000E4D9000800000000F4D9000840B0000860
:10DE3000CCC2000820DD04086C6E0408346B0408B2
:10DE40004C850508F42902087C2D0508502A020893
:10DE500028C10508FC2A0208949604087C8D050850
:10DE6000642B0208C82B02084100450004DA0008B0
:10DE70000000000014DA00082CDA000844DA000878
:10DE8000000000004CDA000840B00008ECC60008B2
:10DE9000000000001C4B0208000000000500050007
:10DEA0007CDA000854C5000800000000604C02083D
:10DEB000244C0208884B020800000000000000000B
:10DEC00000000000CCCB000800000000804C0208DD
:10DED000604C02084C4C0208244C0208004C02081A
:10DEE000E84B0208C44B0208884B0208704B02083A
:10DEF0000000000000000000000000000000000022
:10DF00000000000000000000000000000000000011
:10DF100000000000ECCC00080000000054D803080A
:10DF200088B0020810C80308D01E0408BC4C0208C0
:10DF300000000000000000000000000000000000E1
:10DF4000000000008CBA000800000000E44C020849
:10DF5000000000002CBA00080000000005000500C9
:10DF60008CDA000840B0000820DD04086C6E04085C
:10DF7000346B04084C850508982E0208ECB700089D
:10DF800000000000F84C02080000000054C5000822
:10DF900000000000504D0208244D0208384D0208D0
:10DFA0000000000000000000000000000000000071
:10DFB0009CDA000840B0000820DD04086C6E0408FC
:10DFC000346B04084C8505081C3002083C300208FC
:10DFD00000000000B4DA000840B0000820DD0408AA
:10DFE0006C6E0408346B04084C8505084830020840
:10DFF0006830020800000000CCDA000840B00008D9
:10E0000020DD04086C6E0408346B04084C85050898
:10E01000743002089430020800000000E4DA0008BE
:10E0200040B0000820DD04086C6E0408346B04085E
:10E030004C850508A0300208C0300208000000002E
:10E04000FCDA000840B0000820DD04086C6E04080B
:10E05000346B04084C850508CC300208EC3002080B
:10E060000000000014DB000840B0000820DD0408B8
:10E070006C6E0408346B04084C850508F8300208FF
:10E0800018310208000000002CDB000840B0000836
:10E0900020DD04086C6E0408346B04084C85050808
:10E0A00024310208443102080000000044DB00086B
:10E0B00040B0000820DD04086C6E0408346B0408CE
:10E0C0004C8505085031020870310208000000003C
:10E0D0005CDB000840B0000820DD04086C6E04081A
:10E0E000346B04084C8505087C3102089C31020819
:10E0F0000000000074DB000840B0000820DD0408C8
:10E100006C6E0408346B04084C850508A8310208BD
:10E11000C8310208000000008CDB000840B0000895
:10E1200020DD04086C6E0408346B04084C85050877
:10E13000D4310208F431020800000000A4DB00081A
:10E1400040B0000820DD04086C6E0408346B04083D
:10E150004C85050808320208283202080000000039
:10E16000BCDB000840B0000820DD04086C6E040829
:10E17000346B04084C850508343202085432020816
:10E1800024C8000800000000F4500208E050020813
:10E19000B85002080000000000000000000000006D
:10E1A00020DD04086C6E0408346B04084C850508F7
:10E1B000B4AC02085CE40408A832020800001800AD
:10E1C000D4DB000800000000000000000000000098
:10E1D000000000000000000000000000000000003F
:10E1E000000000000000000000000000000000002F
:10E1F000000000000000000000000000000000001F
:10E20000000000000000000000000000000000000E
:10E2100000000000000000000000000000000000FE
:10E22000ECDB000840B0000820DD04086C6E040838
:10E23000346B04084C850508B0320208F03202083D
:10E240000833020834BB00080000000054C5000871
:10E250000000000058530208EC520208A0520208C5
:10E2600000000000000000000000000040B00008B6
:10E27000ECB70008000000008C530208000000000A
:10E28000ECC600080000000038C6020800000000CC
:10E2900094C7000800000000F4950308F4950308F3
:10E2A000F4950308F4950308000000000000000046
:10E2B00000000000000000008CBA00080000000010
:10E2C0000443030800000000D4B700080000000069
:10E2D0009833020880340208043502080036020828
:10E2E000BCC7020860360208F036020800000000D1
:10E2F000000000000000000000000000000000001E
:10E3000000000000000000004CC1000800000000F8
:10E310000CC200080000000000000C000CDC00082B
:10E3200000000000000000000000000000000000ED
:10E3300000000000000000000000000000000000DD
:10E34000000000001CDC0008000000002CDC0008BD
:10E350001CAC04086C6E0408346B04084C8505087A
:10E3600088380208A4380208C43802086439020850
:10E3700078DF0408E86A0508503A0208703A020893
:10E38000903A0208B03A0208E03A0208183B020844
:10E39000503B0208883B0208C03B0208F83B0208D9
:10E3A000CC2705086855040864CB0508D4CF0508B8
:10E3B000203C0208403C0208803C0208D43C020891
:10E3C000083D0208283D0208483D0208683D020851
:10E3D000883D0208A83D02083422040828220408C7
:10E3E0001C220408C83D0208F83D02082C3E020821
:10E3F00004220408C0210408882104083C3E0208C5
:10E40000603E02084CCD000800000000804D03086B
:10E41000000000001CC4000800000000804D03083C
:10E4200000000000050005003CDC000820DD0408B9
:10E430006C6E0408346B04084C850508C8DC0308BE
:10E44000880505083C340508703E0208CC3E0208E9
:10E45000ECC6000800000000E456020800000000BE
:10E460000500050058DC0008247B04086C6E0408D5
:10E47000346B04084C85050890C80508A86E04088C
:10E48000386305084818050858C50408BC80050805
:10E49000843F0208404B05080500050068DC0008C1
:10E4A00040B0000820DD04086C6E0408346B0408DA
:10E4B0004C850508943F02080500050078DC00083B
:10E4C00040B0000864B8000820DD04086C6E040841
:10E4D000346B04084C850508F43F02081C4B020805
:10E4E000BCBD0008000000006858030888580308F5
:10E4F00000000000000000006CB9000800000000EF
:10E5000064C202087CC20208B4C2020800C3020846
:10E51000545A02088CC3020840C40208305A020848
:10E520002C410308BCC402080000000000000000E9
:10E5300000000000000000000000000000000000DB
:10E5400000000000000000000000000000000000CB
:10E55000A4BD000800000000C8450308000000003A
:10E5600005000500A4DC000840B000087CC70008D6
:10E5700000000000645C0308505C03080000000019
:10E580000000000005000500B4DC000840B00008F1
:10E5900020DD04086C6E0408346B04084C85050803
:10E5A0001441020840B000086CC8000830B60008EA
:10E5B000ECC60008000000004C4B030800000000FF
:10E5C0004CC1000800000000ECCC00080000000076
:10E5D00054D80308A45B020810C80308D01E04081E
:10E5E0007CB00208000000000000000000000000F5
:10E5F00000000000000000004CC400080000000003
:10E6000040B0000812001200C4DC000840B000084E
:10E6100020DD04086C6E0408346B04084C85050882
:10E620004C410208644102088C41020804BB000806
:10E6300000000000A08F020800000000ECC60008E7
:10E6400000000000C0EC02080000000012001200F0
:10E65000E4DC000840B0000820DD04086C6E04080B
:10E66000346B04084C850508A4410208BC4102082B
:10E67000E4410208B4CB0008000000001C7E03083F
:10E68000BC7D0308587D0308F47C0308907C0308D4
:10E69000107C0308907B03082C7B0308000000001B
:10E6A000000000000000000000000000000000006A
:10E6B000000000000000000000000000ECC60008A0
:10E6C00000000000E4840308000000000A000A00C3
:10E6D00004DD000820DD0408104202081842020888
:10E6E0004C85050830C202080A000C0014DD000841
:10E6F00024DD000834DD000840B00008D4CC000858
:10E7000020DD04086C6E0408346B04084C85050891
:10E710004043020858430208744302088C6404080A
:10E72000904302080A000C0044DD000800000000CD
:10E7300054DD000840B00008CCC2000820DD040809
:10E740006C6E0408346B04084C850508A843020865
:10E750007C2D0508C4430208E4430208044402086F
:10E76000949604087C8D05081C4402083444020871
:10E7700002000000A4C9000884BC000801000000D9
:10E780004CCD000802000000A4C9000884BC0008A9
:10E79000F4C1000800000000408B030800000000E6
:10E7A000A4BD000800000000B489030800000000B8
:10E7B000ECC60008000000005C89030800000000AF
:10E7C00020DD04086C6E0408346B04084C850508D1
:10E7D000E0450208104602082C4602082C84040872
:10E7E00050460208704602088846020854C00508D0
:10E7F000ECD8040805000500DCDD000840B0000886
:10E8000020DD04086C6E0408346B04084C85050890
:10E81000F846020805000500ECDD000840B00008DD
:10E8200064B8000820DD04086C6E0408346B04082A
:10E830004C850508504702081C4B02081CC1000803
:10E8400000000000386C0208246C0208F0AA0208DC
:10E85000B8A90208106C020848A9020830A90208E9
:10E86000006C0208286B0208586A020880690208D6
:10E870000000000000000000000000000000000098
:10E880000000000000000000000000000000000088
:10E89000000000000000000000000000ECC60008BE
:10E8A000000000004C4B0308000000008CBA000878
:10E8B00000000000046E0208000000007CCD00088B
:10E8C00000000000606C020800000000A4C3000803
:10E8D000000000005C6D0208A06C0208000000004F
:10E8E0000000000064CA000800000000D46C0208A8
:10E8F0007C6C0208000000000000000004CD00084D
:10E900000000000034C1000800000000A46E0208EE
:10E910003C6E02085C6D0208D46C02080000000026
:10E9200000000000000000000000000005000500DD
:10E930008CDE000840B0000864B8000820DD040840
:10E940006C6E0408346B04084C850508084B0208FB
:10E950001C4B0208BCBD000800000000089F030813
:10E96000289F03080000000000000000ECC600081B
:10E9700000000000E4A40308000000005CBA0008E6
:10E9800000000000B48403080000000012003B00F7
:10E99000A4DE0008000000000000000000000000ED
:10E9A0000000000000000000000000000000000067
:10E9B0000000000000000000000000000000000057
:10E9C0000000000000000000000000000000000047
:10E9D0000000000000000000000000000000000037
:10E9E0000000000000000000000000000000000027
:10E9F0000000000000000000000000000000000017
:10EA00000000000000000000000000000000000006
:10EA100000000000000000000000000000000000F6
:10EA200000000000000000000000000000000000E6
:10EA300000000000C4DE000840B0000820DD04082B
:10EA40006C6E0408346B04084C850508704B020892
:10EA5000884B0208C44B0208E84B0208004C02082D
:10EA6000244C02084C4C0208604C0208804C0208FE
:10EA70000300140098F300080000000000000000EC
:10EA80000000000000000000000000000000000086
:10EA90000000000000000000000000000000000076
:10EAA0000000000000000000000000000000000066
:10EAB0000000000014DF0008D0F3000870380408DC
:10EAC000D01E040854D8030868B00208BC4C0208E1
:10EAD00010C803087035030888B00208E49F0308D3
:10EAE000EC9F03080000000044DF000840B000086D
:10EAF00020DD04086C6E0408346B04084C8505089E
:10EB0000E44C02080000000054DF000840B0000898
:10EB1000000000007CDF000820DD04086C6E0408A3
:10EB2000346B04084C850508F84C020812001200EA
:10EB30008CDF000840B0000820DD04086C6E04087B
:10EB4000346B04084C850508244D0208384D020832
:10EB5000504D0208CCB9000800000000ECB70008D6
:10EB600000000000ACB80308000000000000000036
:10EB700080E1000840B0000820DD04086C6E040845
:10EB8000346B04084C850508B8500208E0500208B0
:10EB9000F45002080000000044E2000840B0000801
:10EBA0000CC50008000000001076020800000000FC
:10EBB0004CB8000800000000C85102080000000026
:10EBC00004C70008000000004C76020800000000A6
:10EBD0004CCD00080000000014D205080000000021
:10EBE00074C00008000000008C64040800000000ED
:10EBF0001CC400080000000014D20508000000003A
:10EC0000020000003CBF00089CC500080300000093
:10EC10003CB900089CC500083CBF00081200120067
:10EC20004CE2000840B0000820DD04086C6E0408C7
:10EC3000346B04084C850508A0520208EC52020807
:10EC4000585302080000000070E2000840B00008BD
:10EC50001052000820DD04086C6E0408346B0408B0
:10EC60004C8505088C5302080500050080E2000869
:10EC7000BCC00008000000004C7C02080C7C0208AC
:10EC8000287B0208887A02080000000000000000CB
:10EC900000000000000000003F003F0090E200087C
:10ECA000ECC6000800000000787C020800000000AC
:10ECB000FCBF000800000000207D020800000000EA
:10ECC00000000100B8E20008C8E2000840B00008F7
:10ECD00003000D0008E30008000000000000000031
:10ECE0000000000000000000000000000000000024
:10ECF00000000000000000000000000010E3000819
:10ED0000C8630408D8540208E05402084C8505087A
:10ED100030550208885502080A000C0004E4000877
:10ED20000000000014E4000840B00008CCC2000855
:10ED300001000000ECC600080500050050E40008D2
:10ED400040B0000820DD04086C6E0408346B040831
:10ED50004C850508E456020820DD040838B4030891
:10ED6000346B04084C85050858260508D496050818
:10ED7000F0B0040804570208AC69040864BF040832
:10ED80003C57020800000000E0E4000840B0000822
:10ED9000A4BD000800000000D887020800000000A1
:10EDA00020DD04086C6E0408346B04084C850508EB
:10EDB000045802086CB900080000000064C2020890
:10EDC0007CC20208B4C2020800C3020884AF030870
:10EDD0008CC3020840C4020860AF030830AF0308C8
:10EDE000BCC4020800000000000000000000000099
:10EDF0000000000000000000000000000000000013
:10EE00000000000000000000000000000000000002
:10EE1000F8E4000820DD04086C6E0408346B040874
:10EE20004C850508C05902082C410308305A0208D5
:10EE3000545A0208A45A02080000000050E50008D5
:10EE400040B000084078000820DD04086C6E04081B
:10EE5000346B04084C850508CC5A0208F45A0208A1
:10EE6000150015006CE5000840B0000840B000082F
:10EE700005000500B0E5000840B0000894BB00089C
:10EE800020DD04086C6E0408346B04084C8505080A
:10EE90002C5B02084C4B030820DD04086C5B020865
:10EEA0005C5B02084C850508249F04083859050856
:10EEB00008A50508BC8B050840B000086CC8000810
:10EEC00030B600083055000820DD04086C5B0208ED
:10EED000745B02084C850508249F0408385905080E
:10EEE00008A50508BC8B050803001400C0E5000850
:10EEF0000000000000000000000000000000000012
:10EF00000000000000000000000000000000000001
:10EF100000000000000000000000000000000000F1
:10EF2000000000000000000000000000C8E500082C
:10EF3000F8E5000870380408D01E040854D8030807
:10EF400068B002087CB0020810C803089C5B020885
:10EF5000A45B0208E49F0308EC9F030840B000088C
:10EF6000ECC60008000000004C4B03080000000045
:10EF7000010000001CBE0008010005002CE600088E
:10EF80000000000000000000000000003CE6000857
:10EF900040B000082100210074E6000854C50008B4
:10EFA000000000004C9102082091020874900208B1
:10EFB00000000000000000000000000020DD040848
:10EFC0006C6E0408346B04084C850508005C02086C
:10EFD000245C020840B000081CB8000800000000D3
:10EFE00004930208449202080000000000000000A0
:10EFF00005000500BCE6000840B00008ACBB0008F6
:10F0000040B00008E0AF00089094000826002600F9
:10F0100090E7000840B0000800000500A0E70008E5
:10F0200000000000000000000000000000000000E0
:10F03000B0E7000840B0000840B00008E0AF0008AA
:10F04000909400084CCD00080000000088A8020839
:10F05000000000001CC400080000000088A802088E
:10F0600000000000A4CC000800000000F495030894
:10F07000F4950308F4950308E8000308848D030859
:10F08000408D0308000000000000000000000000A8
:10F090000000000000000000000000001CC100088B
:10F0A000000000008CA9020870A90208F0AA02085A
:10F0B000B8A9020860A9020848A9020830A90208F4
:10F0C00018A9020800A90208E8A80208D0A80208A6
:10F0D0000000000000000000000000000000000030
:10F0E0000000000000000000000000000000000020
:10F0F0000000000000000000000000002D002D00B6
:10F100003CE8000820DD0408FC68020820690208C9
:10F110004C85050880690208586A0208286B0208B5
:10F12000006C020830A9020848A90208106C020805
:10F13000246C0208386C0208B8A90208F0AA020878
:10F14000050005009CE8000804C700080000000056
:10F150001CD30208000000005CBA00080000000098
:10F1600088AC02080000000000004C00ACE8000879
:10F17000000000000000000000000000000000008F
:10F18000000000000000000000000000000000007F
:10F19000000000000000000000000000000000006F
:10F1A000000000000000000000000000000000005F
:10F1B000000000000000000000000000000000004F
:10F1C000000000000000000000000000000000003F
:10F1D000000000000000000000000000000000002F
:10F1E000000000000000000000000000000000001F
:10F1F000000000000000000000000000000000000F
:10F2000000000000000000000000000000000000FE
:10F2100000000000000000000000000000000000EE
:10F2200000000000000000000000000000000000DE
:10F2300000000000000000000000000000000000CE
:10F2400000000000000000000000000000000000BE
:10F2500000000000000000000000000000000000AE
:10F26000000000000000000000000000000000009E
:10F27000BCE8000800000000CCE80008E4E8000852
:10F28000FCE8000800000000000000000000000092
:10F2900000000000000000000000000004E9000879
:10F2A00040B0000834B8000820DD04086C6E040883
:10F2B000346B04084C850508606C02087C6C0208FD
:10F2C000A06C0208D46C02085C6D0208046E02088F
:10F2D0003C6E0208A46E02085CBA00080000000040
:10F2E000A8AC020800000000CCB900080000000033
:10F2F00040B0000840B00008DCBB0008C4BB0008F8
:10F300001CBB000840B0000840B00008F4BB000877
:10F3100040B00008ACBB000820DD04086C6E040897
:10F32000346B04084C850508C46F02080000000017
:10F3300054E9000840B0000820DD0408EC6F020822
:10F34000F46F02084C850508249F04083859050805
:10F3500008A50508BC8B05088CBA00080000000051
:10F36000F4AE0208000000004CCD000800000000D0
:10F3700084AF02080000000074C000080000000014
:10F380008C640408000000001CC400080000000099
:10F3900084AF0208000000004CC10008000000001B
:10F3A000ECCC00080000000054D8030888B0020824
:10F3B00010C80308D01E04087CB00208000000003A
:10F3C000000000000000000000000000000000003D
:10F3D0004CC40008000000004CC100080000000000
:10F3E000ECCC00080000000054D80308F495030892
:10F3F00010C80308D01E04087CB0020800000000FA
:10F4000000000000000000000000000000000000FC
:10F410004CC4000800000000050005006CE900086D
:10F4200040B00008000000007CE9000840B000087F
:10F43000ECC60008000000004C4B03080000000070
:10F44000E4C8000800000000081E0308581E030856
:10F45000781E0308881E0308401F0308801F030846
:10F46000AC200308502103081C220308C42203080F
:10F470005C23030800240308A424030818250308B8
:10F4800058250308302603083427030834280308C6
:10F49000002A0308982A0308302B0308D02B0308FE
:10F4A000702C0308102D0308F42D0308287102089E
:10F4B00040710208E02E0308182F03080000000026
:10F4C000000000000000000000000000000000003C
:10F4D000000000000000000000000000000000002C
:10F4E000000000000000000000000000000000001C
:10F4F000000000000000000000000000000000000C
:10F5000000000000000000000000000000000000FB
:10F5100000000000000000000000000000000000EB
:10F5200000000000000000000000000000000000DB
:10F530004CC1000800000000ECCC000800000000F6
:10F5400054D80308F495030810C80308D01E040813
:10F55000C0DB030800000000000000000000000005
:10F56000000000000000000040B00008DCBB000804
:10F57000C4BB000820DD04086C6E0408346B04086A
:10F580004C850508A07102080000000054EB00083B
:10F59000CCB90008000000008CBA00080000000090
:10F5A000944A03080000000094CA0008000000000C
:10F5B00014470308984903080000000000000000F9
:10F5C0008CBA000800000000EC6A0308000000008C
:10F5D00094CA000800000000D8670308006A030806
:10F5E000000000000000000020DD04086C6E04082C
:10F5F000346B04084C850508B8710208DC710208F8
:10F60000FC710208207202084072020890B60408D9
:10F610005C720208000000005CEB000840B00008CB
:10F6200084C5000800000000F0400408000000004D
:10F630002CC9000800000000F0400408BC40040889
:10F64000D4400408704004080000000000000000DE
:10F65000000000000000000034C7000800000000A7
:10F660005C40040800000000FCC500080000000029
:10F6700044400408000000008CBA000800000000AC
:10F68000A04204080000000028002800A0EB0008A9
:10F6900040B0000820DD04086C6E0408346B0408D8
:10F6A0004C8505081076020800000000B0EB000849
:10F6B00040B0000827002700C0EB000840B0000859
:10F6C00020DD04086C6E0408346B04084C850508C2
:10F6D0004C7602080A000C00D0EB0008E0EB0008B2
:10F6E000F0EB000840B00008D4CC000840B000089F
:10F6F000ECC600080000000038C602080000000048
:10F70000FCBF00080000000060C602080000000006
:10F71000E4BF0008000000004842030800000000A9
:10F7200094C700080000000000420308904103084D
:10F73000184203080842030800000000000000000F
:10F740000000000000000000BCC300080000000032
:10F750002200220070EC000840B0000820DD040800
:10F760006C6E0408346B04084C850508887A02081E
:10F77000287B02080C7C02084C7C0208050005006E
:10F78000A0EC000840B0000820DD04086C6E0408FE
:10F79000346B04084C850508787C02082E002E0086
:10F7A000B0EC000840B0000820DD04086C6E0408CE
:10F7B000346B04084C850508207D02080000000019
:10F7C0005010010820DD04086C6E0408346B040836
:10F7D0004C850508B4860208D886020824870208EA
:10F7E000508702080000000090ED000840B00008BB
:10F7F000507E000820DD04086C6E0408346B040899
:10F800004C85050894870208D887020840B0000894
:10F8100000000000B4ED000840B00008C07500080A
:10F8200040B0000834BE00080000000058E10208A3
:10F83000000000004CC100080000000044C60008A1
:10F84000000000009CC5000800000000ECEA02086F
:10F85000000000003CBF00080000000058EB020858
:10F8600040EB020830EB02081CEB020804A9050873
:10F870006C6B0408ECEE040808EB0208ECEA0208E2
:10F880008C40050830240508BCB70408D8EA0208F3
:10F890001C930408CCB20508000000000000000022
:10F8A0000000000000000000000000000000000058
:10F8B0000000000000000000000000000000000048
:10F8C0000000000000000000000000000000000038
:10F8D0000000000004CA00080000000058EB020805
:10F8E00040EB020830EB02081CEB020804A90508F3
:10F8F0006C6B0408ECEE040808EB0208ECEA020862
:10F900008C40050830240508BCB70408D8EA020872
:10F910001C930408CCB205080000000000000000A1
:10F9200000000000000000000000000000000000D7
:10F9300000000000000000000000000000000000C7
:10F9400000000000000000000000000000000000B7
:10F9500000000000ECC600080000000070EB020888
:10F96000000000000500050060EF000840B000083E
:10F9700094BB000820DD04086C6E0408346B040896
:10F980004C850508848F02084C4B03088CBA00088C
:10F9900000000000EC6A03080000000094CA0008A0
:10F9A00000000000F4950308F4950308000000002F
:10F9B000000000007CC7000800000000DCEB02082B
:10F9C000A8EB020800000000000000003CBF000897
:10F9D00000000000841A03086C1A03085C1A03086C
:10F9E000301A030804A90508841903086C6E04087A
:10F9F0001C1A0308081A0308D0190308986F050891
:10FA0000BCB70408C41903081C930408CCB2050849
:10FA100000000000000000000000000000000000E6
:10FA200000000000000000000000000000000000D6
:10FA300000000000000000000000000000000000C6
:10FA400000000000000000000000000004BB0008EF
:10FA50000000000088EC0208000000008CBD0008D7
:10FA60000000000008ED0208ECEC020800000000B5
:10FA700000000000ECC6000800000000C0EC020816
:10FA80000000000020DD04086C6E0408346B0408DC
:10FA90004C850508DC070408D4070408AC070408F3
:10FAA000B05C04082CF603080C90020838C0050866
:10FAB000B88E0408B49F0508BC680508547C040887
:10FAC000189002082090020828900208CCCB000869
:10FAD00000000000EC370308004F0308CC37030890
:10FAE00098360308C4370308B8EE02085C370308E9
:10FAF000304E03080C37030800000000000000002F
:10FB000000000000000000000000000000000000F5
:10FB10000000000000000000000000009CC500087C
:10FB2000000000002CEF0208000000003CBF0008AD
:10FB30000000000098EF020880EF020870EF020852
:10FB40005CEF020804A90508346B04086C6E040815
:10FB500048EF02082CEF02088C400508986F050852
:10FB6000BCB7040818EF02081C930408CCB20508BF
:10FB70000000000000000000000000000000000085
:10FB80000000000000000000000000000000000075
:10FB90000000000000000000000000000000000065
:10FBA00000000000000000000000000040B000085D
:10FBB000120015009CEF000800000000000000008B
:10FBC0001006010820DD04086C6E0408346B04087C
:10FBD0004C8505086C900208501B0308B41B0308F1
:10FBE00074900208209102084C91020840B000086D
:10FBF0005C910208A8910208DC9102084C85050876
:10FC00002C002C00D8EF000840B0000844920208F5
:10FC10006C6E0408346B04084C8505086492020875
:10FC20000493020840B000087CB8000800000000FF
:10FC3000D01104081834040800000000000000007F
:10FC400040B0000894B800080000000014970208B3
:10FC500050970208E09802082C9B0208709B02084B
:10FC6000B89B0208049C02081C9C020800000000CB
:10FC70000000000000000000000000000000000084
:10FC80000000000000000000000000006CCB000835
:10FC900000000000D0F8020888F802080000000008
:10FCA000000000006CCB000800000000FCF8020817
:10FCB000E4F802080000000000000000ACB80008F2
:10FCC00000000000849E02089C9E0208CC9E020850
:10FCD000EC9E020800000000000000000000000090
:10FCE000000000004CCD000800000000F4A903084B
:10FCF00000000000C4B800080000000048A202088C
:10FD000078A20208A4A20208F0A2020808A204082D
:10FD100000000000000000000000000000000000E3
:10FD2000000000005CBA000800000000F4030308B3
:10FD300000000000DCB8000800000000ECC600086D
:10FD40000000000034040308000000000A000C005A
:10FD500044F000080000000054F0000820DD040812
:10FD60006C6E0408346B04084C85050818A602085C
:10FD70007C2D0508FCA6020838A8020850A8020835
:10FD8000949604087C8D050888A80208B8A8020883
:10FD90002400240064F000082D002D009CF00008D1
:10FDA00040B00008A05F0008F4B8000820DD040897
:10FDB0006C6E0408346B04084C850508D0A8020852
:10FDC000E8A8020800A9020818A9020830A9020838
:10FDD00048A9020860A9020870A902088CA90208B3
:10FDE000B8A90208F0AA0208ECC60008000000004A
:10FDF0004C4B03080000000040B00008ACBB0008FA
:10FE00000000270050100108581001086810010870
:10FE10000000000000000000801001080000000049
:10FE200000000000000000000000000000000000D2
:10FE300000000000000000000000000000000000C2
:10FE400000000000000000000000000000000000B2
:10FE500000000000000000000000000000000000A2
:10FE60000000000000000000000000000000000092
:10FE70000000000000000000000000000000000082
:10FE80000000000000000000000000000000000072
:10FE90000000000000000000000000000000000062
:10FEA00048F1000820DD04086C6E0408346B040877
:10FEB0004C85050810AC020818AC0208D0D2020824
:10FEC00000D302081CD3020840D302086855030877
:10FED000845503089C55030820AC020860AC020856
:10FEE000B8560308D05603080000000058F1000877
:10FEF00040B0000820DD04086C6E0408346B040870
:10FF00004C85050888AC020800000000D8F2000803
:10FF100040B0000820DD04086C6E0408346B04084F
:10FF20004C850508A8AC0208ECC6000800000000DB
:10FF3000400603080000000020DD04086C6E040881
:10FF4000346B04084C850508B4AC02085CE4040872
:10FF500008AD0208ECBD00080000000020AD02085A
:10FF600064AD02080000000000000000CCB90008E9
:10FF700000000000E4B900080000000030C90208D9
:10FF8000BCC90208D4C9020880CA020888CA02088B
:10FF900090CA0208000000000000000000000000FD
:10FFA000000000000000000000000000FCB9000894
:10FFB0000000000014BA0008000000000CB900089E
:10FFC0000000000040B0000800000000E8F2000857
:10FFD00040B00008DCBB00080CBC000834BE0008C0
:10FFE000000000000C0A030800000000FCB9000833
:10FFF0000000000040B00008F4BB000820DD040849
:020000040801F1
:100000006C6E0408346B04084C8505084CAE02087D
:10001000FCAD020840B00008F4BB000820DD040875
:100020006C6E0408346B04084C8505084CAE02085D
:1000300030AE020840B00008F4BB000820DD040820
:100040006C6E0408346B04084C8505084CAE02083D
:1000500064AE02087CC7000800000000E00A030844
:10006000CC0A0308000000000000000040B00008B7
:1000700040B00008ECC6000800000000040F0308B0
:100080000000000040B000080000000058F3000825
:1000900040B0000820DD04086C6E0408346B0408CE
:1000A0004C850508F4AE02080A000C0068F300084D
:1000B00078F3000888F3000820DD04086C6E04085B
:1000C000346B04084C85050830AF020854AF0208B1
:1000D0006CAF02088C64040884AF020803001400AB
:1000E00098F300080000000000000000000000007D
:1000F0000000000000000000000000000000000000
:1001000000000000000000000000000000000000EF
:1001100000000000000000000000000000000000DF
:10012000A0F30008D0F3000840B00008FCBC0008B1
:100130009CBC0008E062000870380408D01E040867
:1001400054D8030868B002087CB0020810C803083D
:100150007035030888B00208E49F0308EC9F030889
:1001600003001400D8F300080000000000000000A5
:10017000000000000000000000000000000000007F
:10018000000000000000000000000000000000006F
:10019000000000000000000000000000000000005F
:1001A00000000000E0F3000810F4000840B0000870
:1001B000FCBC00089CBC000840B0000810630008AC
:1001C00054C5000800000000A410030878100308BC
:1001D0008C10030800000000000000000000000078
:1001E000B4BC000800000000E0B00208E8B002085B
:1001F000F0B00208F8B002080000000000000000A3
:10020000000000000000000040B00008DCBB000857
:1002100040B000085CBA0008000000007C7F0308C2
:10022000000000007CC700080000000098110308CF
:10023000841103080000000000000000ECC6000864
:1002400000000000241203080000000040B0000875
:1002500020DD04086C6E0408346B04084C85050826
:10026000E8B1020834D5020860D50208F8B10208E6
:1002700000B2020818B202082CB2020805000500FC
:1002800030F4000840B0000894BB000820DD0408EA
:100290006C6E0408346B04084C85050848B20208EB
:1002A0004C4B030840B0000840B000086CC8000880
:1002B00030B6000824B9000884C800080000000017
:1002C00070380508E018030810A70508741803081B
:1002D0003C8C0408C091050804A9050880B20408F4
:1002E00028180308905A05088C9F05084421050822
:1002F000A016030864E7040888040508D417030857
:10030000701703088C400508986F0508BCB70408EF
:10031000D01603087C1603085C1603081C93040817
:10032000CCB2050800000000000000000000000042
:1003300000000000000000000000000000000000BD
:1003400000000000000000000000000000000000AD
:10035000000000000000000000000000000000009D
:10036000000000000000000000000000000000008D
:10037000000000000000000000000000000000007D
:1003800000000000000000007CC100080000000028
:100390009CC5000800000000A01603080000000033
:1003A0003CBF0008000000007038050810A70508D1
:1003B0003C8C0408C091050804A9050880B2040813
:1003C000905A050844210508A01603088C4005082A
:1003D000986F0508BCB704087C1603081C93040832
:1003E000CCB2050800000000000000000000000082
:1003F00000000000000000000000000000000000FD
:1004000000000000000000000000000000000000EC
:1004100000000000000000000000000000000000DC
:1004200084C800080000000070380508E0180308C0
:1004300010A70508741803083C8C0408C09105082F
:1004400004A9050880B2040828180308905A050872
:100450008C9F050844210508A016030864E70408DA
:1004600088040508D4170308701703088C40050892
:10047000986F0508BCB70408D01603087C1603085B
:10048000B01603081C930408CCB205080000000055
:10049000000000000000000000000000000000005C
:1004A000000000000000000000000000000000004C
:1004B000000000000000000000000000000000003C
:1004C000000000000000000000000000000000002C
:1004D000000000000000000000000000000000001C
:1004E000000000000000000000000000000000000C
:1004F0009CC5000800000000081A03080000000066
:100500003CBF000800000000841A03086C1A0308AE
:100510005C1A0308301A030804A9050884190308A3
:10052000401903081C1A0308081A0308D019030805
:10053000986F0508BCB70408C41903081C93040885
:10054000CCB2050800000000000000000000000020
:10055000000000000000000000000000000000009B
:10056000000000000000000000000000000000008B
:10057000000000000000000000000000000000007B
:1005800004CA000800000000841A03086C1A03085B
:100590005C1A0308301A030804A905088419030823
:1005A000401903081C1A0308081A0308D019030885
:1005B000986F0508BCB70408C41903081C93040805
:1005C000CCB20508000000000000000000000000A0
:1005D000000000000000000000000000000000001B
:1005E000000000000000000000000000000000000B
:1005F00000000000000000000000000000000000FB
:10060000DCC40008000000001CC700080000000057
:100610007CC7000800000000B41B0308501B03083F
:1006200000000000000000008CBA0008000000007C
:10063000944A03080000000094CA0008000000006B
:10064000F4950308F4950308000000000000000082
:100650000000000040F400082CBA00080000000070
:1006600040B0000840B000080300130030F5000857
:10067000000000000000000000000000000000007A
:10068000000000000000000000000000000000006A
:10069000000000000000000000000000000000005A
:1006A00000000000000000000000000038F5000815
:1006B00040B00008DCBB0008C4BB0008000000001C
:1006C00090F5000840B00008DCBB000820DD0408FD
:1006D0006C6E0408346B04084C8505088CB802085D
:1006E00040B000080000550098F500080000000028
:1006F00000000000000000000000000000000000FA
:1007000000000000000000000000000000000000E9
:1007100000000000000000000000000000000000D9
:1007200000000000000000000000000000000000C9
:1007300000000000000000000000000000000000B9
:1007400000000000000000000000000000000000A9
:100750000000000000000000000000000000000099
:100760000000000000000000000000000000000089
:100770000000000000000000000000000000000079
:100780000000000000000000000000000000000069
:100790000000000000000000000000000000000059
:1007A0000000000000000000000000000000000049
:1007B0000000000000000000000000000000000039
:1007C0000000000000000000000000000000000029
:1007D0000000000000000000000000000000000019
:1007E0000000000000000000000000000000000009
:1007F00000000000000000000000000000000000F9
:1008000000000000000000000000000000000000E8
:1008100000000000000000000000000000000000D8
:1008200000000000000000000000000000000000C8
:10083000000000000000000000000000A8F5000813
:1008400054C5000800000000004F03089C4E030838
:10085000304E03080000000000000000000000000F
:1008600040B0000854C5000800000000004F030815
:1008700098360308304E0308000000000000000016
:1008800000000000CCCB000800000000EC3703089B
:10089000004F0308CC37030898360308C437030811
:1008A000783703085C370308304E03080C37030819
:1008B0000000000000000000000000000000000038
:1008C0000000000000000000000000000000000028
:1008D0000000000000005500C0F500080000000006
:1008E0000000000000000000000000000000000008
:1008F00000000000000000000000000000000000F8
:1009000000000000000000000000000000000000E7
:1009100000000000000000000000000000000000D7
:1009200000000000000000000000000000000000C7
:1009300000000000000000000000000000000000B7
:1009400000000000000000000000000000000000A7
:100950000000000000000000000000000000000097
:100960000000000000000000000000000000000087
:100970000000000000000000000000000000000077
:100980000000000000000000000000000000000067
:100990000000000000000000000000000000000057
:1009A0000000000000000000000000000000000047
:1009B0000000000000000000000000000000000037
:1009C0000000000000000000000000000000000027
:1009D0000000000000000000000000000000000017
:1009E0000000000000000000000000000000000007
:1009F00000000000000000000000000000000000F7
:100A000000000000000000000000000000000000E6
:100A100000000000000000000000000000000000D6
:100A2000000000000000000000000000D0F50008F9
:100A3000BCB802086C6E0408346B04084C850508C9
:100A4000249F04083859050808A50508BC8B05082B
:100A5000A0420408B4420408E042040840B0000880
:100A60001900230020F6000830F6000800000000FE
:100A700058F6000800000000000000000000000020
:100A800000000000000000000000000068F6000800
:100A90000000000078F600084CC1000800000000CB
:100AA00024BF00080000000060620308346B0408E3
:100AB000000000000000000014C900080000000051
:100AC000A8D90408000000004CC100080000000084
:100AD0003CB9000800000000DC3F030828C0020801
:100AE00040C00208000000000000000000000000FC
:100AF00054B9000800000000DC3F030828C00208C9
:100B000040C00208243F0308703F0308083F030861
:100B10003C3F03080000000000000000000000004F
:100B200000000000000000000000000000000000C5
:100B30004CC10008000000009CC500080000000037
:100B40003C3F0308000000003CBF0008000000001C
:100B5000DC3F030810A70508AC3F0308703F0308FB
:100B600004A90508346B04086C6E04085C3F030894
:100B70003C3F0308243F0308986F0508BCB70408EE
:100B8000083F0308E83E0308B03E030800000000E9
:100B90000000000000000000000000000000000055
:100BA0000000000000000000000000000000000045
:100BB0000000000000000000000000000000000035
:100BC00000000000000000004CC40008000000000D
:100BD0004CCD00080000000030C2020800000000F8
:100BE000ECC6000800000000448503080000000077
:100BF00040B000086CB900080000000064C20208A0
:100C00007CC20208B4C2020800C3020884AF030811
:100C10008CC3020840C4020860AF03082C410308DB
:100C2000BCC402080000000000000000000000003A
:100C300000000000000000000000000000000000B4
:100C400000000000000000000000000040B00008AC
:100C500084B9000805000500F0F6000840B000085F
:100C60009CB9000820DD04086C6E0408346B04088D
:100C70004C85050838C602082E002E0000F7000833
:100C800040B0000820DD04086C6E0408346B0408D2
:100C90004C85050860C602083E004D0010F70008AC
:100CA00020F7000800000000000000000000000025
:100CB0000000000000000000000000000000000034
:100CC0000000000000000000000000000000000024
:100CD000000000000000000048F7000840B00008D5
:100CE000B4B9000814C9000800000000A8D904081D
:100CF000000000004CC1000800000000E4C800082B
:100D000000000000F4950308F4950308781E03081A
:100D1000F4950308F4950308F4950308AC20030840
:100D2000502103081C220308C42203085C23030883
:100D300000240308A4240308F49503085825030895
:100D4000302603083427030834280308002A030840
:100D5000982A0308302B0308D02B0308702C0308B3
:100D6000102D0308F42D0308F4950308F4950308E7
:100D7000E02E0308F49503080000000000000000C6
:100D80000000000000000000000000000000000063
:100D90000000000000000000000000000000000053
:100DA0000000000000000000000000000000000043
:100DB0000000000000000000000000000000000033
:100DC0000000000000000000000000000000000023
:100DD0000000000000000000000000000000000013
:100DE00000000000000000000000000014C900081E
:100DF00000000000A8D90408000000004CC1000851
:100E00000000000014C9000800000000BC430308F3
:100E1000000000004CC1000800000000CCB9000830
:100E200000000000E4B900080000000030C902081A
:100E3000BCC90208D4C9020880CA020888CA0208CC
:100E400090CA02080000000000000000000000003E
:100E5000000000000000000000000000FCB90008D5
:100E60000000000014BA0008000000002CBA0008BE
:100E700000000000ECC6000800000000A0640308A9
:100E8000000000005CBA00080000000004450308F0
:100E9000000000008CBA000800000000EC6A0308A3
:100EA0000000000094CA000800000000D867030892
:100EB000006A0308000000000000000044BA0008B7
:100EC00000000000C4CA02080000000014C90008A5
:100ED00000000000A8D90408000000004CC1000870
:100EE000000000005CBA000800000000184603087B
:100EF0000000000074BA00080000000014C90008D7
:100F000000000000A8D90408000000004CC100083F
:100F100000000000ECC600080000000024460308A2
:100F2000000000008CBA000800000000944A03088A
:100F30000000000094CA00080000000014470308E5
:100F40009849030800000000000000008CBA000867
:100F500000000000A04204080000000040B00008AB
:100F60000200000004BB0008ECC6000840B0000806
:100F700014C9000800000000A8D9040800000000FF
:100F80004CC100080000000040B00008A4BA0008EE
:100F90000000000058CF020800000000DCBE00087E
:100FA00000000000184E0308FC4D0308F44D030830
:100FB000000000000000000000000000BCBA0008B3
:100FC0000000000060CF020878CF02088CCF020832
:100FD00000000000000000000000000040B0000819
:100FE000D4BA0008000000000CD002080000000085
:100FF00020DD04086C6E0408346B04084C85050879
:1010000090D0020898D00208DCBE00080000000062
:101010001851030804500308E84F030800000000BB
:101020000000000000000000BCBD0008000000003F
:101030002C510308205103080000000000000000AC
:10104000A4BD000800000000A85203080000000032
:10105000ECBA00080000000004BB0008000000001B
:1010600084550308000000008CBD0008000000004B
:101070009C550308685503080000000000000000AC
:10108000ECC6000800000000B8560308000000008D
:1010900004C700080000000010550308000000000D
:1010A000A4BD000800000000345803080000000040
:1010B000F4BE000800000000ECD60208FCD60208CE
:1010C00068D70208000000000000000000000000D7
:1010D0004CC10008000000004CC4000800000000E3
:1010E00014C9000800000000086A0408000000009D
:1010F0004CC10008000000004CC4000800000000C3
:1011000040B0000820DD04086C6E0408346B04084D
:101110004C8505085CDF02080000000024F8000888
:1011200040B00008DCBB0008C4BB00081CBB0008C2
:1011300020DD04086C6E0408346B04084C85050837
:1011400040E1020858E1020814C90008000000004C
:10115000FCD60508000000004CC10008000000009B
:101160004CC10008000000000CC200080000000094
:1011700040B0000814C9000800000000A8D9040805
:10118000000000004CC10008000000004CC1000835
:10119000000000000CC2000800000000A4C9000804
:1011A0000000000068C10408B0D504081005050857
:1011B000B4C5040814640508F0F804080000000031
:1011C000000000000000000000000000000000001F
:1011D0000000000014C90008000000009C30050851
:1011E000000000004CC10008000000004CC10008D5
:1011F000000000000CC20008000000008CC90008BC
:1012000000000000AC41050804C00408B01905083E
:10121000744C05087C8F0508ACDA04087081050859
:10122000C0140508743C050840CF040828BE050812
:10123000CC9605089C960408000000000000000001
:10124000000000000000000000000000000000009E
:10125000000000000000000000000000000000008E
:1012600000000000000000000000000084BF000833
:1012700000000000586C0308206C0308AC6B0308E6
:10128000746B030800000000000000000000000074
:10129000000000004CC100080000000024C200084B
:1012A0000000000014F60408982C0508142905080D
:1012B000E0AF05089CDE04084CC104080CC104081A
:1012C000249F0508B49B0508A8DA0508D4C40408BF
:1012D000B0920508BC6604088CAD0408000000004C
:1012E00000000000000000000000000000000000FE
:1012F00000000000000000000000000000000000EE
:1013000000000000000000000000000000000000DD
:10131000000000004CC4000800000000CCC8000819
:10132000000000000CEE040834D4040820A80408CF
:101330000000000000000000000000004CCD00088C
:1013400000000000F49503080000000074C00008CD
:1013500000000000F4950308000000001CC4000811
:1013600000000000F49503080000000024C20008FB
:101370000000000044A10508F86E050864CE0508C9
:10138000F49503089CDE040828DB04080CC104085B
:10139000180E05087C930408685F0408BC5B040809
:1013A00010DB050804B7050878C404080000000035
:1013B000000000000000000000000000000000002D
:1013C000000000000000000000000000000000001D
:1013D000000000000000000000000000000000000D
:1013E0000000000014C9000800000000A0A10508CA
:1013F000000000004CC10008000000006CCB000899
:10140000000000004CA20508840E05080000000042
:1014100000000000ACC100080000000034420508D4
:10142000000000004CC10008000000000CC20008D1
:10143000000000001CCA000800000000240B050882
:10144000E4BB0408000000000000000054C20008D3
:101450000000000028C80408EC580508546D040872
:10146000FC1D050800000000000000000000000056
:10147000000000004CC1000800000000CCC80008BB
:101480000000000090810508007A0508E8CB0408F8
:10149000000000000000000000000000CCC80008B0
:1014A00000000000D8FF040884D205080C9F04083F
:1014B0000000000000000000000000004CCD00080B
:1014C00000000000BCFF04080000000074C0000819
:1014D00000000000A4850408000000001CC40008EF
:1014E00000000000BCFF0408000000004CC1000820
:1014F0000000000040B0000834CD000820DD0408E2
:101500006C6E0408346B04084C85050800E302087F
:1015100024E3020840E3020864E3020880E30208CF
:101520000300560034F8000800000000000000002E
:1015300000000000000000000000000000000000AB
:10154000000000000000000000000000000000009B
:10155000000000000000000000000000000000008B
:10156000000000000000000000000000000000007B
:10157000000000000000000000000000000000006B
:10158000000000000000000000000000000000005B
:10159000000000000000000000000000000000004B
:1015A000000000000000000000000000000000003B
:1015B000000000000000000000000000000000002B
:1015C000000000000000000000000000000000001B
:1015D000000000000000000000000000000000000B
:1015E00000000000000000000000000000000000FB
:1015F00000000000000000000000000000000000EB
:1016000000000000000000000000000000000000DA
:1016100000000000000000000000000000000000CA
:1016200000000000000000000000000000000000BA
:1016300000000000000000000000000000000000AA
:10164000000000000000000000000000000000009A
:10165000000000000000000000000000000000008A
:10166000000000000000000000000000000000007A
:101670003CF80008F4CA000800000000A4A1040817
:101680000000000034BB00080000000014C900087E
:1016900000000000F0C10508000000004CC1000877
:1016A000000000000F00110044F8000854F8000882
:1016B000D4F80008BCB10508ECEE04086C6B040813
:1016C0004C850508CCB205081C930408D8EA02082A
:1016D000BCB70408302405088C400508ECEA020871
:1016E00008EB020804A905081CEB020830EB02080D
:1016F00040EB020858EB02080500050054F9000809
:1017000040B0000820DD04086C6E0408346B040847
:101710004C85050870EB02084CC100080000000071
:10172000ECC6000800000000F4950308000000006B
:1017300084C50008000000005CEA04080000000006
:101740002CC90008000000005CEA0408DCD205088F
:10175000D05A050878CF05080000000000000000FE
:101760000000000000000000000055008CF9000897
:101770000000000000000000000000000000000069
:101780000000000000000000000000000000000059
:101790000000000000000000000000000000000049
:1017A0000000000000000000000000000000000039
:1017B0000000000000000000000000000000000029
:1017C0000000000000000000000000000000000019
:1017D0000000000000000000000000000000000009
:1017E00000000000000000000000000000000000F9
:1017F00000000000000000000000000000000000E9
:1018000000000000000000000000000000000000D8
:1018100000000000000000000000000000000000C8
:1018200000000000000000000000000000000000B8
:1018300000000000000000000000000000000000A8
:101840000000000000000000000000000000000098
:101850000000000000000000000000000000000088
:101860000000000000000000000000000000000078
:101870000000000000000000000000000000000068
:101880000000000000000000000000000000000058
:101890000000000000000000000000000000000048
:1018A0000000000000000000000000000000000038
:1018B0000000000000000000000000000000000028
:1018C0009CF9000815001500B4F9000840B00008A4
:1018D00020DD04086C6E0408346B04084C85050890
:1018E000A8EB0208DCEB020814C9000800000000A5
:1018F000A8D90408000000004CC100080000000046
:101900004CCD000800000000C47F04080000000067
:101910001CC4000800000000C47F04080000000090
:101920000F001000F0040108CCF90008BCB1050854
:101930006C6E0408841903084C850508CCB20508B0
:101940001C930408C4190308BCB70408986F050861
:10195000D0190308081A03081C1A030804A905086B
:10196000301A03085C1A03086C1A0308841A030867
:101970009CC5000800000000243D05080000000090
:101980003CBF0008000000007038050810A70508DB
:101990003C8C0408C091050804A9050880B204081D
:1019A000905A050844210508243D05088C40050887
:1019B000986F0508BCB70408F49503081C93040845
:1019C000CCB205080000000000000000000000008C
:1019D0000000000000000000000000000000000007
:1019E00000000000000000000000000000000000F7
:1019F00000000000000000000000000000000000E7
:101A000084C800080000000070380508E860040879
:101A100010A70508980405083C8C0408C091050827
:101A200004A9050880B20408F4950308905A050833
:101A30008C9F050844210508243D050864E7040837
:101A40008804050874DA0508E00305088C400508D9
:101A5000986F0508BCB70408D49D0508F4950308E1
:101A6000E4A905081C930408CCB205080000000096
:101A70000000000000000000000000000000000066
:101A80000000000000000000000000000000000056
:101A90000000000000000000000000000000000046
:101AA0000000000000000000000000000000000036
:101AB0000000000000000000000000000000000026
:101AC0000000000000000000000000000000000016
:101AD0004CCD00080000000054C0050800000000C4
:101AE0001CC400080000000054C0050800000000ED
:101AF00004C1000800000000C41F0508D0D6050876
:101B0000F416050840FF0408C0920408B0660508F2
:101B100018130508ACB10408ACB4040880E7040845
:101B20001CD80508AC5304081CB705081CAC0508F4
:101B300000000000000000000000000000000000A5
:101B40000000000000000000000000000000000095
:101B50000000000000000000000000000000000085
:101B600000000000000000004CC100080000000060
:101B70009CC5000800000000D4D705080000000044
:101B80003CBF0008000000001C6B0508ACC605083F
:101B900064910408BCC4040804A9050880B20408C0
:101BA000905A050864A20408D4D7050824E504085F
:101BB00070270508FC8C050854E90408BC5104088A
:101BC000C4AA05080000000000000000000000009A
:101BD0000000000000000000000000000000000005
:101BE00000000000000000000000000000000000F5
:101BF00000000000000000000000000000000000E5
